:020000040800F2
:100000000020001045060308AD06030855530008FC
:10001000AD060308AD060308AD06030800000000A6
:10002000000000000000000000000000AD06030812
:10003000AD06030800000000AD0603084168000893
:10004000AD060308AD060308AD060308AD060308B8
:10005000AD060308AD060308E923000815250008CE
:10006000D92400089D24000861240008E53B00080D
:10007000D53B0008C53B0008B53B0008A53B000880
:10008000913B00087D3B0008AD060308AD06030860
:10009000AD060308AD060308AD06030825240008D5
:1000A000A5590008E5590008955900080D5A00089F
:1000B000D5590008C5590008B5590008AD06030810
:1000C000AD060308AD060308AD060308AD06030838
:1000D000AD06030835120008B91100083D110008EB
:1000E000AD230008AD060308AD060308AD060308FE
:1000F000AD060308AD060308AD060308AD06030808
:10010000000000000000000000000000AD06030831
:10011000AD060308AD06030899DB02087DDB020883
:10012000693B0008553B0008413B00082D3B000897
:10013000193B0008AD0603080000000000000000A5
:10014000AD060308AD060308AD0603080000000075
:10015000000000000000000000000000000000009F
:100160000000000000000000AD060308AD06030813
:10017000AD060308000000000000000000000000C1
:0801800000000000AD060308B9
:1001880070B4EFF31186502383F31288436B1A6817
:10019800D20720D45D686DB9446A826A944217D048
:1001A80081691144D9600ED9A21A5A60846200226A
:1001B80080F850201A6842F00102F1B21A6081F307
:1001C800118870BC704701698A1A5A608562EEE727
:1001D800012380F85030F1B281F3118870BC704768
:1001E800436A8269D154436A0169426B01338B4285
:1001F80028BF00234362002A2FD0EFF31181502338
:1002080083F31288436B1A68D2072CD470B45E68E3
:100218006EB9456A826A954217D084691444DC60D5
:100228000ED9AA1A5A608562002280F850201A68EE
:1002380042F00102C9B21A6081F3118870BC70479C
:100248000469A21A5A608662EEE7012380F85030EA
:10025800C9B281F3118870BC7047C26C136843F04F
:10026800800313607047C9B281F31188704700BFDB
:10027800026B10B462B1036CC2684469D11A013BC5
:10028800615C5DF8044B08BF13460364C8B270474D
:10029800016A4369C4685B5C0131A14228BF114609
:1002A80001625DF8044BD8B2704700BF436B13B1CD
:1002B80090F850007047836A406A181AB0FA80F0C4
:1002C80040097047416A836A99420AD3CB1A416B45
:1002D800026961B14968501E0B4483420AD2C01AB0
:1002E800704702691144CB1A416B0029F2D1501EA4
:1002F800C01A704700207047036B43B1026C5B68FB
:1003080093422FBF981AC0689B1AC0187047C269D9
:10031800036A9A422FBFD01AC0688018C01A704763
:100328000A4B30B503F1140493F900205D78072ACD
:10033800C8BF143A811804330D7313F8025C85544E
:1003480013F8012C0A76A342EED130BDEC2E030837
:1003580003682DE9F041DF691FB13B46BDE8F04174
:100368001847002A164611DD04460D460E4400E0E3
:1003780023689B68204698470028F9D0236815F819
:10038800011B1B6820469847AE42F1D1BDE8F081B9
:1003980000232322027043708370C37070472D239B
:1003A80043702E2303712F23C3717047F0B48489DF
:1003B8004FF6FF764FF47A740BB300292ED00F78DE
:1003C800013101E0B44217D00589013CAD07A4B260
:1003D800F8D507734FF47A7402E0BCB2B4420BD07C
:1003E8000589ED0704F1FF37F7D5057BEDB20AB1B2
:1003F80015700132013BDFE7094B984202D001201A
:10040800F0BC7047074A538B01339BB25383508B20
:1004180080B2003018BF0120F0BC7047FF27D3E737
:10042800003800402067002040F2E93300E09BB12B
:100438000289013B12F0020F9BB2F8D0017340F21F
:10044800E93300E043B10289013B12F0010F9BB28E
:10045800F8D0007BC0B27047064B984201D0FF200D
:100468007047054A538B01339BB25383508BC0B2FC
:10047800704700BF0038004020670020002870B592
:100488001EDB0928044620DD012303EB83035B0000
:10049800B0FBF3F2092AF8D87BB10E4EB4FBF3F0A7
:1004A8000928CCBF57223022A6FB03E5024403FBF0
:1004B8001044EB0801F8012BF0D100230B7070BD3C
:1004C8002D230B7040420131DBE7303001F8010B7E
:1004D800F3E700BFCDCCCCCC884230B44FF0010458
:1004E8002ED301FB04F4B0FBF4F58D42F9D284B1AC
:1004F800AAB901E0B0FBF4F5092DCCBF5722302290
:100508002A4404FB150003F8012BB4FBF1F4002C7A
:10051800F0D100221A7030BC7047B0FBF4F5092DF9
:10052800CCBF372230222A4404FB150003F8012BE4
:10053800B4FBF1F4002CF0D100221A7030BC7047E3
:100548000546002AEBD1D7E703685A1C02601970E8
:10055800704700BF2DE9F047089C2578002B80469E
:1005680089460CBF4FF0200A4FF0300A661C35B39D
:10057800002A29DD334601E0024698B113F8011B31
:10058800501E0029F8D1971E60B13D46013D5146E5
:100598004046C8476B1C002BF8DC257827EAE77033
:1005A800013055B1041B29464046C847301916F892
:1005B800015B002DF7D1BDE8F087BDE8F087002A80
:1005C80004DC2846BDE8F0870020EBE7571EDCE78F
:1005D80083684268D0ED037A00EB830101339342CC
:1005E80081ED040A836004BF0023836000EB83036A
:1005F80093ED047A036870EE277A9A42C0ED037A85
:1006080077EEC77AC0ED037A0CDA013307EE103AB9
:10061800F8EEC76AB7EE007A87EEA60A036030EEF6
:10062800070A704707EE102AB8EEC77A87EE870ADE
:10063800704700BF90ED057A90ED004AD0ED066A4C
:10064800D0ED014AD0ED047A90ED035AD0ED025A6C
:10065800A4EE007AB0EE406AB0EE470AB0EE667AD1
:10066800A6EE247A67EEC07AA0EE457AE6EE257A01
:1006780080ED057AC0ED067A704700BFD0ED057AA7
:1006880090ED013AD0ED003AD0ED064A90ED024ADD
:1006980090ED077A90ED035A90ED086AD0ED045A70
:1006A800C0ED067AF0EE406A27EE830AC0ED056ACF
:1006B800A3EEA60A80ED087AA4EE240AA5EE470A5E
:1006C800A5EEC60A80ED070A704700BFD0ED007A94
:1006D80090ED017A30EE670AE7EE007AB0EE670A2D
:1006E800C0ED007A704700BF704700BF0A449142CE
:1006F80014D030B40139551E41F2210211F8014FCE
:10070800082380EA042004044CBF82EA4000400029
:10071800013B80B2F7D18D42F0D130BC704700BFA9
:1007280050F8043C012280F84520103803B11847DE
:10073800704700BF90F8203033B1012B03D14FF43C
:1007480000638382704770474FF4806383827047E9
:10075800704700BF704700BF2DE9F04FDFF81CB2AB
:10076800DFF81CE2BBF80020DEF80060BBF90430BB
:10077800BBF90250BBF90A80C2EB261404FB04F44F
:1007880024135200C2EBE60203FB04F305FB02F25A
:100798009B1303EBE223B3F5FA364FEAE37589B00E
:1007A80045F1FF373246A6FB0645CDE9024502FB77
:1007B80007F205EB4202CDE90467029EBBF9084047
:1007C800039208FB02FC4FEAE87906FB09CC3A469B
:1007D800A8FB0689049ECBF81830E51704FB02F243
:1007E80006FB0522A4FB0667E14417444FEA1822DA
:1007F80042EA096200924FEA292201923D03DDE9AB
:100808000078340345EA16553F19BBF80660069090
:1008180048EB05083C1C48F5004503EB8302A4FBA4
:10082800068906FB0599803213124FEA69064FEADA
:10083800E977079356EA07038A4600F09280DDE9D4
:100848000489BBF90E20DEF80440BBF910004946C4
:10085800C4F5801ED317DDE9024502FB01F108FB50
:100868000311A2FB08230B444FEA43492B46C11747
:1008780000FB03F304FB0133A0FB0401BBF90C40AC
:100888001944E30001937346DC170023009349EAF7
:10089800D2394FEA4248DDE9002310EB080041EB6A
:1008A8000901E50712184FEACE744B4145EA5E0587
:1008B800A41A65EB0305221945EB050312196B41D0
:1008C80099019001801841EA926159418B00820098
:1008D80043EA9073101943EB05018B00820043EA49
:1008E800907310460019194632463B4669412FF06D
:1008F800D1FCBBF916204C13450B45EAC14502FB58
:1009080004F6D31705FB0366A2FB05233344BBF9A2
:10091800146002FB04F405FB034406FB01FEA2FB82
:100928000523F717234400FB07EE540EA6FB0067C8
:10093800774444EAC3144FEAD64800194FEA63657E
:1009480048EA473869414FEAE74918EB0008BBF91C
:10095800124049EB01094FEA182646EA09662001C8
:100968003618069B0BB1360A1E60BAF1000F02D08A
:10097800079BCAF8003009B0BDE8F08F583E002048
:1009880074230020704700BF2DE9F041364F374DE2
:10099800B7F80AC02A893B89B7F91240B7F914E0B9
:1009A800EE68B7F90250B7F90E80A2EB0C0203FB10
:1009B80002F3DA139644E30293FBFEF31344A3F520
:1009C8007A6E0EFB0EF4B7F90CC0FB6122130EFB16
:1009D80005F5B7F9044002FB08F8ED1202FB0CF22A
:1009E800B7F900C00EFB04F405EBE825B7F920E0E1
:1009F800FF88121402EB643205EB8C0505FA0EF53C
:100A08000232023592104CF25034A6EBA50502F5DD
:100A1800004244FA0EF404FB05F407FB02F2D20B81
:100A2800002CB9BFB4FBF2F252006400B4FBF2F23E
:100A3800141204FB04F50E4E40F6DE3404FB05F4F4
:100A480003EB830306FB02F524145B0004EB254447
:100A5800083304F6CF641B1102EB241200B10260C4
:100A680001B10B60BDE8F081243E00207423002012
:100A780043E3FFFF2DE9F04FDFF8F8C1DFF8F8E1B5
:100A8800BCF80A70DEF81060BCF80C30BCF808A09E
:100A98003C028BB0361B4FF00004CDE90034009CBB
:100AA800BCF806304FEA17654FF0000767EB0507FB
:100AB800B946B046A4FB06670024CDE90634009C7D
:100AC800002304FB09770024CDE90034AAFB08239E
:100AD800CDE90223039AF30D00930AFB092303933C
:100AE800009B43EA47230093029B4FEAD31AFB1566
:100AF8000193039B4AEA436ADDE9002344464D46D5
:100B0800CDE90845069C12F5FA62A4FB086743F193
:100B1800000304FB0977CDE90623BCF80440039BD6
:100B2800BCF802204FEAE31B230C0593230404932B
:100B3800340A44EA07643D12DDE904674FEAC23823
:100B480016EB0A0647EB0B0718EB0408DDE9063439
:100B58004FEA524949EB0509B3F5FA6F74F10004FD
:100B6800B246BB463CDADDE90067BC00B20044EAA5
:100B78009673B41847EB030522463C462B4602FB06
:100B880004F406FB0344A2FB06232344940844EA26
:100B980083749D105B104FEA3202B8EB040869EBCE
:100BA8000509BAEB020A6BEB030BDDE90623304CAF
:100BB8004FF0FF35A242AB412CDBDDE90856A5FB1F
:100BC800052305FB06F403EB4403D40F44EA43046E
:100BD800DD17DDE90623121B63EB0503CDE90623C8
:100BE800DEF81440A4FB082304FB0933540D44EA3F
:100BF800C3245D15B4EB0A0A65EB0B0B4FEADA3335
:100C080043EA4B4300B1036009B1069B0B600BB08C
:100C1800BDE8F08F40F6AC52B4184FF0000347EB34
:100C280003052246A2FB022304FB05F403EB44035D
:100C3800941843EB0305A4185D414FEA850CA60000
:100C48004CEA947CB41A6CEB0305DF00D6006D10F7
:100C58004FEA340447EA5277921B63EB0703B8EB79
:100C6800040869EB05091AEB020A4BEB030BA4E72E
:100C780024FAFFFF483E00207423002070B5044684
:100C880082B01430E56D06236A464321A847B0B107
:100C98009DF804009DF800609DF801109DF8025031
:100CA8009DF803209DF8053041EA062143EA002318
:100CB80042EA0522A187E287A4F84030012002B069
:100CC80070BD00BF70B5044682B00830656A06235F
:100CD8006A463B21A847A8B19DF804009DF800602A
:100CE8009DF801109DF802509DF803209DF80530ED
:100CF80041EA062143EA002342EA0522E1822283EF
:100D08006383012002B070BD10B490E80600047B34
:100D180040690223A3404B6013685DF8044B4FF60B
:100D2800FE710B401360FFF72BBA00BF70B4046864
:100D3800037B2268022101FA03F31A4213D04269A5
:100D48000A49582000FB02124FF6FE765068528975
:100D5800C5680068296831402960C168D24392B2E9
:100D68000A40C260636070BC704700BF846A00209C
:100D780030B4094B1C7864B1084B002503EBC4045C
:100D88001A6899885562D06808330143A342D16034
:100D9800F6D130BC704700BF446D0020486D00207C
:100DA80010B40268047B11680223A340194209D0D9
:100DB8000649406800240C7001684FF6FE74214013
:100DC800016053605DF8044B704700BF93590020E1
:100DD800F0B4334C00EB800004EB80046468002C12
:100DE8005BD0304E49004FF42040CDB2B061A169CC
:100DF800090444D460682C4F45F08071384041F4B0
:100E0800903101434FF420406160B06103E0411E1E
:100E1800002838D00846A1698F07F8D54FF420403C
:100E2800A262B06102E0421E68B31046A2691106D0
:100E3800F9D562681C4945F0007545F480350A40CB
:100E480015434FF420406560B06102E0421ED0B106
:100E58001046A2699207F9D5A362A3694FF420400E
:100E68009B06B06105D4431E68B11846A3699B066A
:100E7800F9D52023B061E3610120F0BC7047411E21
:100E880008B10846B3E7094A138801339BB24FF00B
:100E9800FF31B1611380F0BC70472046F0BC704749
:100EA8009860002074230020009800FC104A00205D
:100EB800134600200A4668218AE700BF30B5044679
:100EC800C06C61710368A26823F00103036087B0F6
:100ED800A379009213F004023DD04FF4805213F02E
:100EE8000203019244D102934FF4806300220393DA
:100EF80011F00103059237D1049308238D07694641
:100F080048BF049323F0FCFD6079E36CA17900F0FD
:100F18000202002A15BF4FF440324FF480324FF4DA
:100F28000034002410F0010F586808BF2246CC078F
:100F38004CBF024320EA02025A609A6809074CBF74
:100F480042F0080222F008029A601A6842F0010290
:100F58001A6007B030BD13F0020301920BD04FF4B2
:100F6800005513460295C1E7042304930C23C5E7F3
:100F78004FF40053B7E70293B8E700BF10B5044633
:100F8800C06CA160036823F001030360A37986B0F5
:100F980013F00402009141D04FF4805213F0020381
:100FA800019244D102934FF4806362790393D1078D
:100FB8004FF000030493059345BF042304930823CB
:100FC8000C236946920748BF049323F099FD607982
:100FD800E36CA17900F00202002A15BF4FF44032F9
:100FE8004FF480324FF40034002410F0010F586899
:100FF80008BF2246CC074CBF024320EA02025A60CF
:101008009A6809074CBF42F0080222F008029A6069
:101018001A6842F001021A6006B010BD13F002030C
:10102800019207D04FF4005113460291BDE74FF4E7
:101038000053B7E70293B8E7002326220360027043
:1010480027228270012243600271837170472DE963
:10105800F341056906460F467DBBD0F80080C8F30A
:101068000A0323B30023D6F8008001931FF068FC1D
:10107800042819D1214C236943F001032361BBB231
:10108800A8F800301FF05CFC04282ED108F10203F8
:101098000193019B3F0C1F801FF052FC2369042819
:1010A80023F00103236125D06FF0010505E01FF04F
:1010B80047FC042805D04FF0FF35284602B0BDE8AC
:1010C800F0810E4C236943F002032361C4F81480B5
:1010D800236943F0400323611FF032FC236904288D
:1010E80023F002032361BDD0E5E7236923F0010360
:1010F8002361D9E7336804333360DEE70020024018
:10110800F8B504460D468E180027B54201D120696E
:10111800F8BDE368591CE160234415F8012B1A72E5
:101128000429F2D1A1682046FFF791FFE76020610A
:10113800EBE700BF1D4B70B59C68E36C226BDD6963
:10114800C2B1636B2BB12B0702D5E36C08221A627C
:1011580070BD2A06F7D5A26A616A8A421FD0511C5F
:10116800A069A162825C2069E66C81423285EAD37B
:10117800A362E8E7A906E4D5E26A1AB1988C80B2BE
:101188009047DEE7E1699B8C6069DBB24E1CE66143
:101198004354E169E368994228BFE261D1E7E26C10
:1011A800136823F080031360CDE700BFCC31002023
:1011B8001D4B70B55C68E36C226BDD69C2B1636B73
:1011C8002BB12B0702D5E36C08221A6270BD2A06E0
:1011D800F7D5A26A616A8A421FD0511CA069A16230
:1011E800825C2069E66C81423285EAD3A362E8E733
:1011F800A906E4D5E26A1AB1988C80B29047DEE776
:10120800E1699B8C6069DBB24E1CE6614354E1697D
:10121800E368994228BFE261D1E7E26C136823F0E2
:1012280080031360CDE700BFCC3100201D4B70B5A3
:101238001C68E36C226BDD69C2B1636B2BB12B07B1
:1012480002D5E36C08221A6270BD2A06F7D5A26A95
:10125800616A8A421FD0511CA069A162825C206920
:10126800E66C81423285EAD3A362E8E7A906E4D5B1
:10127800E26A1AB1988C80B29047DEE7E1699B8CEC
:101288006069DBB24E1CE6614354E169E368994248
:1012980028BFE261D1E7E26C136823F08003136092
:1012A800CDE700BFCC31002003685B6A03B1184763
:1012B800704700BF03681B6A03B11847704700BF37
:1012C80003682DE9F041DF691FB13B46BDE8F041F5
:1012D8001847002A164611DD04460D460E4400E064
:1012E80023689B68204698470028F9D0236815F89A
:1012F800011B1B6820469847AE42F1D1BDE8F0813A
:1013080003689B69184700BF03685B69184700BFFB
:101318000368DB68184700BF03689B68184700BF6D
:1013280003685B68184700BF03681B68184700BF5D
:10133800014B1868F8E700BFA4720020054B53F86A
:10134800203033B11A689B88918A0B4218BF1B045E
:1013580093617047C460002003682DE9F04F03F1E2
:101368003845644EAD0A0124755D05F01F066D0908
:10137800022D04FA06F400F0A280032D00F0A480E8
:10138800012D52D08088B0FA80F4C4F11F04A4B2B1
:10139800E50803EB850504F007042E6AA4000F276F
:1013A800A74026EA07062E622E6A01F0030702FA12
:1013B80004F47A1E3443012AC1F3810CC1F30018E6
:1013C8002C62C1F3411135D9C60700F19780850712
:1013D80000F1A380440700F1B180020700F1BF804B
:1013E800C60600F1CD80850600F1DB80440600F1D9
:1013F800E980020600F1F780C60500F10581850540
:1014080000F11381440500F12181020500F12F81CB
:10141800C60400F13D81850400F14B81440400F1CC
:101428005981020455D4BDE8F08F334D6E693443B9
:101438006C61A7E7002422464FF0010E4FF0030924
:1014480004E00132102A04F10204ECD00EFA02F68C
:1014580036EA0005F5D1D3F808A009FA04F5ED43FA
:101468000AEA050AC3F808A0D3F808B00CFA04FA87
:101478004AEA0B0AC3F808A0B3F804A01FFA8AFACC
:101488002AEA06069E80B3F804A008FA02F646EA9D
:101498000A06B6B29E801E682E401E60D3F800A0D1
:1014A80007FA04F646EA0A061E60D3F80CA001FA09
:1014B80004F605EA0A0A46EA0A05DD60C1E70E4DA8
:1014C800AE693443AC615DE70B4DEE693443EC61C2
:1014D80058E71A6822F040421A601A6842EA877789
:1014E8001F60DA6822F0404242EA8171D960BDE8A3
:1014F800F08F00BF50590308001002401A6822F00C
:1015080003021A601A683A431A60DA6822F0030282
:101518000A438507DA607FF55DAF1A6822F00C028E
:101528001A601A6842EA87021A60DA6822F00C0226
:1015380042EA81024407DA607FF54FAF1A6822F069
:1015480030021A601A6842EA07121A60DA6822F052
:10155800300242EA0112DA6002077FF541AF1A68E9
:1015680022F0C0021A601A6842EA87121A60DA6822
:1015780022F0C00242EA8112C606DA607FF533AF74
:101588001A6822F440721A601A6842EA07221A603E
:10159800DA6822F4407242EA01228506DA607FF5B1
:1015A80025AF1A6822F440621A601A6842EA872254
:1015B8001A60DA6822F4406242EA81224406DA605C
:1015C8007FF517AF1A6822F440521A601A6842EA87
:1015D80007321A60DA6822F4405242EA0132DA60CD
:1015E80002067FF509AF1A6822F440421A601A68A9
:1015F80042EA87321A60DA6822F4404242EA8132CB
:10160800C605DA607FF5FBAE1A6822F440321A602C
:101618001A6842EA07421A60DA6822F4403242EA5B
:1016280001428505DA607FF5EDAE1A6822F44022A2
:101638001A601A6842EA87421A60DA6822F440227D
:1016480042EA81424405DA607FF5DFAE1A6822F487
:1016580040121A601A6842EA07521A60DA6822F4DD
:10166800401242EA0152DA6002057FF5D1AE1A68EB
:1016780022F440021A601A6842EA87521A60DA684D
:1016880022F4400242EA8152C604DA607FF5C3AE12
:101698001A6822F040721A601A6842EA07621A60F1
:1016A800DA6822F0407242EA01628504DA607FF566
:1016B800B5AE1A6822F040621A601A6842EA876278
:1016C8001A60DA6822F0406242EA81624404DA6011
:1016D8007FF5A7AE1A6822F040521A601A6842EAEB
:1016E80007721A60DA6822F0405242EA0172DA6040
:1016F80097E600BF036803F138422DE9F04F920ADC
:10170800584DAA5C02F01F0552090124022A04FA66
:1017180005F400F08C80032A00F08E80012A3CD06A
:1017280001F003077A1E012AC1F3810CC1F30018E6
:101738008088C1F3411135D9C60700F19780850724
:1017480000F1A380440700F1B180020700F1BF80D7
:10175800C60600F1CD80850600F1DB80440600F165
:10176800E980020600F1F780C60500F105818505CC
:1017780000F11381440500F12181020500F12F8158
:10178800C60400F13D81850400F14B81440400F159
:101798005981020455D4BDE8F08F334A55692C436A
:1017A8005461BDE7002422464FF0010E4FF00309B3
:1017B80004E00132102A04F10204ECD00EFA02F619
:1017C80036EA0005F5D1D3F808A009FA04F5ED4387
:1017D8000AEA050AC3F808A0D3F808B00CFA04FA14
:1017E8004AEA0B0AC3F808A0B3F804A01FFA8AFA59
:1017F8002AEA06069E80B3F804A008FA02F646EA2A
:101808000A06B6B29E801E682E401E60D3F800A05D
:1018180007FA04F646EA0A061E60D3F80CA001FA95
:1018280004F605EA0A0A46EA0A05DD60C1E70E4A37
:1018380095692C43946173E70B4AD5692C43D461AD
:101848006EE71A6822F040421A601A6842EA8777FF
:101858001F60DA6822F0404242EA8171D960BDE82F
:10186800F08F00BF50590308001002401A6822F098
:1018780003021A601A683A431A60DA6822F003020F
:101888000A438507DA607FF55DAF1A6822F00C021B
:101898001A601A6842EA87021A60DA6822F00C02B3
:1018A80042EA81024407DA607FF54FAF1A6822F0F6
:1018B80030021A601A6842EA07121A60DA6822F0DF
:1018C800300242EA0112DA6002077FF541AF1A6876
:1018D80022F0C0021A601A6842EA87121A60DA68AF
:1018E80022F0C00242EA8112C606DA607FF533AF01
:1018F8001A6822F440721A601A6842EA07221A60CB
:10190800DA6822F4407242EA01228506DA607FF53D
:1019180025AF1A6822F440621A601A6842EA8722E0
:101928001A60DA6822F4406242EA81224406DA60E8
:101938007FF517AF1A6822F440521A601A6842EA13
:1019480007321A60DA6822F4405242EA0132DA6059
:1019580002067FF509AF1A6822F440421A601A6835
:1019680042EA87321A60DA6822F4404242EA813257
:10197800C605DA607FF5FBAE1A6822F440321A60B9
:101988001A6842EA07421A60DA6822F4403242EAE8
:1019980001428505DA607FF5EDAE1A6822F440222F
:1019A8001A601A6842EA87421A60DA6822F440220A
:1019B80042EA81424405DA607FF5DFAE1A6822F414
:1019C80040121A601A6842EA07521A60DA6822F46A
:1019D800401242EA0152DA6002057FF5D1AE1A6878
:1019E80022F440021A601A6842EA87521A60DA68DA
:1019F80022F4400242EA8152C604DA607FF5C3AE9F
:101A08001A6822F040721A601A6842EA07621A607D
:101A1800DA6822F0407242EA01628504DA607FF5F2
:101A2800B5AE1A6822F040621A601A6842EA876204
:101A38001A60DA6822F0406242EA81624404DA609D
:101A48007FF5A7AE1A6822F040521A601A6842EA77
:101A580007721A60DA6822F0405242EA0172DA60CC
:101A680097E600BF10B50409013C052C17D80D4BAB
:101A780033F8142000F00F0042FA00F313F00103CA
:101A88000DD0012303FA00F0013810402EF052FC6B
:101A9800054A064B125D104403EBC00010BD002040
:101AA80010BD00BFB85C0308C45C0308646800206C
:101AB8002DE9F04F4A484B4B4B4C4FF090414FF0BB
:101AC800010A4FF002094FF004084FF0080C4FF0DC
:101AD800100E20274026802530F8022B12F0010F27
:101AE80003D01960A3F804A0083312F0020F03D042
:101AF8001960A3F80490083312F0040F03D019609A
:101B0800A3F80480083312F0080F03D01960A3F873
:101B180004C0083312F0100F03D01960A3F804E0D2
:101B2800083312F0200F02D019609F80083312F09A
:101B3800400F02D019609E80083312F0800F02D047
:101B480019609D80083312F4807F05D04FF4807BA4
:101B58001960A3F804B0083312F4007F05D04FF4DD
:101B6800007B1960A3F804B0083312F4806F05D025
:101B78004FF4806B1960A3F804B0083312F4006FB7
:101B880005D04FF4006B1960A3F804B0083312F4C1
:101B9800805F05D04FF4805B1960A3F804B0083368
:101BA80012F4005F05D04FF4005B1960A3F804B08D
:101BB800083312F4804F05D04FF4804B1960A3F816
:101BC80004B00833D20B04D04FF4004219609A8055
:101BD800083301F58061A1427FF47EAFBDE8F08F44
:101BE800B85C03086468002000180048002867D023
:101BF80003682DE9F04F03F138445C4EA40A01252F
:101C0800345D04F01F066409022C05FA06F558D065
:101C1800032C00F0A580012C58D08088B0FA80F4FD
:101C2800C4F11F04A4B2E50803EB850504F007041A
:101C38002E6AA4000F27A74026EA07062E622E6AFE
:101C480001F00307A2407C1E3243012CC1F3810C32
:101C5800C1F300182A62C1F341113CD9C60700F14B
:101C68008980850700F19580440700F1A380020769
:101C780000F1B180C60600F1BF80850600F1CD8075
:101C8800440600F1DB80020600F1E980C60500F198
:101C9800F780850500F10581440500F113810205EF
:101CA80000F12181C60400F12F81850400F13D81F6
:101CB800440400F14B81020400F15981BDE8F08F22
:101CC80070472B4CA6693543A561A6E7284C666981
:101CD80035436561A1E7002422464FF0010E4FF01D
:101CE800030904E00132102A04F10204E6D00EFAD6
:101CF80002F636EA0005F5D1D3F808A009FA04F58A
:101D0800ED430AEA050AC3F808A0D3F808B00CFAAC
:101D180004FA4AEA0B0AC3F808A0B3F804A01FFAA9
:101D28008AFA2AEA06069E80B3F804A008FA02F6A0
:101D380046EA0A06B6B29E801E682E401E60D3F898
:101D480000A007FA04F646EA0A061E60D3F80CA0BB
:101D580001FA04F605EA0A0A46EA0A05DD60C1E75F
:101D6800034CE6693543E56157E700BF505903085E
:101D7800001002401A6822F003021A601A683A43F7
:101D88001A60DA6822F003020A438507DA607FF5F1
:101D98006BAF1A6822F00C021A601A6842EA8702CE
:101DA8001A60DA6822F00C0242EA81024407DA601B
:101DB8007FF55DAF1A6822F030021A601A6842EAAD
:101DC80007121A60DA6822F0300242EA0112DA6079
:101DD80002077FF54FAF1A6822F0C0021A601A682E
:101DE80042EA87121A60DA6822F0C00242EA8112D7
:101DF800C606DA607FF541AF1A6822F440721A60AD
:101E08001A6842EA07221A60DA6822F4407242EA43
:101E180001228506DA607FF533AF1A6822F4406242
:101E28001A601A6842EA87221A60DA6822F4406265
:101E380042EA81224406DA607FF525AF1A6822F467
:101E480040521A601A6842EA07321A60DA6822F4C5
:101E5800405242EA0132DA6002067FF517AF1A688B
:101E680022F440421A601A6842EA87321A60DA6835
:101E780022F4404242EA8132C605DA607FF509AFB2
:101E88001A6822F440321A601A6842EA07421A6055
:101E9800DA6822F4403242EA01428505DA607FF5C9
:101EA800FBAE1A6822F440221A601A6842EA874296
:101EB8001A60DA6822F4402242EA81424405DA6074
:101EC8007FF5EDAE1A6822F440121A601A6842EAE9
:101ED80007521A60DA6822F4401242EA0152DA60C4
:101EE80002057FF5DFAE1A6822F440021A601A680C
:101EF80042EA87521A60DA6822F4400242EA8152C2
:101F0800C604DA607FF5D1AE1A6822F040721A6012
:101F18001A6842EA07621A60DA6822F0407242EAF6
:101F280001628504DA607FF5C3AE1A6822F0406268
:101F38001A601A6842EA87621A60DA6822F0406218
:101F480042EA81624404DA607FF5B5AE1A6822F08D
:101F580040521A601A6842EA07721A60DA6822F078
:101F6800405242EA0172DA6002047FF5A7AE1A68AD
:101F780022F040421A601A6842EA87771F60DA68DE
:101F880022F0404242EA8171D960BDE8F08F00BF7B
:101F9800002852D0036803F138422DE9F04F920A25
:101FA800504DAA5C02F01F0552090124022A04FAC6
:101FB80005F443D0032A00F09080012A43D001F0B1
:101FC80003077A1E012AC1F3810CC1F30018808827
:101FD800C1F341113CD9C60700F18880850700F19B
:101FE8009480440700F1A280020700F1B080C60681
:101FF80000F1BE80850600F1CC80440600F1DA804D
:10200800020600F1E880C60500F1F680850500F1BA
:102018000481440500F11281020500F12081C60403
:1020280000F12E81850400F13C81440400F14A81CD
:10203800020400F15881BDE8F08F70472A4A95697B
:102048002C439461BBE7284A55692C435461B6E791
:10205800002422464FF0010E4FF0030904E001323C
:10206800102A04F10204E6D00EFA02F636EA000558
:10207800F5D1D3F808A009FA04F5ED430AEA050AF0
:10208800C3F808A0D3F808B00CFA04FA4AEA0B0A15
:10209800C3F808A0B3F804A01FFA8AFA2AEA0606C9
:1020A8009E80B3F804A008FA02F646EA0A06B6B219
:1020B8009E801E682E401E60D3F800A007FA04F622
:1020C80046EA0A061E60D3F80CA001FA04F605EAEF
:1020D8000A0A46EA0A05DD60C1E7034AD5692C43C6
:1020E800D4616CE750590308001002401A6822F0C6
:1020F80003021A601A683A431A60DA6822F0030287
:102108000A438507DA607FF56CAF1A6822F00C0283
:102118001A601A6842EA87021A60DA6822F00C022A
:1021280042EA81024407DA607FF55EAF1A6822F05E
:1021380030021A601A6842EA07121A60DA6822F056
:10214800300242EA0112DA6002077FF550AF1A68DE
:1021580022F0C0021A601A6842EA87121A60DA6826
:1021680022F0C00242EA8112C606DA607FF542AF69
:102178001A6822F440721A601A6842EA07221A6042
:10218800DA6822F4407242EA01228506DA607FF5B5
:1021980034AF1A6822F440621A601A6842EA872249
:1021A8001A60DA6822F4406242EA81224406DA6060
:1021B8007FF526AF1A6822F440521A601A6842EA7C
:1021C80007321A60DA6822F4405242EA0132DA60D1
:1021D80002067FF518AF1A6822F440421A601A689E
:1021E80042EA87321A60DA6822F4404242EA8132CF
:1021F800C605DA607FF50AAF1A6822F440321A6021
:102208001A6842EA07421A60DA6822F4403242EA5F
:1022180001428505DA607FF5FCAE1A6822F4402297
:102228001A601A6842EA87421A60DA6822F4402281
:1022380042EA81424405DA607FF5EEAE1A6822F47C
:1022480040121A601A6842EA07521A60DA6822F4E1
:10225800401242EA0152DA6002057FF5E0AE1A68E0
:1022680022F440021A601A6842EA87521A60DA6851
:1022780022F4400242EA8152C604DA607FF5D2AE07
:102288001A6822F040721A601A6842EA07621A60F5
:10229800DA6822F0407242EA01628504DA607FF56A
:1022A800C4AE1A6822F040621A601A6842EA87626D
:1022B8001A60DA6822F0406242EA81624404DA6015
:1022C8007FF5B6AE1A6822F040521A601A6842EAE0
:1022D80007721A60DA6822F0405242EA0172DA6044
:1022E80002047FF5A8AE1A6822F040421A601A6804
:1022F80042EA87771F60DA6822F0404242EA817139
:10230800D960BDE8F08F00BF10B1036882881A85D4
:10231800704700BF10B1036882889A61704700BF98
:1023280010B5014600BF074C23689868FFF7ECFF1B
:1023380023685868FEF778F823689868FFF7EAFF7B
:1023480000BF10BD5067002038B10029838802689B
:1023580014BF002110218B409361704710B40A4BC1
:102368000A4A1C7801238340234052F8200029B9E7
:10237800B3FA83F149095DF8044BE5E7191C18BF66
:1023880001215DF8044BDFE7C0600020C460002035
:1023980030B1036882881B8A1A4214BF01200020CA
:1023A800704700BF2DE9F0410B4E356873691D4039
:1023B80010D0DFF828800127B5FA85F4C4F11F048E
:1023C80008EB840307FA04F4D86903689847A5431F
:1023D8007461F1D1BDE8F08100040140742300204C
:1023E8002DE9F0410B4E356873691D4010D0DFF8B8
:1023F80028800127B5FA85F4C4F11F0408EB84038B
:1024080007FA04F4D86903689847A5437461F1D1C1
:10241800BDE8F08100040140742300202DE9F0415B
:102428000B4E356873691D4010D0DFF828800127EE
:10243800B5FA85F4C4F11F0408EB840307FA04F421
:10244800D86903689847A5437461F1D1BDE8F08164
:1024580000040140742300202DE9F0410B4E35683B
:1024680073691D4010D0DFF828800127B5FA85F47C
:10247800C4F11F0408EB840307FA04F4D86903685D
:102488009847A5437461F1D1BDE8F081000401408B
:10249800742300202DE9F0410B4E356873691D4007
:1024A80010D0DFF828800127B5FA85F4C4F11F049D
:1024B80008EB840307FA04F4D86903689847A5432E
:1024C8007461F1D1BDE8F08100040140742300205B
:1024D8002DE9F0410B4E356873691D4010D0DFF8C7
:1024E80028800127B5FA85F4C4F11F0408EB84039A
:1024F80007FA04F4D86903689847A5437461F1D1D1
:10250800BDE8F08100040140742300202DE9F0416A
:102518000B4E356873691D4010D0DFF828800127FD
:10252800B5FA85F4C4F11F0408EB840307FA04F430
:10253800D86903689847A5437461F1D1BDE8F08173
:102548000004014074230020002800F084802DE955
:10255800F0418488B4FA84F4C4F11F04651C82B085
:102568006BD0E5B205F0FC0606F1804606F580362C
:1025780005F00305D6F808E0374F0068AD004FF0C6
:102588000F0C0CFA05FC2EEA0C0E07EB840CC0F3BA
:102598008720CCF81C10C6F808E0D6F80880DFF8C9
:1025A800C4C0DFF8C4E000FA05F10120A04041EA08
:1025B8000801B160CCF80000DEF80050274EDFF8C3
:1025C800AC80C1430D40CEF8005035680D403560F1
:1025D800DEF80050224E0543CEF80050D8F80050DF
:1025E8000D40C8F800505CF8085C34442940102BB2
:1025F8004CF8081C247DACF1080C21D003F1804371
:1026080003F58233196801431960274497F85C3051
:10261800934212DD2644002196F824308DF80430C8
:102628009411012301A887F85C208DF805408DF8E6
:1026380006108DF8073021F06BFF02B0BDE8F0817D
:10264800D8F800300343C8F80030DCF80010014324
:10265800CCF80010D9E77047742300200404014027
:10266800EC2E030814040140000401400804014052
:1026780070B5044690F85900002833D104F11405C8
:10268800236E80226B2128469847642004F036F890
:10269800236E284603226B219847236E94F8542012
:1026A8001921284698470F2004F028F8236E94F83B
:1026B800522028461A219847236E284618221B21A3
:1026C8009847236E284618221C219847236E2846CF
:1026D8000222372198472846236E01223821BDE877
:1026E80070401847FFF7BEF90546FFF751FE00286E
:1026F800C4D115B12023E871AB7128460021FFF73A
:1027080047FC2146054B41F8103F28460823F02294
:10271800FFF71AFF284623F055F9AFE72907000805
:102728000B490C4A8B6943F0010310B58B611368A0
:10273800094C43F48053136004F11C00402200212B
:1027480030F01BFB4FF0FF33E365C4F85F3010BD7A
:1027580000100240000001407423002003685B6AF7
:10276800184700BF2DE9F041044618460D461646A5
:1027780098462DF0C5F82768E6722844A0722946C5
:102788007D69434632462046AC46BDE8F041604785
:10279800036810B504461B689847236820469B6861
:1027A8009847A37B0133A37310BD00BF10B503681E
:1027B80004469B689847FF2301226373227310BD68
:1027C800427A02B9704710B504460368406804F1BC
:1027D8000A0198470023637210BD00BF437A5A1C50
:1027E8000344D2B242729972037A934200D802B972
:1027F800704710B504460368406804F10A01984719
:102808000023637210BD00BF30B40B4D002305F1E7
:102818002C0101E0272B0CD011F8132082424FEA3B
:10282800430403F10103F5D12C4494F82D0030BC86
:102838007047002030BC7047EC2E030870B5448800
:1028480006460D46C4F30B0422460021284630F004
:1028580094FA3369094A934209D3094A934206D242
:10286800224628461946BDE870402DF071BF23B1B5
:1028780021462846BDE87040184770BD38A00308B7
:102888002BA10308064B07498B4202D300231846A5
:1028980070471A88C2F30B029042F8D01433F3E75A
:1028A800B09B030838A00308024A136823EA000013
:1028B8001060704718400020F8B5174D2B78A32BEF
:1028C80028D16B78BE2B25D1022229464FF6FF70FE
:1028D800FDF70CFF114FAC1C22884AB1A618BE4266
:1028E80018D2052A16D92146FDF700FF3446F3E72A
:1028F80021460222FDF7FAFE0222A118FDF7F6FE94
:102908000634074B641B1C8041F60F53C31A584208
:102918005841F8BD0020F8BD00F003080000040885
:10292800124A00202DE9F04FDFF848914C4F8BB048
:102938000326A7EB09071822002104A830F01DFA86
:10294800484BCDF8109005971A69120604D5464AE7
:102958005A6002F188325A6001228DF8242034220C
:10296800DA60424B424C1B88ADF8003002226946BF
:1029780004A8FEF7C5FB022269464FF6FF70FDF773
:10298800B5FEDFF8F4A080464FF0000B544536D36F
:102998000AAC002524F8245D0222214604A8FEF78B
:1029A800AFFB022221464046FDF7A0FE40BAC043D5
:1029B800ADF80800022202A904A8FEF7A1FB0798B7
:1029C80060B106ABC0F104022946184430F0D5F9CD
:1029D800069904A8FEF73BFB079508909DF824305C
:1029E800089A23B11F490B6943F080030B61013E2C
:1029F8002DD0002A9FD1FFF75FFF50B32CE06588E8
:102A08008DF80DB0C5F30B05AB1DADF80830238864
:102A1800C3F30B02ADF80A201B0B062202A904A877
:102A28008DF80C30FEF76CFB062202A94046FDF734
:102A38005DFE616880462A4604A8FEF761FB61686E
:102A480040462A46FDF752FE143480469EE7002A87
:102A5800D1D0052003F09AF90BB0BDE8F08F00BF84
:102A6800000004080020024023016745662F030880
:102A7800B09B030800F0030838A003080378202B54
:102A8800024600F10100F9D0092BF7D02D2B2CD0EC
:102A98002B2B03BF5378B7EE000A0246B7EE000AA5
:102AA800A3F13001C8B209289FED467A10D8F2EE9A
:102AB800046A07EE901AF8EEE77A12F8013FE7EE9B
:102AC800267AA3F13001C8B20928B0EE677AF0D9A6
:102AD8002E2B4CD003F0DF03452B0BD0F7EE007AFA
:102AE80067EE276A20EE260A70475378BFEE000A81
:102AF8000246D5E710B451782D2959D02B290ABFA1
:102B08009178501C901C0024A1F13003092B53D854
:102B1800002303EB830301EB430310F8011FA1F12A
:102B28003002092AA3F13003F3D9B3F59A7F28BFFD
:102B38004FF49A73072B42D9DFED236A1A46F7EE52
:102B4800007A083A072A67EEA67AFAD803F007034C
:102B58002BB1F2EE046A013B67EEA67AFBD124B3EF
:102B6800C7EE276A5DF8044B20EE260A70475378B3
:102B7800A3F13001C8B2092802F10102AAD8F2EE85
:102B8800046AF0EE665A07EE901AF8EEE77A12F841
:102B9800013F87EEA66AA3F13001C8B2092866EEA4
:102BA800A56A37EE067AEED994E767EE276AD9E781
:102BB800901C91780124A7E7F7EE007ACFE7F7EEAB
:102BC800007AC5E70000000020BCBE4CB5EEC00A84
:102BD800DFED317AF1EE10FACCBF30EE270A30EE95
:102BE800670ADFED2E7A20EE270A30B5FDEEC07AAF
:102BF80087B017EE904A054684EAE470002303A9DB
:102C0800A0EBE4700193009302931EF0CBF8002C24
:102C1800ACBF20232D2303A88DF800302CF070FEC4
:102C2800012803A924D002282DD0032805BF30236A
:102C3800684668468DF8013030F0C5F868462CF0D3
:102C48005FFE0338C4B222466946284630F019F9B7
:102C580000232B5528462CF053FE2E22431C2A54C1
:102C68000DEB0401E81830F0CBF8284607B030BD6A
:102C7800302368468DF801308DF802308DF8033026
:102C880030F0A1F8DAE7302368468DF801308DF886
:102C9800023030F098F8D1E76F12033A00007A4416
:102CA8002DE9F041064615460846B6FBF2F43CB954
:102CB80005FB1464124B1B5D00F8013BBDE8F08175
:102CC800B4FBF2F767B90E4B05FB174705FB146415
:102CD800DA5D00F8012B1B5D00F8013BBDE8F081CF
:102CE800B7FBF2F8B8F1000F02D04046FFF7D8FF63
:102CF80005FB1878024B13F8082000F8012BE3E7CE
:102D0800345F030830B402681146531C036011F89D
:102D1800024B0160D31C517803609378151D056040
:102D28001B0443EA0123D078234343EA006030BC04
:102D3800704700BF0368591C1A46016012F8021B4D
:102D48000260587841EA0020704700BF03685A1CA7
:102D580002601878704700BF38B504460068154609
:102D68002DF0F6FC22682A44226038BD036810B4AE
:102D78000A0A5C1C04601A7003685A1C0260197005
:102D88005DF8044B704700BF03685A1C026010B41A
:102D9800197003680A0A5C1C04601A7003680A0C3C
:102DA8005C1C04601A700368090E5A1C02601970D2
:102DB8005DF8044B704700BF03685A1C0260197025
:102DC8000368090A5A1C0260197070472DE9F04718
:102DD800002488B080460F461E46A14605AD531C08
:102DE8000393117839B3252933D1931CCDF810906A
:102DF8000393507830284ED04FF0000AA0F13003EA
:102E0800DBB2092B42D96C2819D0642800F09380D2
:102E180024D825281CD063D9582876D063281BD1FC
:102E280031784046B847039A531C03931178043607
:102E380001340029D7D1204608B0BDE8F087039BAC
:102E48005A1C03921B78642B7CD02AD8252B54D18A
:102E5800252140460134B847039AC0E7732833D088
:102E680044D975284FD106F1040E30682B4600224C
:102E78000A217646FDF730FB049A009553463946F9
:102E88004046FDF767FB039A0444A8E704AA03A990
:102E980026F0BEFCB7E7D31C039390784FF0010AE5
:102EA800ACE7732B10D05BD9752B3AD0782B96D121
:102EB800A3F15802B2FA82F2306852092B46102167
:102EC8000436FDF709FBD7E73368049A00933946BF
:102ED80000234046FDF73EFB04360444039A7EE790
:102EE8000028B9D1204608B0BDE8F0876E28B3D1D4
:102EF800039A336804361C6071E72AD9582BD7D057
:102F0800632B8DD06BE77828A6D1A0F15802B2FACE
:102F180082F2306852092B461021FDF7DDFA04369B
:102F2800AAE706F1040E30682B4600220A217646ED
:102F3800FDF7D2FAA0E7331D306829461E46FDF793
:102F48009DFA99E7331D306829461E46FDF796FA23
:102F580092E7002B7FF443AF204608B0BDE8F08726
:102F68006E2BC6D03BE700BF0EB400B584B005ABEE
:102F7800019053F8042B0649039301A8FFF726FF95
:102F8800019B00221A7004B05DF804EB03B070478F
:102F9800510500080FB430B583B006AB0A490B4899
:102FA80053F8042B096800680193FFF70FFF084CDA
:102FB80005462068FEF7A8F90028FAD0284603B08D
:102FC800BDE8304004B07047C0310020C431002053
:102FD800A4720020DFED2B7AB4EEE70AF1EE10FAC6
:102FE8004ADDDFED296A9FED297A01E0B0EE670A34
:102FF800B4EEC70AF1EE10FA70EE667AF6DC9FEDD1
:10300800247AF4EEC77AF1EE10FA38D5DFED1E6AAD
:103018009FED207A01E0F0EE407AF4EEC77AF1EE07
:1030280010FA37EEA60AF6D4DFED1B7AB4EEE70AFB
:10303800F1EE10FA14DDDFED137A37EEC00A60EE18
:10304800006A9FED166A9FED167ADFED167AA6EEF6
:10305800867A20EE266AE6EE877AA6EE270A704779
:10306800DFED117AB4EEE70AF1EE10FA44BFDFEDB6
:10307800087A37EEC00AE2E7F0EE407ABFE7B0EE32
:10308800670AD1E7DB0F4940DB0FC940E4CB1641A3
:10309800DB0F49C0E4CB16C1DB0FC93F92E741B94A
:1030A8009730083C15A82ABEDB0FC9BF80EAE07339
:1030B800A3EBE0738B4205DB002801DD401A704763
:1030C80002D17047002070470844704709B909E0E9
:1030D800194690FBF1F301FB13030846002BF7D1C7
:1030E800084670470146FBE79FED317A70EE077A94
:1030F800FDEEE76A16EE903A2033402B02D99FED99
:103108002D0A7047B4EEC70AF1EE10FA0FDDB0EEE3
:10311800677A9FED296ADFED296A01E0B0EE677AE8
:10312800B4EEE67AF1EE10FA77EEC67AF6DC9FEDA9
:10313800247AF4EEC77AF1EE10FA0FD5B0EE677A7A
:103148009FED1D6ADFED1F6A01E0B0EE677AB4EE0D
:10315800E67AF1EE10FA77EE867AF6D49FED147AD5
:10316800F4EEC77AF1EE10FA1DDC9FED177AF4EE53
:10317800C77AF1EE10FA44BF9FED117A77EE677ABD
:1031880027EEA76ADFED115ADFED116A9FED117A7C
:10319800E6EE256A67EE865AA6EE267AE5EE877A87
:1031A800B0EE670A70479FED0C7A77EE677AE7E72B
:1031B800DB0FC93F00000000DB0FC940E4CB16411C
:1031C800DB0F49C0E4CB16C1DB0FC9BF92E741B999
:1031D8009730083C15A82ABEDB0F494010B507EE0A
:1031E800901A2DED028BB8EE678ADFED217A28EE72
:1031F800008A044628EE278AB0EE480A2DF0FCFC27
:10320800F0EE408AB0EE480A2DF058FCF7EE007A4E
:103218009FED187AF0EE675AE8EE875A0023A3610B
:10322800B0EE676AC7EEA56A63612362E361A8EE40
:10323800C76ABDEC028B77EEC07AB6EE007AF8EE7C
:10324800005A27EE877A20EE250A27EE267A26EE00
:10325800266A67EEA67A20EE260A84ED046AC4ED93
:10326800017A84ED007A84ED027A84ED030A10BDB8
:1032780027D4D236F304353F10B44C09012250F854
:10328800243001F01F0102FA01F10B4340F8243009
:103298005DF8044B704700BF4B0901F01F0150F85F
:1032A8002320012303FA01F1114214BF184600201C
:1032B800704700BF074A084B10781B78074A8342BB
:1032C80096BFC31AC3F18003002012681844104443
:1032D800704700BF48410020C540002068750020A5
:1032E800064A074B10781B7883428ABFC3F18003D4
:1032F800C01AC018C0F17F00704700BF48410020C5
:10330800C540002030B5144C237883B01BB9012088
:10331800237003B030BD052200238DF800208DF8FE
:10332800013000BF0D4D2B689868FEF7EDFF2B6844
:1033380001AA6946586826F0EDF82B689868FEF7E8
:10334800E9FF00BF9DF8053003F0010383F0010099
:10335800237003B030BD00BF6267002050670020B3
:1033680070B5064C0646256803E023685B1BB3422C
:1033780003D8FFF7C7FF0028F7D070BDF86000201A
:103388002DE9F04F89B0B2F1000A0290049103933D
:1033980040F3B0800B46002201EB8A0153F8040B7E
:1033A8008B420244FAD1039B0592002B00F09A80CD
:1033B800059B002B6AD0544B059A1B68DFF85C917B
:1033C80000920099DAB25118B1F5807F8CBFC2F52E
:1033D8008072009A01924D4A92689A426DD9190CEE
:1033E8001A0A4FF0020406208DF81F308DF81E20AF
:1033F8008DF81D108DF81C40FFF7B2FF0620FEF770
:103408008FFF434A0123137000BFD9F80030986832
:10341800FEF77AFFD9F8003007A95868002226F08D
:103428003BF80024049D029E019FA34629684FEAA9
:10343800840800220B46013471B1B9422AD2D9F866
:10344800000031684068FCF7B1FF2A68336813440C
:103458003360BF1AC5F800B0A24505F1040506F1AE
:103468000406E3D1D9F800309868FEF753FF00BF8F
:10347800254B019900981B68421A0092224A0B4476
:103488001360039A32B3009A002A9AD1059809B0BA
:10349800BDE8F08F029CD9F8003054F8081058683D
:1034A80000223B46FCF782FF54F808202B683A4478
:1034B800DF1B44F808202F60D4E70598009C1549C5
:1034C800154A001B0590059800230B70137009B06E
:1034D800BDE8F08F059B009A9B1A0593059809B0E3
:1034E800BDE8F08FFFF70EFF00287FF461AF039B64
:1034F8000593CBE7039C1CB9FFF704FF0594C5E7C8
:1035080000230593C2E700BF6875002088210020CA
:103518006267002048410020C54000205067002015
:1035280070B5104D104E2B7831788B4284B016D080
:103538000E4A03921A4402928CBF0C46CA1A04A976
:103548008CBFC3F180020024012341F8102D02A88A
:1035580002220194FFF714FF002333702B7004B08C
:1035680070BD00BFC540002048410020C840002071
:1035780070B5194C194D23782978994284B027D011
:10358800174A03921A44029234BF0E46CA1A04A973
:1035980034BFC3F180020026002341F8102D02A891
:1035A80002220196FFF7ECFE23781844C0B2030606
:1035B8002B7848BF80F080008342207002D0002022
:1035C80004B070BD002301202B70237004B070BDBF
:1035D800012004B070BD00BFC54000204841002054
:1035E800C840002008B545F20820FFF7B9FE0620BC
:1035F800FEF796FE064B0122C7201A70FEF790FED2
:1036080004480549054A002303700B70136008BD80
:103618006267002048410020C540002068750020EE
:103628002DE9F04182B00346060C050A0324062062
:103638008DF80730884617468DF805608DF80650D6
:103648008DF80440FFF78CFEC0B100BF0D4C236815
:103658009868FEF759FE236801A95868002225F0EA
:103668001BFF23684246002158683B46FCF79EFE34
:1036780023689868FEF74EFE00BF384602B0BDE8E2
:10368800F08100BF50670020F0B5124B9D6885B0EF
:103698000DB905B0F0BDED0A14D0002704AE7C19B1
:1036A8006410E00210226946FFF7BAFF0F2809DD0F
:1036B8006B4653F8042B01320AD1B342F9D125469F
:1036C800AF42ECDBFFF72CFF034BED021D60E0E798
:1036D800671CF5E78821002068750020B0F1FF3FDE
:1036E8000AD0022810B403DC5DF8044BFDF770BB68
:1036F80000205DF8044B70470020704710B4044662
:10370800134690F904000A4661795DF8044BE5E731
:103718000378012B00D070473122F421EEE700BF77
:10372800044B93F820209201343202F0FC02F42179
:10373800E4E700BF243E00202E22F421DEE700BF8C
:103748000278012A00D070474821D7E70278012A79
:1037580000D070475821D1E7F0B55B4B5B4A97B072
:103768001968914200AF00F0A3805949594A0023D3
:103778004FF47000C1F888003B607B60136843F425
:103788008033136003E03B68B3F5A04F09D013689A
:1037980003F400337B603B6801333B607B68002B9C
:1037A800F1D04C4B1B6813F4003318BF01237B6026
:1037B8007B68012B52D0464C464B474AE260474A49
:1037C800596A11605A6A42F080725A625A6942F420
:1037D800FC025A610025032207F10801012341F682
:1037E800FF764FF09040FD60BE603A73BB7321F0E6
:1037F800E3F94FF6FF7307F108013948BB6021F080
:10380800DBF907F108013748374E21F0D5F907F100
:103818000801364821F0D0F907F10801344821F0B1
:10382800CBF907F10801334821F0C6F907F1080080
:1038380020F078FFBB683049304AA1FB03133049B8
:103848009B0CF0204FF0070E5C370B60566084F835
:1038580023009560C2F800E0BD46F0BD294A1D4B23
:10386800122111605A685A605A685A605A6842F4BC
:1038780080625A605A6822F47C125A605A6842F48C
:10388800E8125A601A6842F080721A601A68920147
:10389800FCD559680F4A21F003015960596841F075
:1038A80002015960536803F00C03082BFAD182E730
:1038B80000221A6062B6144B1B6883F30888134B06
:1038C8001B689847FEE700BFFC9F0020EFBEADDEF7
:1038D80000ED00E0001002400005FA05884F0020C6
:1038E80000040048000800483F190100000C004887
:1038F800001000480014004883DE1B4310E000E07D
:10390800FC6000200020024000D8FF1F04D8FF1FE1
:1039180070B50F4C0F4DC0EBC00004EB8004686914
:1039280026693043686182B09209667BA1600025F0
:10393800012101A863618DF804608DF805208DF8D8
:1039480006508DF8071020F0E3FD02B070BD00BFEF
:103958000820002000100240074BC0EBC00030B424
:1039680003EB8000054C056963692B4363610176AD
:10397800427630BC704700BF08200020001002408B
:103988002DE9F04F5E4C54F8204083B0002C71D0E4
:10399800666D984691465B4B7268E264A16023604D
:1039A80004F15A014FF4807304F5AD726161A261AC
:1039B800E36023610746307E21F066F9F068A8B11C
:1039C800514B00215A68904203F11C0300F0928089
:1039D80001310C29F6D100207A1CD2B20C21FFF754
:1039E800BBFFE36CF26822632433A364B068D8B1E8
:1039F800454B00215A68904203F11C0378D00131ED
:103A08000C29F7D100257A1CD2B20B212846FFF7E2
:103A1800A3FF2346F27E3D492846FFF779FFE36C72
:103A2800B26862632833636494F85900FEF71AF8A1
:103A3800054694F85800FEF715F818F0080F824666
:103A480096F819B01AD0CDB118F0110F4FF00B033A
:103A580007F1010714BF4E213E21EF715A46AB71A1
:103A68002846FEF7C3F818F0010F45D0236B5BB367
:103A7800636B4BB3204603B0BDE8F08F18F0010F1D
:103A88000CBF4FF02E084FF04E0819F0020F09D066
:103A980045B10B227B1CAA71EB7128465A46414658
:103AA800FEF7A4F819F0010FE0D0BAF1000FDDD04D
:103AB80001370C238AF807705A4641468AF80630BF
:103AC8005046FEF793F8D1E7337FB27E8DF8042095
:103AD8009B090021012201A88DF805308DF80610F8
:103AE8008DF8072020F014FD204603B0BDE8F08FC4
:103AF800CDB288E7C8B26FE72846FEF705FCB5E700
:103B0800CC310020682F030808200020110D000880
:103B18000348D0F83C3113B100F59A701847704744
:103B2800082000200348D0F8203113B100F58C702C
:103B380018477047082000200348D0F804310BB11B
:103B4800FC301847704700BF082000200348D0F811
:103B5800E8300BB1E0301847704700BF082000205C
:103B68000348D0F8CC300BB1C4301847704700BFB9
:103B7800082000200348D0F8B0300BB1A83018470F
:103B8800704700BF082000200348D0F894300BB1DC
:103B98008C301847704700BF082000200248836F08
:103BA8000BB1703018477047082000200248C36DD9
:103BB8000BB1543018477047082000200248036CA6
:103BC8000BB1383018477047082000200248436A74
:103BD8000BB11C3018477047082000200248836842
:103BE80003B11847704700BF08200020F0B53E4CCD
:103BF800059D00EB800004EB80046468002C71D004
:103C08003A4E49004FF42040CFB2B061A16909048F
:103C180054D46068DFF8E0E047F4903100EA0E0021
:103C280001434FF420406160B06103E0411E002869
:103C380048D00846A1698907F8D54FF42040A26208
:103C4800B06103E0421E00283CD01046A26952062B
:103C5800F8D5274A6168DFF8A0E0B06142EA03427C
:103C6800174301EA0E0217436760C3B1013BDBB299
:103C780001332B44A0694FF4204210F0040002F1F4
:103C8800FF3207D1511C26D0A06910F0040002F1C0
:103C9800FF32F7D0626A05F8012B9D42EAD14FF452
:103CA8002040B06102E0431E60B11846A3699B063C
:103CB800F9D52023B061E3610120F0BD411E08B1B0
:103CC8000846A3E70B4A138801339BB24FF0FF3134
:103CD8001380B161F0BD0749B2610B8801339BB213
:103CE8000B80F0BD2046F0BD9860002074230020B2
:103CF80000240002104A0020009800FC70B590F9DA
:103D080004506C1C82B00AD0022D08DC16460A4604
:103D1800417900962846FFF769FF02B070BD002080
:103D280002B070BD70B50378012B82B004D10623B0
:103D38006A46F721FFF7E2FF9DF801209DF804305D
:103D48009DF800609DF803509DF802409DF805001D
:103D5800074912011B0142EA063243EA053342EAE7
:103D6800141243EA10134A600B6002B070BD00BF22
:103D78007423002010B582B001AA0323F621FFF7AF
:103D8800BDFF9DF80530094A9DF804409DF80600DE
:103D9800B2F9202006491B0243EA04430343C2F157
:103DA8000802D340CB6002B010BD00BF243E002003
:103DB8007423002000B583B001AA0223F621FFF77F
:103DC8009DFF9DF804109DF80530034A43EA01233E
:103DD800138103B05DF804FB7423002000B5037859
:103DE800012B83B004D1032301AA0021FFF786FF2A
:103DF8009DF805309DF804209DF806001B0243EA53
:103E08000243184303B05DF804FB00BF08B5FFF791
:103E1800E5FF014B586108BD7423002008B5FFF782
:103E2800DDFF014B186108BD74230020F0B585B093
:103E380002AB04460093032206231E210020FFF74D
:103E4800D5FE00283CD09DF808509DF809109DF833
:103E58000A709DF80B209DF80C609DF80D3041EA22
:103E6800052142EA072243EA062309B212B21BB22D
:103E7800144D06EE901A07EE102A07EE903AF8EE67
:103E8800E66A95ED005AD5ED025A95ED016AB8EE4D
:103E9800C77AF8EEE77A66EE856A27EE257A67EE46
:103EA800867AFDEEE66ABDEEC77AFDEEE77A16EE93
:103EB800901A17EE102A17EE903A2180A28063809C
:103EC80005B0F0BD000000202DE9F043322083B09A
:103ED80002F014FC0022104611231E21FFF7FEFBFE
:103EE800602301221E210020FFF7F8FB642002F066
:103EF80005FC6846FFF79AFF0024DFF89081254605
:103F080026460A27012302221E210020FFF7E6FB8E
:103F1800322002F0F3FB6846FFF788FFBDF902E0A4
:103F2800BDF90410BDF900208E457346A8BF0B46A5
:103F38009342A8BF134643454FF0010075440C4413
:103F48001644C0F29380FDF7F9F9013FDAD14FF03A
:103F580001090022104612231E21FFF7BFFBDFF8DC
:103F68002C810A27012302221E210020FFF7B6FB1D
:103F7800322002F0C3FB6846FFF758FFBDF902E0A4
:103F8800BDF90410BDF900208E457346A8BF0B4645
:103F98009342A8BF134643454FF00100A5EB0E0519
:103FA800A4EB0104A6EB02065DDBFDF7C7F9013FB0
:103FB800D8D107EE906AF8EEE76A07EE905AB8EEA5
:103FC800E77A07EE904ADFED2B5A9FED2B5A2B4EDE
:103FD800F8EEE77A85EEA66A0022104670231E21C5
:103FE800C5EE876A85EE277AB0EEC66AF0EEE66A15
:103FF800F0EEC77A86ED006AC6ED016AC6ED027A70
:10400800FFF76CFB202301221E210020FFF766FB2F
:104018000023184602221E21FFF760FB642002F0ED
:104028006DFBB9F1000F04D14FF07E53336073601C
:10403800B360134C206810B1FEF7AAF918B9012033
:1040480003B0BDE8F0830F490F4B41F8643FF022FD
:1040580008232068FEF778FA206821F0B3FC0120D5
:1040680003B0BDE8F0834FF00009A2E74FF0000964
:104078006FE700BF00406F4601C05E4600000020A9
:104088001C3E0020742300205D07000801F0FFFF9C
:10409800F0B587B00DF10F03054600930222012306
:1040A8000C210020FFF7A2FD18B19DF80F30DB07A7
:1040B80003D40024204607B0F0BD04AB00930322CC
:1040C80006230C210020FFF791FD0DF10F0300934B
:1040D800092201230C210020FFF788FD044600284F
:1040E800E7D09DF80F0010F00C00E2D19DF811E028
:1040F8009DF810109DF813709DF812209DF815601A
:104108009DF8143041EA0E2142EA072243EA0623C9
:10411800C1EB8131C2EB8232C3EB83338900920059
:104128009B0029806A80AB800A2201230C21FFF7BB
:10413800D5FABFE710B5002384B018460A220C212F
:10414800FFF7CCFA142002F0D9FA0F230A220C2127
:104158000020FFF7C3FA0A2002F0D0FA03AB00935D
:10416800102203230C210020FFF740FD0A2002F053
:10417800C5FA002318460A220C21FFF7AFFA0DF101
:104188000B040A2002F0BAFA0094012302220C213F
:104198000020FFF72BFD0094012309220C210020A9
:1041A800FFF724FD01230A220C210020FFF796FACD
:1041B800012004B010BD00BF00B583B000200092FC
:1041C8000A466821FFF712FD03B05DF804FB00BF43
:1041D8001749184B184A194810B4D1F8884044F4C4
:1041E8007004C1F888401C6844F001041C605C68D5
:1041F80022405A601A6822F0847222F480321A60CF
:104208001A6822F480221A605A6822F4FE025A6060
:10421800DA6A22F00F02DA621A6B002410404FF0BB
:10422800006218639C608A605DF8044B704700BFA9
:1042380000ED00E0001002400CC07FF8CCFC00FF4D
:1042480038B50B4C23688BB15A68821A002A054688
:1042580004DA0CE05A68AA1A002A07DB9A68226076
:1042680018461A6890472368002BF3D138BD38BD2B
:10427800943700200B4B002210B4027203F5A0748F
:10428800032102E0072A09DC9979890702D51979FF
:10429800815401329C4203F11403F3D15DF8044BBD
:1042A800704700BF5859030810230370704700BFB8
:1042B800012310B415211424222244704171C270C4
:1042C8000370037183705DF8044B70472C2202233E
:1042D80002704370704700BF08B512F057FD024BDB
:1042E800024ADA60FEE700BF00ED00E00400FA05CC
:1042F800024A034B1278197819F0ECBFF423002016
:10430800F52300202DE9F0470569C3681D4028D032
:104318000F4606464FF000484FF00009B5FA85F3FE
:1043280028FA03F2D2431B3B32611540042B16D8FE
:10433800DFE803F03129211903007B6A002B32D012
:1043480003F1FF3A1FFA8AFAC7F824903C6A34B19D
:1043580023682046514698476468002CF8D1002D00
:10436800DCD1BDE8F0873868716B036889B298477B
:10437800002DD3D1F5E77868B16B036889B2984707
:10438800002DCBD1EDE7B868F16B036889B2984787
:10439800002DC3D1E5E7F868316C036889B2984706
:1043A800002DBBD1DDE7F36A1FFA83FACEE700BF21
:1043B8002DE9F04F2DED028BA0F10A0389B00C46D0
:1043C800E72B00F25886DFE813F01C015606560664
:1043D80056065606560656065606560656065606F5
:1043E80056065606560656065606560656065606E5
:1043F800560656065606560656062D015606560603
:1044080056066B055606560656064B0156065801C3
:1044180056065D0256062C02560624025606D3039B
:104428005606FC01560656065606F501EE015606D6
:10443800E70156065606E0015606B8015606560626
:1044480056069C015606560656065606E1055606B9
:10445800FC0056064D040106560656065606560634
:1044680056065606560629055606EC045606B8049E
:104478005606640456061002560656065606560692
:10448800B6057B05D9052506E800560656069A03A3
:104498001A035606E302C70256065606560656067D
:1044A800BC02560656069B025606560656068C024F
:1044B8007502860344035606560656063503560605
:1044C80026032D0456065606560656065606560662
:1044D80056065606560656065606560656065606F4
:1044E8005606B60556065606560656065606560685
:1044F80056065606560656065606560656065606D4
:1045080056065606560656065606560656065606C3
:1045180056065606560656065606560656065606B3
:1045280056065606560656065606560656065606A3
:104538005606560656065606560656065606560693
:104548005606560656065606560656065606560683
:104558005606560656065606560656065606560673
:104568005606560656065606560656065606560663
:104578005606560656065606560656065606560653
:104588005606560656065606560656065606560643
:104598005606560656062204F803A74E337853B13A
:1045A800A64F002537F8021F2046FEF705FC337892
:1045B8000135AB42F6DC012009B0BDEC028BBDE849
:1045C800F08F9D4E3378002BF5D09D4F0025B846CF
:1045D800236817F81520591C21601A7098F80110E3
:1045E80001EB810101EB810101F2EE2189B2204644
:1045F800FEF7E2FB33780135AB4208F10208E7DC4D
:10460800D9E7904D28462BF07BF90028D3DD2B46BF
:104618000544226813F8011B501C9D42206011704C
:10462800F7D1C8E7884D05F15006287827F09EFA9B
:104638002368027A591C21601A7023686A78591C09
:1046480021601A702368AA78591C21601A7023689F
:10465800EA780435591CAE4221601A70E5D1AAE700
:104668000B687A4A581C11782060197023685278B0
:10467800591C216001201A709EE7754D0B682A7A33
:10468800591C21601A70A98B2046FEF795FB298BCF
:104698002046FEF791FB698B2046FEF78DFB2368C9
:1046A800EA7C591C21601A70A98C2046FEF784FB0D
:1046B800E98C2046FEF780FB2368AA7F591C2160FD
:1046C8001A70236895F82020591C21601A70698C8B
:1046D8002046FEF771FB2368EA7A591C21601A709C
:1046E800E9682046FEF750FB23682A7C591C2160A4
:1046F8001A70236895F82120591C216001201A702E
:104708005AE7FEF7FFFD2368524D002803F1010127
:104718000CBF0222032221601A7029882046FEF766
:1047280033FBA9682046FEF72FFBFEF7C3FD0146C1
:104738002046FEF729FB01203EE70B68434A464D19
:104748001178464A581C2060197011682046FEF7F7
:104758001BFB23683E4A591C127A21601A7029886B
:104768002046FEF729FBA9882046FEF725FB298964
:104778002046FEF721FB00212046FEF71DFB2046C0
:104788000021FEF719FB012016E7084608223049E8
:10479800FEF7E2FA01200FE70B68314A581C9178BE
:1047A8002060197062E70B68012299182160104691
:1047B8001A7001E72B4B08461968FEF7E5FA012045
:1047C800FAE6294D294E05F1280795F90210284BDC
:1047D80093F906208A4203F1080300F04F849E42B1
:1047E800F6D10835BD42F0D1E5E60B68214A2249E9
:1047F800D078224A5D1C2560187023684979581CB6
:10480800206019702368D278591C216001201A7021
:10481800D2E60B680E4A591C527D216001201A709D
:10482800CAE6174D05F1800655F8041F2046FEF725
:10483800ABFAAE42F8D1BEE668490020C65F002058
:104848003C390020C4590020847500208075002060
:104858005C4F002088210020F831002018400020FB
:10486800DC780020883E002068670020FC4D00208E
:10487800D44D0020403A0020245E0020103E002045
:104888008C580020A94D05F14006B5F88010204647
:10489800FEF792FA236895F88220591C21601A7055
:1048A800236895F883200435591CAE4221601A709C
:1048B800EBD180E60A689E4B9E491878551C256006
:1048C800107022685878551C2560107022689B78F3
:1048D800501C206013702046C988FEF76DFA01202D
:1048E8006AE6944D08462988FEF766FA69882046E4
:1048F800FEF762FA2046A988FEF75EFA01205BE619
:104908008D4D05F16006A9882046FEF755FAE9881D
:104918002046FEF751FA29892046FEF74DFA23680A
:10492800AA7A591C21601A702368EA7A591C2160F6
:104938001A7055F80C1B2046FEF726FAB542E2D14C
:1049480039E67E4952232268501C2060137011F802
:10495800013F002BF7D12EE679480023226805682D
:1049680003EB4301561C6D5C2660157002682568D0
:104978000A446E1C527826602A70026825680A4428
:1049880001339278691C0A2B21602A70E6D112E65D
:104998006C4D0B682A68591C127821601A702B68B4
:1049A80022689978531C2360002311702A682168B3
:1049B8001A4401335279481C032B20600A70F5D140
:1049C80023682A68591C127A21601A7023682A6899
:1049D800591CD27821601A7023682A68591C1279E8
:1049E80021601A702B6820465989FEF7E5F92A6874
:1049F8002368527A591C21601A702A6836E6524B8D
:104A080008461968FEF7C0F9504B20461988FEF78A
:104A1800D3F90120D0E54E4B4E49B3F9003081FB64
:104A28000321DB17C3EBA101204689B2FEF7C4F9C5
:104A38000120C1E5484D0846298AFEF7BDF9698A73
:104A48002046FEF7B9F92046A98AFEF7B5F90120F4
:104A5800B2E5DFF818E10027FEB2714600232268AC
:104A6800501C206016702268501C20601370226849
:104A780011F8010F0133551C062B25601070EED17B
:104A88000137062F0EF1060EE6D1344900232268BD
:104A9800501C206017702268501C20601370226818
:104AA80011F8010F0133551C0B2B25601070EED146
:104AB80023681E4A581C07212060197023680021AA
:104AC800581C20601970236892F8F020591C216046
:104AD80001201A7070E50B68214A224910781C4A97
:104AE8005D1C2560187023688978581C206019702F
:104AF80023689278591C216001201A705CE51A4DD0
:104B080008462988FEF758F969882046FEF754F9BF
:104B1800B5F904300F4AD91782FB0323C1EBA3016F
:104B2800204689B2FEF748F9012045E59058002053
:104B3800583200206835002050660020902F030866
:104B4800DC590020B87800201C780020EC5900209F
:104B5800103E0020676666665C6A00207359002074
:104B6800244B0020403A0020BC5900204F59002017
:104B7800A34B03F15A0522685979501C2060117023
:104B880022681978501C2060117022685978501CCE
:104B98002060117022689978501C2060117022687A
:104BA800D978501C20601170226819790633501C7E
:104BB8009D4220601170DED1FDE4924B03F1700537
:104BC80022681978501C2060117022685978501C8E
:104BD8002060117022689978501C2060117022683A
:104BE800D978501C2060117022681979501C2060F7
:104BF800117022685979501C2060117022689979C7
:104C08000733501C9D4220601170D9D1D3E47E4DEA
:104C18000846E989FEF7D0F82046A989FEF7CCF8BE
:104C28000120C9E40B68794F591C3A7821601A7041
:104C38003B78002B3FF4BFAC0025EEB2304622F0A3
:104C480053FE23684278591C216030461A7022F0BE
:104C58004BFE01892046FEF7AFF83B780135AB42A1
:104C6800EBDCA8E40B6800255A1C0A601D700B6871
:104C78005A1C0A601D700B685A1C0A602046294697
:104C88001D70FEF781F820462946FEF77DF80120C1
:104C980092E400212046FEF78FF800212046FEF717
:104CA8008BF800212046FEF787F82368584D002628
:104CB8005A1C22601E7023682A68591C92F82C20FE
:104CC80021601A7023682A68591C92F836202160DE
:104CD8001A7023682A68591C92F8372021601A70C4
:104CE80023685A1C22601E7023685A1C22601E709A
:104CF80023685A1C22601E702B682046598FFEF7C5
:104D08005BF82B682046198FFEF756F823682A6847
:104D1800591C92F82E2021601A7023685A1C2260B0
:104D28001E702B682046598EFEF746F82B682046E1
:104D3800998EFEF741F801203EE4364E0B687279F1
:104D4800334D591C21601A702B682046198CFEF7C8
:104D580033F82B682046D98BFEF72EF87189204648
:104D6800FEF72AF8B1892046FEF726F82B68204678
:104D7800598CFEF721F82B682046998CFEF71CF811
:104D8800F1892046FEF718F8318A2046FEF714F814
:104D98002A68236892F82620591C216001201A707D
:104DA8000AE41C4EF378002B00F060820B6808229E
:104DB800591C21601A7023680122991821601A7001
:104DC8002368154D591C2A7921601A702368AA781E
:104DD800591C21601A7029882046FDF7EDFFE989E2
:104DE8002046FDF7E9FF2368F279591C21601A7003
:104DF8002368EA78591C216001201A70FFF7DCBB90
:104E08009C330020B8630020403A00203561002020
:104E1800DC590020244B00205C6A002019F03EFA7F
:104E2800FF28064600F02E8208A9002501F8125D29
:104E38000DF10D008DF80D5019F030F908A800F8A3
:104E4800115D19F01FF908A800F8105D19F00EF9A6
:104E580008A820F8085D19F0FDF823685A1C22609C
:104E68001E7023689DF80D20591C21601A70236854
:104E78009DF80E20591C21601A7023689DF80F2098
:104E8800591C21601A7023689DF81020591C216054
:104E98001A702046BDF81810FDF78EFFFFF78BBB80
:104EA800A54D08462988FDF787FFA9882046FDF704
:104EB80083FF20462989FDF77FFF0120FFF77CBB90
:104EC8009E4B9B8AB3F5006F00F2CE81B3F5806FDD
:104ED80000F2EF81B3F5007F34BF01270227984D18
:104EE80005F10C0655F8041B91FBF7F1204689B231
:104EF800FDF762FFAE42F5D1924D934F05F10C06D6
:104F0800B5EC010AD7ED087A80EE270A2BF028FEC7
:104F180081B22046FDF750FFAE42F1D18B4D05F12D
:104F28000C0655F8041B204689B2FDF745FFB5422B
:104F3800F7D1FFF740BB00258146DFF84882DFF84C
:104F480048B2059504950695079501214FF6FF7A15
:104F580005E001350B2D00F0AF8018F9011F4F1C3B
:104F68004AFA05F3F5D0DE07F3D5BBF800302B413C
:104F7800D807EED506A8FEF77FF9EAE7084610221B
:104F88007349FDF7E9FE0120FFF716BB0B68714D69
:104F9800591C2A7921601A7023686A79591C216082
:104FA8001A7029882046FDF707FF2368AA79591C3B
:104FB80021601A7069882046FDF7FEFE2368EA79A9
:104FC800591C216001201A70FFF7F6BA0B68624E6F
:104FD80001255A1C0A601D700B68B27859192160A6
:104FE8001A7026F0C9FF23685C4A5D495F1927607B
:104FF8001870B1F90010B2F90000FEF767F82368DD
:105008005A192260187031882046FDF7D5FE2846C7
:10501800FFF7D2BA534D544E9FED548ADFF86C8196
:10502800DFED538A05F120070EE0FCEEE77ACDEDBF
:10503800017ABDF8041020460435FDF7BDFEAF42E5
:1050480006F118063FF4B7AA717C0029F3D0494B42
:10505800D5ED007A1B78012BE7D1474B1B68DB04A1
:1050680040F1FA80F5EE407AF1EE10FA40F0238133
:1050780040F2DC51DFE70020FFF79EBA23685A1C94
:105088002260197029882046FDF796FE2368EA7881
:10509800591C21601A7023682A79591C21601A70DA
:1050A8002368AA79591C21601A7023686A79591CE7
:1050B80021601A70FFF795BBDFF8D4A000254FF0E8
:1050C80008080135C5F1200208FA02F2A5F120030B
:1050D8002AFA05F6164328FA03F31E43252D06F08F
:1050E80001024FF000030BD01343EAD0E8B229F0D5
:1050F80019FC0028E5D0294606A8FEF7BDF8E0E728
:105108001E4B1B78DA0700F1C48000251C4E2F4681
:1051180002E00135252D3DD029463046FEF7BCF882
:105128000028F6D0294606A8FEF7B6F8002840F071
:105138008E800137EDE700BFF8310020B448002029
:10514800EC480020C04D0020384B0020FC480020CF
:10515800807300208435002010780020C073002060
:10516800C2730020907300209C6900200000404218
:1051780000E08244806A0020CC4D0020EC5F0020D3
:105188001C730020C02F0308B8590020DB9B9141F5
:1051980090E33FF4664B674DB3F850102046FDF797
:1051A8000BFE654B1988204689B2FDF705FE634B57
:1051B80019684B0103F02002C1F340031343C1F304
:1051C800800243EA4203C1F3C00243EA8203C1F307
:1051D800401243EAC20301F0100119432046FDF7CB
:1051E800EBFD04A904222046FDF7B6FD23682978C3
:1051F800534A581C2060197011886429A8BF64217B
:105208002046FDF7D9FDB9F1960F47D00021204679
:10521800FDF7D2FD2168B7F1190348BFA7F11203C2
:10522800A3F3C4034A1C226020461A460B7005A942
:10523800FDF792FD2368434A581C1021206019701D
:1052480020461188FDF7A0FD0120FFF7B5B93946C2
:1052580004A8FEF711F86CE7F4EEC87AF1EE10FA3C
:1052680045DA4FF47A71E6E6082738E60B68B17834
:10527800354A581C2060197023681278591C21601F
:105288001A709DE523685A1C226001201E70FFF7E2
:1052980093B9069B43F00103069336E7236803227C
:1052A800591C21601A7023686A78591C21601A7089
:1052B800B0E7042713E6F4EEC87AF1EE10FA3FF5EA
:1052C800D7AEF4EEE87AFDEEE77AF1EE10FA17EED3
:1052D800901A1ED86FF4F973303903FB01F140F2CC
:1052E800E73391FBF3F101F2DB5189B2A3E6FDEE5E
:1052F800E77A40F2E73217EE903A303B02FB03F3CD
:1053080088FB0312D917C1EB622101F2E93189B296
:1053180091E640F2F313A1F5836103FB01F140F23A
:10532800E73391FBF3F101F2DD5189B283E600BF67
:10533800F41A0020E0590020104A00203478002098
:10534800144A0020387800206865002008B501213B
:105358000220FDF703F8094B1B7803F00503052B22
:1053680008D000210120FCF7F9FF00210846FCF7CE
:10537800F5FFFEE711F09CFDF3E700BFC831002000
:10538800022828BF022010B4084C094B207000EBFB
:105398008002C0EBC20207495DF8044B013003EB01
:1053A8004203C0B20B6025F0E7BC00BFE059002003
:1053B800EC3E0020DC59002008B513F08DFAFDF70B
:1053C800B1FABDE8084013F06FBA00BF38B5434BD7
:1053D8005A899989914224BF00225A81198ADA8907
:1053E800914224BF0022DA81DA788AB3072A2FD0C3
:1053F8003B493C4D91F85700012400210A282C70A4
:105408009C70D9713DD00C2865D0DFED377A8ABB06
:10541800364C9FED370AA278002918BFF0EE407A83
:10542800062A04D8334901EB820191ED0F0A21794C
:1054380059B3013A032A4DD8F7EE007A87EE800A6D
:105448002BF08EFB2388984228BF1846208038BD51
:10545800D97921B198780428B8BF042098702048D9
:1054680090F857000A280CD00C28CED1DFED227A0C
:10547800002ACDD0072ACBD00A282CD1DFED1F7AFD
:10548800C6E70A20DFED1E7AC1E79B78154A07EECA
:10549800103A1178B8EEC77A27EE277A07EE901AF5
:1054A800F8EEE77A67EE877AB4EEE70AF1EE10FADB
:1054B80010DDC0EE077AFDEEE77A17EE903A102B72
:1054C800A8BF1023012BB8BF0123DBB28B4238BF22
:1054D8000B46137038BDDFED0B7A99E7244B00209B
:1054E800384B0020686500206F1203395C6A002081
:1054F8006F120338902F03080AD7A3390F506E3A5A
:105508005304E9386F12833A38B50C4C0C4DAC4251
:1055180006D2616820461434FDF790F9AC42F8D3FE
:10552800084A094B094C1460002209491A705A703C
:1055380008480860BDE8384018F022BBB09B030853
:1055480038A00308DC590020E0590020EC3E002078
:10555800B87800209048002008B5FFF7D5FF13F071
:10556800BBF9FDF7DFF9BDE8084013F09DB900BFAE
:10557800F0B50C292BD8DFE801F06F2A2A2A4C2A2B
:105588002A2A2B2A2A2A0700046AB2F80CE09788EC
:105598001668674D24F480540462036A4468C1693C
:1055A80023F4005343EA0E3321F4E641A84243EAC8
:1055B800073341EA062100F0B58005F50065A842E9
:1055C80000F0B08092684460C16102640362F0BD7B
:1055D800046A96899588D2F800E0554F24F48074BF
:1055E8000462036A4468C16923F4007343EA06232A
:1055F80021F07301B84243EA052341EA0E017ED047
:105608004C4DA8427BD092684460C161C26303627A
:10561800F0BD046A96899588D2F800E0444F24F0DA
:1056280010040462036A4468816923F0200321F0AE
:10563800807143EA061321F4E641B84243EA0513B0
:1056480041EA0E2148D03B4DA84245D092684460BB
:10565800816182630362F0BD046A9389B2F804E051
:105668001768334E24F001040462056A44688169AE
:1056780043EA0E0321F4803125F002059BB221F0A4
:105688007301B04243EA050341EA070114D0294DEA
:10569800A84211D005F54065A8420DD005F58065F2
:1056A800A84209D005F58065A84205D092684460F3
:1056B800816142630362F0BDD689158A578A23F057
:1056C800080333433D43D68824F4407423F004038D
:1056D800ADB233432C43E9E7D589178AD68823F03E
:1056E800800343EA051324F44064558A23F04003F9
:1056F80044EA870443EA061344EA8504A6E7D58901
:10570800178AD68823F4006343EA052324F4405417
:10571800558A23F4806344EA071443EA062344EADB
:10572800051470E7158A24F4804444EA851449E78F
:10573800002C0140003401402DE9F84F4FF48C72E1
:1057480000218248824C834D834E844FDFF82882A3
:10575800DFF828922DF011FB81488249DFF820E21A
:10576800DFF820C200221359834200F0C380B3F14E
:10577800804F00F0D580AB4200F0D980B34200F0F2
:10578800D880BB4200F0D780734500F0D6806345CF
:1057980000F0A680434500F0D2804B4500F0D2804F
:1057A800DFF8E4A1534508BF4FF4802300F09A8046
:1057B8001432B2F5AA7FD6D1654D6B4F6B4E05F505
:1057C800AA784FF0030A4FF0020903E01435454563
:1057D80000F08E80AB79002BF8D02B791C09013CA6
:1057E800052C03F00F03F1D837F8140040FA03F240
:1057F800D207EBD54FF0010B0BFA03F3013B18402E
:105808002AF098FD5A4B1B5D184416EBC004DDD0F6
:1058180056F830305748297A03F13842920A825CA8
:1058280002F01F005209022A0BFA00FB71D0032A6A
:1058380068D0012A05D14B4A4A4852694BEA02020C
:105848004261B4F804E0BEFA8EF2C2F11F0292B2CD
:10585800D00803EB800002F00702046A92004FF0C0
:105868000F0C0CFA02FC24EA0C040462046A01FA24
:1058780002F22243002402624FF0010C224603E0A8
:10588800102A04F10204A1D00CFA02F030EA0E0149
:1058980002F10102F4D1D3F808B00AFA04F1C943BD
:1058A8000BEA010BC3F808B0D3F808B0C3F808B086
:1058B800B3F804B01FFA8BFB2BEA00009880988895
:1058C80080B29880186808401860D3F800B009FAC8
:1058D80004F040EA0B001860D8680140D960CFE7AF
:1058E8004FF40053D1F818A043EA0A038B615FE72D
:1058F800BDE8F88FD1F818A04FF4006343EA0A0313
:105908008B6155E7174A1748D2694BEA0202C26110
:1059180097E7144A134892694BEA0202826190E7BA
:105928000123D1F81CA043EA0A03CB6140E7022314
:10593800F7E70423F5E71023F3E72023F1E74FF413
:105948008033CFE74FF40033CCE700BF3076002038
:1059580058590308000400400008004000100040A7
:10596800002C014000100240B85C03086468002065
:10597800C45C03085059030800400140004401403A
:105988000014004000340140004801400149024829
:10599800FEF7B8BC207700200048014001490248C2
:1059A800FEF7B0BCD0760020004001400149024813
:1059B800FEF7A8BCA876002000080040014902486C
:1059C800FEF7A0BC807600200004004002494FF09A
:1059D8008040FEF797BC00BF5876002010B5064CF3
:1059E80006482146FEF78EFC04F1C8010448BDE8CC
:1059F8001040FEF787BC00BF30760020002C014025
:105A08000044014001490248FEF77CBC3076002082
:105A1800002C01402DE9F0410468514DA30AAB4226
:105A280000F084800AD94F4DAB4277D00135AB42A4
:105A38005FD0023DAB426DD0BDE8F0814A3DAB423C
:105A480070D00135AB4258D0B3F5801FF4D14FF078
:105A5800480E012647794FEA970C00296AD0B00012
:105A6800634685190227D4F80C809F400CEB450348
:105A7800BFB23D4D03F1040C47EA080745F823106F
:105A880045F82C20E760EFF31181502282F3128849
:105A9800821905EBC2021369002B32D0136204335A
:105AA800821905EBC202576917B11F6053690433A5
:105AB800821905EBC202976917B11F609369043315
:105AC800821905EBC202D76917B11F60D369043385
:105AD8000027CAB21F6082F31188304405EBC0006A
:105AE800036A8BB9E3684FF6FE721340E360BDE8C2
:105AF800F0814FF4887E0626ACE74FF0980E032617
:105B0800A8E705EB0E03CBE7E36843F00103E36086
:105B1800BDE8F0814FF0C00E04269BE74FF0E80E79
:105B2800052697E74FF0700E022693E74FF0200EF8
:105B380000268FE7BF08022306FA03F0BB40DB43C9
:105B4800E768094D9BB23B4087190CEB470CE360B3
:105B58000CF1040345F82C1045F8232093E700BF07
:105B68004B001000510010003076002030B503685B
:105B78005C4D18885C4CB4FBF2F20139013AAB4237
:105B880094B283B089B282B266D05848834263D057
:105B9800B3F1804F60D0A0F5983083425CD000F517
:105BA8008060834258D0524883425BD000F58060C1
:105BB80083427DD022F4407200F58C3092B2834249
:105BC8001A80D9621C850ED0484A93420BD002F540
:105BD8004062934207D002F58062934203D002F5F7
:105BE8008062934201D100221A8601225A611A88E2
:105BF8003C4992B242F001028B421A8062D0B3F162
:105C0800804F61D03B4A934260D002F58062934254
:105C18005ED002F5006293425CD002F58062934246
:105C28005AD002F59032934258D002F5406293421E
:105C380056D002F5806293421ED002F580629342EC
:105C480008BF092219D002A84FF0012340F8043DEB
:105C58001EF05EFC03B030BD254822F0700283427E
:105C680092B2A3D101201A80D9621C8558611A8882
:105C780092B202431A80C5E708221F4B03EBC20306
:105C880001A893F85D408DF80440012300228DF8A7
:105C980005308DF807308DF806201EF039FC1B2CD6
:105CA800D8D1164B019301A81EF032FC03B030BDC9
:105CB80001201A80D9621C8558611A8892B2024361
:105CC8001A809CE70022D8E70122D6E70222D4E70F
:105CD8000322D2E70422D0E70522CEE70622CCE74A
:105CE8000722CAE7002C014000A24A040034014000
:105CF8000010004000040040902F03081901000123
:105D0800204B98422DD0B0F1804F2CD0A3F594337E
:105D180098422AD003F58063984228D003F500639F
:105D2800984226D003F58063984224D003F5903337
:105D3800984222D003F54063984220D003F580634F
:105D4800984207D003F58063984208BF092202D021
:105D58000020704708220C4B03EBC20393F85C0049
:105D680070470022F7E70122F5E70222F3E7032252
:105D7800F1E70422EFE70522EDE70622EBE7072229
:105D8800E9E700BF002C0140902F03082DE9F04FF0
:105D9800013085B0C3B203938E4D8F4F8F4C904E18
:105DA8000A230293DFF840921FF082FC4FF4FA7A3C
:105DB8004FF0100C4FF47A70D9F80430C3F308038D
:105DC800002B40F0C880EFF31183002B40F0C38014
:105DD8002968A26800BF2B689942F9D1D7F800E07A
:105DE80000FB0EF39B1AB3FBFEF300FB01314FF0EF
:105DF800010E0191D9F80430C3F30803002B40F0D9
:105E08008E80EFF31183002B40F089802B68A16806
:105E180000BF2A689342F9D1D7F800B000FB0BF213
:105E2800521AB2FBFBF200FB0323019A9B1AB3F54B
:105E38007A7FDFD3BAF1010ABED1039B002B40F071
:105E4800C4804FF47A7ADFF8A09150464FF0100CD6
:105E5800D9F80430C3F30803002B40F09980EFF31E
:105E68001183002B40F094802968A26800BF2B683A
:105E78009942F9D1D7F800E000FB0EF39B1AB3FB67
:105E8800FEF300FB01314FF0010E0191D9F8043007
:105E9800C3F308033BBBEFF3118323BB2B68A16853
:105EA80000BF2A689342F9D1D7F800B000FB0BF283
:105EB800521AB2FBFBF200FB0323019A9B1AB3F5BB
:105EC8007A7FE3D3BAF1010AC2D1029B013B029364
:105ED8007FF468AF4349444B4448454A0860DA6058
:105EE80005B0BDE8F08FEFF311888CF31288A16834
:105EF8002368DB0344BFC6F800E0A1682B6832685A
:105F08005FFA88F888F31188D7F800801A4400FBF4
:105F180008F35B1AB3FBF8F300FB0233CDE7EFF3AA
:105F280011888CF31288A1682368DB0344BFC6F884
:105F380000E0A1682B6832685FFA88F888F3118856
:105F4800D7F800801A4400FB08F35B1AB3FBF8F398
:105F580000FB023369E7EFF311828CF31288D4F85F
:105F680008E02368D90303D501233360D4F808E097
:105F78002B683168D2B282F311883A68194400FB61
:105F880002F3A3EB0E03B3FBF2F300FB01312EE7A0
:105F9800EFF311828CF31288D4F808E02368D90350
:105FA80003D501233360D4F808E02B683168D2B2F6
:105FB80082F311883A68194400FB02F3A3EB0E033D
:105FC800B3FBF2F300FB01315DE718461FF0E0F97F
:105FD80037E700BFF8600020FC60002010E000E018
:105FE800F4600020FC9F002000ED00E0EFBEADDE75
:105FF8000400FA052DE9F047AB4FAC4E12F06CFCEB
:10600800BE421ED2DFF82C83DFF82C934446258845
:1060180062197DB14A450DD2052D0BD933886188A7
:10602800C3F30B03994200F0EE80144625886219E9
:10603800002DEFD1716830461436FCF7FFFBBE42E5
:10604800E4D39B4A1378A3F1170102290FD9994980
:1060580011F83300002840F0F880D800014449784E
:1060680029B1954911F83330002B00F01681934C73
:106078006378022B84BF002363702378022B84BFCC
:10608800002323708E4B9A78042A00F0FD8032B9E1
:106098001A88B2F5F07F84BF4FF4F0721A80894DE8
:1060A800894A2B681A40002A00F0FA80D80700F1C4
:1060B800E680590400F1DE801A0700F1D6809B04BF
:1060C80000F1CC80814D2B685A8C998C914224BF69
:1060D80000225A84FFF77AF91AF00CFA10B97C48B2
:1060E80024F014F98020FCF7DFFB4FF40010FCF7D4
:1060F800DBFB4FF00070FCF7D7FB4FF08060FCF73C
:10610800D3FB6378022B06D8724A734903EB430327
:1061180002EB83030B602378022B07D803EB830180
:106128006E4AC3EBC10302EB43032B6028F072FCF9
:10613800002130226A482CF020FE286822F030FC2A
:10614800684B2E6803F1500102E0043399427AD07B
:106158001A78002AF9D19C78D8788442F5D2624915
:10616800624B91F804E06248624D5C6B624B2860B8
:10617800C827642111FB0E71DFF8C0E159605F4F39
:1061880030F8061C5E4DAEF8001000219960D96009
:10619800196159619961D96183F8201083F8211038
:1061A8003A702E600CB114F0C9FC564B9FED565A4C
:1061B8001B88564A9FED566A5579564C564957489A
:1061C800086006EE903AF8EEE66A1388C5EE265A9D
:1061D80007EE103A53881279C4ED005A07EE903A48
:1061E800B8EEC77A4E4BF8EEE77A1D725A7227EE70
:1061F800067A67EE867ABDE8F04783ED017AC3ED4B
:10620800007A12F051BB63799B077FF40EAF716877
:1062180094F804A03046FCF711FB3388BAEB133F1F
:1062280004D01436BE42FFF4F1AE0AE773887068F2
:10623800AA1FC3F30B039A4204F10601A8BF1A462A
:106248002AF086FAEDE7012289E7D8000C1864687D
:10625800002C7FF403AF17241470FFE63148FCF7D5
:1062680023FB4020FCF720FB2CE72F48FCF71CFB06
:106278002B6824E72D48FCF717FB2B681CE72C48F4
:10628800FCF712FB2B6814E79A8AB2F57A7FBFF401
:1062980006AF4FF47A729A8201E718231370E6E684
:1062A80043F001032B6001E738A00308B09B030803
:1062B80080750020E4550308485B0308E059002076
:1062C8005C6A00201840002009600002DC590020A8
:1062D8006867002090480020B8780020EC3E002035
:1062E800742700208475002084350020B4480020DD
:1062F800463A0020F4720020184900209921002015
:10630800A82700208C320020C0C9FB48E4230020C5
:1063180017B7D13890320020683300203661023D2B
:1063280044330020094000020160000209200002F5
:106338000860000202F0030800000408503A002038
:1063480008B512F0C9FAFCF7EDFA12F0ADFAFFF74A
:1063580051FE0120BDE8084024F00EBD2DE9F04FA4
:10636800013085B0C3B203930B4602918B4C8C4E1F
:10637800002B00F099808B4D8B4FDFF830921FF087
:1063880097F94FF4FA7A4FF0100C4FF47A70D9F865
:106398000430C3F30803002B40F0DE80EFF31183D1
:1063A800002B40F0D9802968A26800BF2B68994269
:1063B800F9D1D7F800E000FB0EF39B1AB3FBFEF30C
:1063C80000FB01314FF0010E0191D9F80430C3F3FD
:1063D8000803002B40F08780EFF31183002B40F077
:1063E80082802B68A16800BF2A689342F9D1D7F848
:1063F80000B000FB0BF2521AB2FBFBF200FB0323C6
:10640800019A9B1AB3F57A7FDFD3BAF1010ABED19C
:10641800039B002B40F0BD804FF47A7ADFF88C9113
:1064280050464FF0100CD9F80430C3F30803002B82
:1064380075D1EFF31183002B71D12968A26800BFD1
:106448002B689942F9D1D7F800E000FB0EF39B1AAC
:10645800B3FBFEF300FB01314FF0010E0191D9F8B7
:106468000430C3F3080313BBEFF31183FBB92B68A4
:10647800A16800BF2A689342F9D1D7F800B000FBA1
:106488000BF2521AB2FBFBF200FB0323019A9B1A90
:10649800B3F57A7FE3D3BAF1010AC4D1029B013B79
:1064A8000293002B7FF467AF05B0BDE8F08FEFF3E0
:1064B80011888CF31288A1682368DB0344BFC6F8EF
:1064C80000E0A1682B6832685FFA88F888F31188C1
:1064D800D7F800801A4400FB08F35B1AB3FBF8F303
:1064E80000FB0233D2E7EFF311888CF31288A1681E
:1064F8002368DB0344BFC6F800E0A1682B68326854
:106508005FFA88F888F31188D7F800801A4400FBEE
:1065180008F35B1AB3FBF8F300FB023370E7EFF301
:1065280011828CF31288D4F808E02368D90303D5C4
:1065380001233360D4F808E02B683168D2B282F3C3
:1065480011883A68194400FB02F3A3EB0E03B3FB6E
:10655800F2F300FB01317FE7EFF311828CF312882D
:10656800D4F808E02368D90303D501233360D4F8AD
:1065780008E02B683168D2B282F311883A6819446E
:1065880000FB02F3A3EB0E03B3FBF2F300FB0131B4
:1065980018E718461EF0FCFE3EE700BF10E000E0DA
:1065A800F4600020F8600020FC60002000ED00E0AE
:1065B800204B5B68C3F3080330B4BBB9EFF3118316
:1065C800A3B91D4B1D4C1868A16800BF1A689042FA
:1065D800F9D11B4B1C684FF47A7202FB04F3591A69
:1065E800B1FBF4F130BC02FB00107047EFF31182ED
:1065F800102383F3128811498C680B6813F4803FC9
:10660800104B02D0012018608C680B49D2B20D687B
:10661800186882F311880A4B19684FF47A72284473
:1066280002FB01F31B1B30BCB3FBF1F302FB003090
:10663800704700BF00ED00E0F860002010E000E0C7
:10664800FC600020F46000202DE9F84F8046FFF739
:10665800AFFF254E2549DFF8A0E0254A254D8446A1
:1066680010274FF47A740120DEF80430C3F30803CE
:10667800D3B9EFF31183BBB90B68D2F808A000BFF8
:10668800D1F800904B45F7D1D6F800B004FB0BF9D0
:10669800A9EB0A09B9FBFBF904FB0393A3EB0C0371
:1066A8004345E1D3BDE8F88FEFF3118A87F31288E9
:1066B800D2F808B01368DB0344BF2860D2F808B0EA
:1066C8000B68D5F800905FFA8AFA8AF31188D6F831
:1066D80000A0994404FB0AF3A3EB0B03B3FBFAF302
:1066E80004FB0933DAE700BFFC600020F8600020F3
:1066F80010E000E0F460002000ED00E02DE9F04F2C
:10670800DFF830C1474A4849484E494D804610276E
:1067180018F1FF38C0F08480DCF80430C3F30803B4
:10672800002B5CD1EFF31183002B58D10B689468D0
:1067380000BF08688342F9D1D6F800904FF47A7008
:1067480000FB09FEAEEB040EBEFBF9FE00FB03EEF8
:10675800DCF80430C3F308034FF47A740120FBB962
:10676800EFF31183E3B90B68D2F808A000BFD1F8A2
:1067780000904B45F7D1D6F800B004FB0BF9A9EB14
:106788000A09B9FBFBF904FB0393A3EB0E03B3F56A
:106798007A7FBDD2DCF80430C3F30803002BDFD0C6
:1067A800EFF3118A87F31288D2F808B01368DB0375
:1067B80044BF2860D2F808B00B68D5F800905FFA9B
:1067C8008AFA8AF31188D6F800A0994404FB0AF3E0
:1067D800A3EB0B03B3FBFAF304FB0933D5E7EFF3A1
:1067E800118487F31288D2F808901368D80303D568
:1067F80001232B60D2F808900B682868E4B284F370
:106808001188D6F800A04FF47A7400EB030E04FB4D
:106818000AF3A3EB0903B3FBFAF304FB0E3E97E775
:10682800BDE8F08F10E000E0F8600020FC60002078
:10683800F460002000ED00E030B4EFF31183102283
:1068480082F312880649074C0A6807480132002576
:106858000A602560DBB2026883F3118830BC704798
:10686800F8600020F460002010E000E00F4B1B8867
:10687800014643B90E4B0F4A1B7810680BB981F0DB
:106888000101FBF761BD0C4B5A691AB118B91A68B6
:10689800106058747047094A18681188084A92FBB2
:1068A800F1F2012102605974704700BFD0600020E6
:1068B800D2600020D4600020D8600020F060002062
:1068C80020A107002DE9F04F95B0B0F908500D81CF
:1068D800EDB2442D00AF0C46904600F0C882064643
:1068E80043D9812D00F0FC8100F29980542D00F0ED
:1068F800CE8040F21E816E2D00F08782802D40F000
:106908001B81BF4B93F800A00AF1020A1AF0FF0A94
:1069180000F09980BB4BDFF82083BB4EDFF81CB337
:106928009A4403F101090A2516E0322D00F08A8302
:10693800A5F13C00C0B2132840F28A8300232268E4
:10694800511C216015702268CA4502F101012160BD
:10695800137078D019F8015B0A2DE6D1BBF8003026
:10696800FF2BA8BFFF23DBB2E9E7052D00F06D82FE
:1069780020D8022D00F0838040F29181032D00F091
:106988003A82042D40F0D880A04920462A46FCF7D8
:10699800E3F900212046FCF70FFA22680021531C76
:1069A8000125236028462B46543711706381BD4664
:1069B800BDE8F08F242D60D040F20381282D00F02F
:1069C800DC81382D40F0B8800A68914B0125511CB4
:1069D8002160157022680521501920601170226805
:1069E8000A21501920601170226800215019206076
:1069F800117022681978501920601170226859782E
:106A080050192060117022689978531923602B4619
:106A18001170284654376381BD46BDE8F08FA02D1C
:106A280019D040F21181B82D00F0E381FE2D40F01D
:106A38008380784D05F1080635F8021B2046FCF7DF
:106A4800BBF9AE42F8D101252B462846543763815D
:106A5800BD46BDE8F08F704B08461968FCF794F9FD
:106A68006E4B20461968FCF78FF96D4B1968204664
:106A78000125FCF789F92B46E7E76A4BF6E704227C
:106A8800694920460125FCF767F92B46C1E70B68E1
:106A9800DFF8AC81591C012221601A702368002597
:106AA8009A1822601D70236898F85B20591C216091
:106AB8001A70236898F85A20591C21601A70B8F87F
:106AC80056102046FCF778F929462046FCF774F959
:106AD800B8F858102046FCF76FF9A8F1020508F13C
:106AE800480635F8021F2046FCF766F9AE42F8D191
:106AF80022684E4B0C21501C20605D1811702268D2
:106B080013F8011F501C9D4220601170F7D12368B3
:106B18000222591C21601A70B8F85C102046FCF754
:106B28004BF90125B8F85E102046FCF745F92B46CD
:106B38006FE7522D3FF431AF21462846FDF738FC68
:106B4800034600287FF47FAF742D00F0BB80772DBB
:106B58000DD13268716891421EBF531C33601178A1
:106B6800334A08BF1946204624F0ACFF6BE7F52DE1
:106B780001F0BC82472D00F0A781392D336800F061
:106B8800A88200F29E82212D01F06982292D40F011
:106B9800E1825A1C32601B780A2B01F03F83502B8C
:106BA80041F0D3813046FCF7C5F8DFF89880A8F8A3
:106BB80000003046FCF7BEF80125A8F802002B4675
:106BC80027E7202DB8D10B681A4D591C6A78216027
:106BD8001A7023682A78591C21601A702368AA78C9
:106BE800591C21601A7029892046FCF7E5F82368AA
:106BF8006A79591C21601A702268A979CFE600BF0A
:106C080035610020383003087C290020E559002030
:106C1800D73E002058610020ACF7FF1FB0F7FF1FD8
:106C2800B4F7FF1F184000205C5F0308DD770020E1
:106C3800F1AF02080078002067666666A429002084
:106C4800947700209C2A0020822D7FF475AF0B6872
:106C58008B4A8C4D11788C4A581C20601970118908
:106C68002046FCF7A9F8894B22681B88FF2B02F104
:106C78000101A8BFFF2321601370A96881F31001E7
:106C880089B22046FCF798F8296801F30F0189B208
:106C98002046FCF791F87E4B226819787FE6012D93
:106CA8007FF44AAF0B680022591C21601A702368D0
:106CB8005A1C22601D7022682421531C23602B4615
:106CC8001170A6E63268716891421EBF531C33608A
:106CD8001178704A08BF1946204624F0F3FEB2E640
:106CE8006D4B1E78043616F0FF063FF4ACAE6B4BC6
:106CF800DFF8CC811E4403F1010A4FF00A0924E0B1
:106D0800B9F1500F00F09C81B9F15A0F00F0B5812C
:106D1800B9F1320F00F0B481A9F13C00C0B21328D8
:106D280040F2B1810025294623685A1C226020467A
:106D380083F80090FCF740F829462046FCF73CF819
:106D4800B2453FF480AE1AF8019BB9F10A0FD7D1CA
:106D5800534B9D68196805EB85054FF6FF736D0069
:106D68009D42A8BF1D469942A8BF194625EAE57568
:106D780021EAE171ADB289B2D6E70B68DFF8449138
:106D8800484E591C022221601A7023684FF00608E9
:106D98005A1C226083F8008023680A22591C21604B
:106DA8001A70236801255A1922601D70B9F800105D
:106DB8002046FCF701F8B9F802102046FBF7FCFF63
:106DC80023685A19226083F80080236850225919D1
:106DD80021601A7023680022591921601A703188BD
:106DE8002046FBF7E9FF71882046FBF7E5FF2B46B5
:106DF8000FE62D4B3AE60B685A1C0A601D700B68AB
:106E08000222591C21601A70C7E5204B0A681B88AA
:106E18001C4DFF2BA8BFFF23511C21601370A968CC
:106E280081F3100189B22046FBF7C6FF1F4B2046AD
:106E38001988FBF7C1FF296801F30F0189B22046C1
:106E48000125FBF7B9FF2B46E3E50B22184920463D
:106E5800FBF782FF082217492046FBF77DFF012533
:106E6800072215492046FBF777FF2B46D1E5002A74
:106E78003FF4E9AD114B136001252B46C9E500BF6E
:106E880056620020205B002000780020406200202D
:106E9800287800206DB902083561002048300308C1
:106EA800D42900209C2A0020903300201678002046
:106EB800645F0308705F03087C5F0308E142000811
:106EC800A02A0020F0320020726835687B623046C4
:106ED800551BFBF717FF052D38627B6A01F2858188
:106EE8008026B346012594E80600521A103AB242A9
:106EF800B8BF1FFA82FB924A396A92683A61521AFD
:106F08009345396A7B622046FA6088BF1FFA82FB84
:106F1800FBF73AFF7B6A002B01F04581002D41F019
:106F2800BE802368C7F800D05D71C0B00533C7F8CC
:106F380004D0FB61BBF1000F01F0DD823B6A3A69C6
:106F4800934281F0D482AA463E6A7D62BC60802565
:106F58005446FB681C1B7A4BB4F5807F28BF4FF45E
:106F680080749B68A2199A4288BF9C1BFCF7D8FAC8
:106F780022467C6830462146FCF752FBF969786165
:106F880004EB000C0B78BB6164452ED2DFF8C0918E
:106F98000CF1FF3C04F1FF3E1EF8013F09EB8302B0
:106FA80019F823405688ECB100234FF4004204F14D
:106FB800FF3832424FEA520202D00878284308705C
:106FC8006D0806D10AF1010A4D701FFA8AFA0131DB
:106FD8008025D34503D8F4456BD8434569DB013395
:106FE8009C42E6D1F445D7D1F9617B6A7A691344AA
:106FF8009BB2D3457B6206D97B6A3A6A1C46D6188F
:107008003B699E42A5D3BC68802D1CBF0AF10103D1
:107018001FFA83FA0AF1020189B22046FBF7CCFE77
:107028002368796A01255A19226020461D70FBF7EA
:10703800C3FE2368534423602B46D7F800D0E8E406
:10704800404B86E63388FF2BA8BFFF23DBB276E4EC
:1070580020F04AFC00283FF471AC03780A2B2ED8A4
:10706800B0F9023088FB0312DB17C3EBA2039BB213
:10707800FF2BA8BFFF23DBB261E4334B5D6869E6F1
:1070880098E8220067E620F02FFC00283FF44AAE7B
:1070980003780A2B3FF646AEB0F90430B0F9061073
:1070A80003EB830383F3500521EAE171ADB289B2A2
:1070B8003AE6FB69BC681A463B7E1370A4E70023D6
:1070C800D9E7552D17D0572D44D14FF0FF352B4612
:1070D8009FE45A1C32601A780A2A01F0CB803046A5
:1070E800FBF734FE3046FBF731FE01253046FBF74F
:1070F8002DFE2B468DE45A1C326093F80080B8F1BF
:10710800FF0F01F03C81B8F1FE0F01F0C28030465C
:10711800FBF710FE96E80C009B1A002B07DD531CAA
:10712800336013781BB9B8F10B0F41F21D81B8F128
:10713800240FCAD8054B012523F818002B4668E40C
:1071480088210020082A0020142A00209477002093
:107158005830030871680B3DCA1AEF2DB5D801A045
:1071680050F825F0D77C0008D3700008D3700008C9
:10717800D3700008D3700008D3700008D3700008DB
:10718800D3700008D3700008D3700008D3700008CB
:10719800D3700008D3700008D3700008D3700008BB
:1071A800D3700008D3700008D3700008D3700008AB
:1071B800D3700008D3700008D3700008D37000089B
:1071C800D3700008837C0008D3700008617C000835
:1071D800D3700008A57E0008D3700008D37000089B
:1071E800D37000087D7E0008D3700008237E000855
:1071F800D3700008F17D0008D3700008CB7D00082B
:10720800D3700008B97D0008D3700008617D0008BC
:10721800D37000080D7D0008D3700008D3700008F3
:10722800D3700008D37000084F6A0008D3700008B4
:107238007D7F0008D3700008D3700008637F0008C2
:10724800D3700008097F0008D3700008D3700008C5
:10725800D3700008D3700008CF7E0008D3700008F0
:10726800D3700008D3700008E77F0008D3700008C7
:10727800997F0008D3700008D370000827800008A1
:10728800D3700008D3700008D3700008D3700008CA
:10729800D3700008D3700008D37000088D7B0008F5
:1072A800D3700008DF7A0008D37000086D7A0008F0
:1072B800D3700008D5790008D3700008AD790008AC
:1072C8008F790008D3700008D3700008D3700008C5
:1072D800D3700008D3700008D3700008D37000087A
:1072E800D3700008D3700008D3700008D37000086A
:1072F800D3700008D3700008D3700008D37000085A
:10730800D3700008D3700008D3700008D370000849
:10731800D3700008D3700008D3700008D370000839
:10732800D3700008D3700008D3700008D370000829
:10733800D3700008D3700008D3700008D370000819
:10734800D3700008D3700008D3700008D370000809
:10735800D3700008D3700008D3700008D3700008F9
:10736800D3700008D3700008D3700008D3700008E9
:10737800D3700008D3700008D3700008D3700008D9
:10738800D3700008D3700008D3700008D3700008C9
:10739800D3700008D3700008D3700008D3700008B9
:1073A800D3700008D3700008D3700008D3700008A9
:1073B800D3700008D3700008D3700008D370000899
:1073C800D3700008D3700008D3700008D370000889
:1073D800D3700008D3700008D3700008D370000879
:1073E800D3700008D3700008D3700008D370000869
:1073F800D3700008D3700008D3700008D370000859
:10740800D3700008D3700008D3700008D370000848
:10741800D370000865790008D3700008497900081E
:10742800D3700008D3700008D3700008D370000828
:10743800D3700008D3700008D3700008D370000818
:10744800D3700008D3700008D3700008D370000808
:10745800D3700008D3700008EB780008D3700008D8
:10746800B3780008D370000811780008B7770008CF
:107478009B770008D370000881770008D370000854
:107488005977000847770008E7760008D3700008A6
:10749800B7760008D3700008D37000088D7600080E
:1074A8005F7600084B76000823760008037600080C
:1074B800D9750008D3700008C1750008D37000089A
:1074C800D3700008D3700008D3700008D370000888
:1074D800D3700008D3700008D3700008D370000878
:1074E800D3700008D3700008D3700008D370000868
:1074F800D3700008A1750008D3700008D370000885
:1075080047750008D3700008D3700008D3700008CE
:10751800D3700008D3700008D3700008D370000837
:107528002D750008A84B1B78DB073FF5CEAD01256C
:10753800FDF742FFFEF75EFD2B46FFF76ABA5A1CBD
:1075480032601A780F2A3FF6C0AD991C3160C2EB41
:10755800C2029E4958788854D81C30600A449978E9
:107568005170191D3160D9789170591D31601979A0
:10757800D170991D316059791171D91D316099798E
:10758800517103F108013160DB799371012520F015
:10759800C1FF2B46FFF73DBA3046FBF7CBFBDFF8C0
:1075A8003882A8F80E003046FBF7C4FB0125A8F87E
:1075B8000C002B46FFF72DBA3046FBF7BBFB844A7D
:1075C80000EB80004300012513802B46FFF721BA0A
:1075D8003046FBF7AFFBDFF82082A8F810003046F2
:1075E800FBF7A8FBA8F812003046FBF7A3FB012520
:1075F800A8F814002B46FFF70CBA1A46591C31603C
:1076080012F8020B3260DA1C597832609A781BF053
:1076180071FA00287FF417AA57E51A46591C3160F9
:107628006C4912F8020B087032606B495A788A70FC
:10763800DA1C3260664A9B78937001252B46FFF767
:10764800E8B9664B664918684E22012529F080F88A
:107658002B46FFF7DEB919465A1C3260614A11F809
:10766800020B1070316059785170D91C31609B78C9
:1076780093703046FBF75EFB5B4B0125D8802B46A9
:10768800FFF7C7B93046FBF755FBDFF85C81A8F870
:1076980000003046FBF74EFBA8F802003046FBF727
:1076A80049FB0125A8F804002B46FFF7B2B9DFF81B
:1076B8004C9199F80030002B3FF4C5A9DFF84081C0
:1076C80000253046FBF736FB0FF0DEFA99F800305C
:1076D800A8EC010A01359D42F3DBFFF7B4B90D2A86
:1076E8007FF4F3AC5A1C32601D78072D3FF6EDACE1
:1076F800DFF8109130464FF00C08FBF71BFB08FB36
:1077080005F809EB0805A8803046FBF713FBE8806D
:107718003046FBF70FFB336828811A46591C316045
:1077280012F8021BA97232605B78EB723046FBF7E5
:10773800E9FA012549F808002B46FFF76AB93046EF
:10774800FBF7F8FA294B012518802B46FFF761B99A
:107758005A1C32601878060600F1D2861A4B1B783C
:10776800DD073FF570A9032828BF00200125FDF794
:1077780007FE2B46FFF74DB9134B1B78D8073FF58B
:1077880062A90125FDF7E8FEFEF734FC2B46FFF75A
:1077980040B90D4B1B78DA073FF555A9144A137801
:1077A800012543F0040313702B46FFF732B9064B4B
:1077B8001B78D9073FF547A90E4B4FF4C87201252E
:1077C8001A802B46FFF725B9EC5F0020B86300202C
:1077D800103E0020244B0020403A0020DC590020B5
:1077E800C038030858320020683500205432002081
:1077F800FC770020D87800205C6A002035610020E2
:10780800BC34002050660020092A7FF75EACDFF800
:1078180068831A46591CD8F80050316012F8021BC8
:10782800297032605A78AA70DA1C32609A78642A11
:1078380003F10401A8BF64226A713160DA78642A0E
:1078480003F10501A8BF6422AA7131601A79EA71AF
:107858009A1D32605A79642A03F10701A8BF64228D
:107868002A7231609A79EA7003F108023260DB7992
:107878002B713046FBF75EFA726833686881D11A5B
:1078880000290CDD591CD8F800003160521A002A72
:107898001978417203DD9A1C32605B7843700125C8
:1078A80027F0B8F82B46FFF7B4B8A84A1068DA1CD6
:1078B80001462133951E356012F8035C0D70551E84
:1078C800356012F8025C4D70326012F8015C8D7000
:1078D8000332934201F10301ECD121F0CDF9FFF716
:1078E800B2B8C2F34705122D3FF6EFABC5B107F1A9
:1078F800500307F12A0A03EB4508D146A8F12608E8
:107908003046FBF717FA29F8020FC845F8D1904B13
:107918003AF8022F23F8022FD145F9D1112D09D8B1
:107928008C4A6B00023B13440021223223F8021FC9
:107938009A42FBD1884A01231D461370FFF769B8A4
:10794800DFF8388200233046C8F80030FBF7DAF950
:107958000125C8F800002B46FFF75BB81A46591CEA
:10796800316012F8025B3260DA1C5878326099781C
:10797800002D00F0D085012D7FF465A826F016F9BA
:107988002B46FFF746B8754A127812F001017FF4CA
:107998009CAB5A1C32601878012526F049F82B4612
:1079A800FFF737B81A46591C31606D4912F8020BB7
:1079B800C87032606B495A784A71DA1C32606A4A78
:1079C8009B78D37001252B46FFF723B83046FBF789
:1079D800B1F93046FBF7AEF93046FBF7ABF9304664
:1079E800FBF7B4F93368594D1946581C2A683060BA
:1079F80011F8020B82F82C003160597882F83610A1
:107A0800D91C31609B7882F837303046FBF79EF9F5
:107A18003046FBF79BF93046FBF798F93046D5F826
:107A28000080FBF787F9A8F83A003046D5F80080BF
:107A3800FBF780F933687268A8F83800D11A012971
:107A48000ADD591C2A6831601B7882F82E303046CE
:107A5800FBF77CF933687268D31A032B00F361854E
:107A680028683AE75A1C3260384DDFF814811B78D1
:107A780088F805303046D5F80090FBF75BF9A9F88F
:107A880020003046D5F80090FBF754F97268336847
:107A9800A9F81E00D11A072900F3BB84D11A0329BB
:107AA80000F3A984D21A002A05DD591C2A6831601E
:107AB8001B7882F82630FDF789FC17F0DFFF2B4B87
:107AC8001B68002B00F03B852868012520F0B6FDD7
:107AD8002B46FEF79EBF1A46591C3160DFF8A0807E
:107AE80012F8021B88F80210326021495A780A708D
:107AF800DA1C32601F4D9A782A711A1D3260DB78C1
:107B0800092BA8BF09233046AB70FBF713F933687C
:107B180072682880D11A012905DD3046FBF70AF979
:107B280033687268E8819A4240F04D84FDF74EFC54
:107B3800336872689A423EF486AF5A1C32601B78EA
:107B4800EB7001252B46FEF764BF00BFDC5900200F
:107B5800E6360020E83600200C370020EC5F0020D5
:107B6800403A0020245E0020103E0020647500206A
:107B7800686500205C6A0020B878002090330020F7
:107B8800244B00203046FBF7D5F8054616F086FB57
:107B9800FF283EF458AF3F2D00F2578407F15008F4
:107BA800002308F8243D4FEAD509414607F12B0088
:107BB80087F82B3009F1010916F070FA97F82B3085
:107BC8005FFA89F905F007054B4505F1010503D171
:107BD80097F82C30AB4203D02946484616F04AFBAA
:107BE80033687268D21A012A7EF72DAF5A1C07F142
:107BF8005000326000221D7800F8252D16F042FA58
:107C080097F82B30AB420AD0B24B1B683BB19A793C
:107C1800AA4204D31B681B690BB1284698473368EE
:107C28005A1C3260404600221D7887F82C2016F036
:107C38001DFA97F82C30AB423EF405AFA54B1B68F4
:107C4800002B3EF400AF1B685B69002B3EF4FBAED3
:107C580028469847FEF7F7BEDFF8A0820023C8F849
:107C680000303046FBF74EF8D8F8003001250343C2
:107C7800C8F800302B46FEF7CCBE5A1C32601D787F
:107C8800132D3FF622AA9A1C326058787B6223F0A3
:107C980053FF00283FF419AA7B6A8F4A017802F83B
:107CA8002510D91C316002EB850299785170191D95
:107CB8003160D8789070581D306088491B79D3702E
:107CC8000868012526F034FE2B46FEF7A2BE844B39
:107CD800102A4FF0000128BF1022196059609960DE
:107CE800D9601974002A3EF4AEAE3168013B0A44EB
:107CF8000131316011F8010C03F8010F9142F7D1FD
:107D0800FEF7A1BE0721B2FBF1F1C1EBC105521B81
:107D18007FF4DBA9C9B201F1FF395FFA89F90029BB
:107D28003EF491AEDFF8BCA109F1010915465A1CD1
:107D3800326093F900106B4B4FF0000893F9022062
:107D48008A4203F1080300F0EA8208F10108B8F159
:107D5800050FF3D1FFF7B9B95A1C32601A780E2A09
:107D68003FF6B3A9991C31605D78032D3FF6ADA9A4
:107D78005D48062101FB02F1421803F1030E55711B
:107D8800C6F800E09D784554191D3160D9785170C6
:107D9800591D316019799170991D31605979D170E7
:107DA800D91D31609B79137101252B46FEF731BE31
:107DB8005A1C32604D4A1B78537501252B46FEF735
:107DC80028BE591C31601D781F2D3FF67EA9052A53
:107DD8007FF47BA93046FAF795FF454B43F8250019
:107DE80015F0CEFEFEF72FBE414D05F14008304696
:107DF800FAF7A0FF3368A5F88000591C1A463160CD
:107E080012F8021B85F8821032605B7885F883309F
:107E18000435A845EBD1FEF716BE5A1C3260334D27
:107E28001B782B723046FAF785FFA8833046FAF79D
:107E380081FF28833046FAF77DFF32686883531C38
:107E480033601278EA747268D31A032B00F3308314
:107E58003368D11A052900F31B83D21A002A7EF74A
:107E6800F2AD5A1C32601B7885F8213001252B466B
:107E7800FEF7CFBD581C30601E4A1D781570091AD0
:107E880000297EF7E0AD991C31605B78003318BF9C
:107E98000123012553702B46FEF7BBBD3046FAF788
:107EA80049FFDFF85480C8F800003046FAF742FF6F
:107EB800C8F804003046FAF73DFF0125C8F8080065
:107EC8002B46FEF7A6BD0125FBF78CFB2B46FEF7DC
:107ED800A0BD00BFD859002084750020DC590020BF
:107EE800C4590020686700209C3300205C4F0020A4
:107EF8009058002080750020F8310020184000209C
:107F08005A1C3260C94A1B78DFF858831370002363
:107F1800C8F800303046FAF7F5FE3368D8F8002084
:107F2800C349C44D10435A1CC8F8000032601B787E
:107F38000B723046FAF7FEFE28603046FAF7FAFE72
:107F480068603046FAF7F6FEA8603046FAF7F2FEA7
:107F58003046FAF7EFFEFEF776BDB74A03F108019F
:107F68000133336013F8010C02F8010F9942F7D17D
:107F7800FEF769BD591C1A463160B04912F8020B68
:107F8800887032605B784B7001252B46FEF741BD47
:107F98005A1C326093F80080B8F1110F3FF695A88B
:107FA8009A1C3260A64D5B7805F818303046FAF70F
:107FB800C1FE40F6CA039842A8BF184640F2EE2315
:107FC800984205EB4801B8BF18460125A0F2EE22F9
:107FD8002B46192092FBF0F24A70FEF71ABD1A469A
:107FE800591C984D316012F8021B297132605B7878
:107FF8006B713046FAF79EFE336828805A1C32604F
:108008001B78AB713046FAF795FE336868805A1CC6
:1080180032601B78EB7101252B46FEF7FABC8A4AC1
:108028001278012A3EF60FAD18465A1C3260DFF866
:10803800388210F8022B88F802203060DA1C587851
:1080480032608A1A012A997840F316823046FAF784
:1080580071FE0125A8F800002B46FEF7DABC1A4687
:10806800591C3160794D12F8021B697032605A78D8
:108078002A70DA1C32609B78AB703046FAF75AFEE9
:1080880033682881591C1A46316012F8021B69713D
:1080980032605B78AB7101252B46FEF7BABC6C4B9E
:1080A8003A6A9B68D4F800905A449A4240F2AB80EE
:1080B8003A6AA3EB0208FBF733FA42464946386AA4
:1080C800FBF7AEFA236803442360002D3EF4BBACF3
:1080D80086427EF7B8AC002100E0236801305A1CC4
:1080E800B04222601970F8D1FEF7ADBC33687268EF
:1080F8009A4240F0E180574BFF221A704FF0000A75
:10810800554D25F0C7FA51462022544885F800A05D
:108118002AF033FE87F82CA097F82C30072B00F2B2
:108128005081DFF848914D4E524697F82C3003EBBA
:10813800430309EBC3035B7CE3B197F82C3003EBF3
:10814800430309EBC30320215B699BB197F82C30EB
:1081580003EB430309EBC303586946F82200F9F718
:1081680017FF2B7856F82300FAF7D4F82A7801324B
:10817800D2B22A7097F82C300133DBB287F82C3052
:1081880097F82C30072BD0D92368591C21601A7016
:10819800B8F1000F3EF457AC314BC8F80030012558
:1081A8002B46FEF736BC002D7FF479AF59462046A2
:1081B800FAF702FE23685A1C22601D70244B2668B9
:1081C8009D683B6A0BEB03029542C0F00681FBF702
:1081D800A7F95A463146386AFBF722FA236801257F
:1081E800034423602B46FEF714BC3046FAF7A2FD81
:1081F800326871687B6A9142834640F08680064601
:108208001D46FEF770BEFBF78BF95A464946386A99
:10821800FBF706FA23680344236059E73046FAF768
:1082280089FDDFF84C80FEF7C2BC00BF80750020D6
:108238005C4F0020F83100205B4F0020DC780020E4
:108248003C390020843500200540002000780020BB
:1082580088210020F423002095620020683800203F
:108268005D7E020818400020107800209C690020DC
:10827800F03200209A1C3260B64A59781170D91C25
:10828800316099785170191D3160DB789370FEF771
:10829800DABB9A1C32605D78022D3EF616AF304686
:1082A800FAF748FDAC4B03EB45034FF0FF35A3F855
:1082B8005C002B46FEF7ADBB5A1C19463260A74836
:1082C80011F8022B027031605B784370042A03D9DD
:1082D800FF2A7EF462AB11E7A1490978994205D8D3
:1082E800022A7EF45AABFF2B7EF457AB2368012594
:1082F8005A1922601D70B8F1000F3EF4A4AB994BD7
:10830800C8F800302B46FEF784BB511C3160127848
:108318001D46131C064618BF0123FEF7E4BD0AEBF1
:10832800C80B30468BF80210FAF704FD32682AF8B9
:1083380038001346511C316013F8021B8BF80310E8
:10834800336053788BF80430D31C336093788BF800
:108358000630131D33600135D2788BF80520A94506
:108368007FF4E5ACFEF76FBB7B4B0030984418BF39
:108378000120012588F84A002B46FEF74ABB304603
:10838800FAF7E4FC3368DFF8D0811A46591C3160EB
:1083980012F8021B88F85B1032605B7888F85A3054
:1083A8003046FAF7C7FCA8F856003046FAF7C2FC80
:1083B8003046FAF7BFFC0125A8F858002B46FEF70F
:1083C80028BB5246E0E65A1C32601B78003318BFBF
:1083D800012388F80730FFF7A9BB3B6AED1AFBF7C2
:1083E8009FF82A463146386AFBF71AF9236803448E
:1083F8002360FEF728BB3046FAF79CFCA8F80E006D
:108408003046FAF797FC33687268A8F81000FFF74F
:1084180049BB3046FAF78EFCA8F80A003046FAF74E
:1084280089FCA8F80C003046D5F80090FAF782FCD1
:10843800A9F822003046D5F80090FAF77BFC33689B
:108448007268A9F82400FFF729BB07F12C084046F9
:1084580015F000FEBB8DAB423FF4C2AB424B1B682C
:10846800002B3FF4BDAB1B689B69002B3FF4B8ABF6
:1084780028469847FFF7B4BB3C4B1A88012512FBE6
:1084880000F22B4692FBF1F2A8F80020FEF7C1BAE1
:108498005A1C32601B78EB723046FAF733FC3368AB
:1084A800E8605A1C32601B782B7433687268D4E415
:1084B8003046FAF73FFCA8843046FAF73BFC3368AD
:1084C8007268E884D11A03297FF7C3AC1A46591C8D
:1084D800316012F8021BA97732605B7885F820308A
:1084E8003046FAF727FC336872686884B1E47D6225
:1084F800AA46FEF78FBDDA46C7F824B0FEF78ABD54
:1085080000F07F00032828BF0020012525F06AFB22
:108518002B46FEF77EBA012520F026FA2B46FEF7F9
:1085280078BA3046D5F80080FAF704FCA8F832008B
:1085380030462E68FAF7FEFBB086FFF791BA0C4872
:108548000C490D4A0D4B036001250B6013602B4647
:10855800FEF75FBAD73E002094770020F42300206E
:1085680035610020F9420008D8590020C073002066
:10857800A8640020FC64002064650020F10600085F
:108588002DE9F04F2DED028B93B083461AF0BAFF18
:10859800B94B1D7825B113B0BDEC028BBDE8F08F47
:1085A800B64B1B685B05F6D5B54FB64E3B68002B3E
:1085B8005CD0B54C3168D4F810218A1A7C2A55D978
:1085C80094F81421DFF810839FEDB08AC4F81011D5
:1085D800013284F814214FF0240A5E20984750464F
:1085E8003B689847AA4BF8EC016A9B8A07EE103A59
:1085F800F8EEE66AB8EEC77A0AF1010AC6EE877A9B
:108608005FFA8AFA67EE887AFDEEE77ACDED027AAC
:10861800BDF908905FFA89F01AF0E2FEC9F3072065
:108628001AF0DEFEBAF1270F3B68D6D15E209847D4
:108638003B6830209847974BD3F800805FFA88F062
:108648001AF0CEFEC8F307201AF0CAFE3B685E2077
:10865800984794F8143113F0030800F0898113F057
:10866800070801F07782282B01F04A838A4B1B7890
:10867800002B72D0844C894AD4F81831ABEB030331
:10868800934200F2898794F82091B9F1000F35D10F
:10869800DFF84882D8F80000F8F742FEC0B2012897
:1086A8000FD902287E4F41F0C4833B78002B41F05C
:1086B8001086D4F82431ABEB0303B3F57A6F81F05D
:1086C800B787D4F82831002B47D094F82031C3B9A4
:1086D800744B1B689B7801211E3B00228B4284F857
:1086E800201184F8342141F26687D8F8000002216D
:1086F80004301AF0EDFD94F82C3111E0D4F828314B
:108708005BB3D4F8303140F6B732ABEB0303934296
:1087180023D994F82C31002B01F0DB82DFF8BC81DF
:10872800013BDBB284F82C31002B00F0A987D4F888
:10873800287194F8342117F8011B94F83531D8F8CA
:108748000000C4F828710A44013384F8342184F8FD
:108758003531F8F7E9FDC4F830B1534BD6F800804D
:108768001B7843B1514F386828B1514B1B78013BF6
:10877800012B40F295874F4B1B7863B14E4F3B68F6
:108788004BB1414CD6F80090D4F84C31A9EB030317
:10879800632B00F22081DFF8488198F80030022B23
:1087A80001F076823E4F97F87430032B00F0528721
:1087B800424B1B7873B1424D2B685BB1324CFDF7CD
:1087C800F7FED4F85831029044F61F62C31A934258
:1087D80000F25C813B4B1B78002B40F083803A4BC6
:1087E8001B7843B1284CD4F8A83203F5C333A0331F
:1087F8009B4580F07F86354B1B78002B3FF4CBAE32
:10880800214E334C334D06F2C9272068F8F788FD0E
:1088180000283FF4C0AE2068F8F77AFD2B78804630
:108828005A1E33B120682A70F8F77AFD0028F2D171
:10883800B1E603223946781E2AF085FA96F8C8323E
:1088480096F8C92286F8CB8283F47F4383F0FF032E
:108858009B1A1FFA88F89BB2B8EB132FD5D196F85C
:10886800CA22DBB29A42D0D1781E1FF0B7F82B7813
:1088780018442870C9E700BF8A480020CC4D002062
:10888800F05C0020F8600020F823002000007A4403
:10889800B4480020EC590020825D00203F0D030001
:1088A8001C000020EC5C0020845D00202C5B002074
:1088B8008C5D0020945D0020785E00209C5D002087
:1088C800A05D0020E05D0020F15D0020A65D002095
:1088D800AC5D0020B05D0020EC480020E85C002082
:1088E8005E3800205B4C2278A2B15B4B9B7A53B177
:1088F800FDF75EFE594B1B68C31AA3F57A73B3F5EF
:10890800FA6F07D82278564B56491868F8F7D8FCFA
:1089180000232370544CD4F8A03203F5C333A0339A
:108928009B45FFF45CAF514DC4F8A0B22B78002BE7
:1089380041F049834E4D2B78002B41F031824D494F
:1089480094F8A4228D5CE90701F10685AA0701F1D4
:10895800C6846B0701F1B283474A94F8A4321178B0
:10896800013393FBF1F201FB123384F8A43236E7AA
:10897800D4F8102141F288339A4201F226823B68EA
:108988005E2098473B68142098473C4B3C4AB3F913
:10899800043082FB03124FEAE378C8EBA2080FFA0F
:1089A80088F85FFA88F01AF01BFDC8F307201AF060
:1089B80017FD3B685E2098473B681C2098470020BD
:1089C8001AF00EFD00201AF00BFD3B685E20984758
:1089D80094F8143143E6DFF8A4A0DFF8A48041201E
:1089E8001AF024FCBAF9023088FB0320DB17C3EB2A
:1089F800A00080B21AF000FCBAF9003088FB03200E
:108A0800DB17C3EBA00080B21AF0F6FBBAF904300A
:108A180088FB0320DB17C3EBA00080B21AF0ECFB45
:108A2800184B38681978F8F77FFC94F8503113F030
:108A3800010801F01F82144AC4F84C910133DBB2DB
:108A4800A2FB0312D20802EB8202A3EB420384F8D2
:108A58005031A0E6745D00205C4F0020CC37002028
:108A6800E45D0020345D0020F8230020E85D00204C
:108A7800E95D0020EC5D0020F05D0020BC5900207D
:108A88006766666670600020CDCCCCCC94F85E3109
:108A9800002B41F08081DB4B1A6802F00803002BA1
:108AA80048F603414AF60B404BF60F4349F6074791
:108AB80004BF03460F4612F0040F4FF0190118BF08
:108AC8001F46920684F85E1103D547F4804747F0A5
:108AD8002007CD4B5A79C7F30909002A41F0D585FB
:108AE8009B79002B41F0D786984664204FF0FF3AD7
:108AF8004FF0000C0A970B97ADF834C0CDF83AC088
:108B0800CDF83EC0CDF842C0CDF83090ADF83680F3
:108B1800ADF838A08DF846000AAF0FCFDFF800E3B4
:108B280084F805C0AEE80F0097E80F00AEE807002C
:108B38002EF8023B71464FF0010C1B0CFE271F203C
:108B4800C82201F81E39A770A27184F807C0E07026
:108B580094F86E01207180F0F10383EA0313DAB20E
:108B6800130983F0E70343EA022383EAC2031BB233
:108B780083EA0312D2B2C3F3072383EA121343EA48
:108B8800022383EAC2031BB283F0C80282EA0212FC
:108B9800D2B2C3F3072383EA121343EA022383EA18
:108BA800C2031BB283EA0C0787EA0717FFB2C3F3B5
:108BB800072282EA171242EA072200EB0C0382EA34
:108BC800C7070EEB0C0084F86E31278011F8013BC3
:108BD8007B4083EA0313DBB21A0982EA172242EACE
:108BE800032282EAC3031BB29FB281422780EDD1E0
:108BF80083F07C0383EA0313DBB24FEA131E8EEA89
:108C0800172E8EEA032E8EEAC30E0FFA8EFE1FFA77
:108C18008EFADFF810C2A4F800A05FFA8EFE4FEAC1
:108C28001A2A84F828A084F827E00CF5CB7804F1F8
:108C38002209DCF80000DCF80410DCF80820DCF875
:108C48000C3047460FC70CF1100CCC45B846F0D194
:108C5800DCF8000038606D4F9CF8043088F8043068
:108C680007F1270884F8BDE184F8BEA117F8011FB1
:108C78002868F8F759FBB845F8D194F85F31002B0C
:108C880041F084806249326809780A2084F85F01DB
:108C9800002901F009825F4F01293888069041F2C6
:108CA8000F860229B7F802E001F00A85B888059016
:108CB800032901F0FE85F8880490042901F015863F
:108CC8000529388901F00C860629B7F80A9001F0C1
:108CD80003860729B7F80C8001F0FB85FB8903930D
:108CE80094F86E110A920B4683F0300282EA02125F
:108CF800D2B217094849079387F07A0747EA02274B
:108D08000988237187EAC202444FC1EB012187FB1E
:108D1800013A069B4FF0000C63F30F0C059B6EF3B2
:108D28001F4C4FF0000E63F30F0E049BCDF82CC0C0
:108D380012B28A440027C91763F31F4EC1EB6A2A8F
:108D4800039BCDF830E082EA021160F30F070020A0
:108D5800C9B268F30F00C2F3072269F31F4782EA1A
:108D6800111263F31F404FF000090D978DF83DA0D5
:108D78000E908DF83C9042EA01220DF1280C82EA0F
:108D8800C107BCE80F003FB287F0C80888EA081896
:108D9800DFF88CE084F805905FFA88F8C7F30727B6
:108DA800AEE80F0087EA181747EA08239CE8030093
:108DB80083EAC8031BB283F023024EF8040B82EA4D
:108DC8000212D2B2C3F30723079F83EA1213704635
:108DD80043EA022383EAC20207F1010C20F81419BE
:108DE8004FF023081621FE27C82384F86EC122807D
:108DF80084F807800EF1020EA770E170A371114686
:108E080012E000BF34780020007800208F25002071
:108E180068490020C85F00201678002003082080D9
:108E280000240020FA23002010F8013B4B4083EA7D
:108E38000313DBB21A0982EA112242EA032282EA08
:108E4800C3031BB299B270452180EDD183F0F403BE
:108E580083EA0313DBB24FEA131E8EEA112E8EEA61
:108E6800032E8EEAC30E0FFA8EFE1FFA8EF8E44F19
:108E7800A4F800804FEA182C5FFA8EFE84F81EE0F2
:108E880084F81FC07968BA683868FB6807F5CB783A
:108E9800A8E80F0038697969BA6904F29717A8E851
:108EA800070004F2B51884F8B5C184F8B4E117F8DE
:108EB800011F2868F8F738FAB845F8D194F866C160
:108EC800BCF1000F40F05C87CE4B94F86E71B3F99B
:108ED8000010B3F90220B3F904309FEDCB6ADFF834
:108EE80044E384F805C007EE103A33680A9387F024
:108EF8006A0383EA031306EE901AD9B20B0983F0CA
:108F0800D50343EA012383EAC1031BB283EA0311B1
:108F18005242C9B207EE902AC3F3072383EA11131A
:108F280043EA0123F8EEE77AF8EEE66AB8EEC77A84
:108F380083EAC1031BB267EE867A66EE866A27EE7D
:108F4800067A002083F0C808CDED0C7ACDED0B6AC7
:108F58008DED0D7A0E900F90109088EA08160DF19D
:108F68002809F6B2C3F30728B9E80F0088EA1618EB
:108F780048EA062888EAC6080FFA88F8AEE80F001B
:108F880088F01E0699E8070086EA0616F6B2C8F3C6
:108F9800072383EA161343EA06238EE8070083EAC9
:108FA800C6061C20C8214FF005084FF01E0CFE23F2
:108FB8007A1CE070A17184F8668184F807C0A370F8
:108FC800AEF1100127710EF10C00268084F86E2195
:108FD80011F8013B734083EA0313DBB21A0982EAF2
:108FE800162242EA032282EAC3031BB29EB28142DE
:108FF8002680EDD183F0270383EA0313DBB24FEA1F
:10900800131E8EEA162E8EEA032E8EEAC30E0FFA70
:109018008EFE1FFA8EFC7A4FA4F800C05FFA8EFE0F
:109028004FEA1C2C84F825C084F824E007F5CB7897
:1090380004F1220938687968BA68FB6846460FC6A1
:1090480010374F45B046F5D1704E3B88A8F8003030
:1090580006F1240784F8BAE184F8BBC116F8011FA9
:109068002868F8F761F9B742F8D194F867A1BAF11E
:10907800000F40F07F86664B1B68052213F0140F23
:1090880084F8672140F08987DFED627A94F86EC131
:109098005C4B614AB3F90410B2F906205F4E604890
:1090A800CDED0C7A8CF0220383EA0313DFB23B097F
:1090B80083F0590343EA072383EAC703B2F5FA6F3B
:1090C8001BB2A8BF4FF4FA6283EA0317FFB2B2F5E6
:1090D8007A7FC3F3072383EA1713B8BF4FF47A7272
:1090E8004FF0640E43EA0723A2F57A720EFB02F2F0
:1090F80083EAC70386FB02E680FB01E01FB2D217B2
:10910800C9174FF00008C2EBA612C1EBA00187F007
:10911800C806ADF83A20ADF83810CDF82880CDF85B
:109128002C80CDF834800DF1280E86EA0616BEE8AC
:109138000F00F6B2C7F3072787EA161747EA06278C
:1091480087EAC606374FDEF800E084F804C00FC788
:1091580036B286F04A0383EA0313DBB2C6F307216B
:1091680081EA13113A4641EA03210CF1010C81EA24
:10917800C303142042F810E9FE264FF04A0E0021DE
:1091880084F86EC14FF0C80CE0702380043784F86F
:1091980007E0A670617184F806C0184612F8011B32
:1091A800414081EA0111C9B20B0983EA102343EA5D
:1091B800012383EAC10109B288B2BA422080EDD105
:1091C80081F0140181EA0111C9B24FEA111E8EEA39
:1091D800102E8EEA012E8EEAC10E0FFA8EFE1FFAAD
:1091E8008EF6074F26804FEA16295FFA8EFE84F81E
:1091F8001D9084F81CE079683868BA68FB6813E049
:10920800FA230020BC59002088C3E43A8F250020A7
:109218003478002000000000C85F0020D34D6210A1
:109228006766666600240020B7F8188007F5CB7CCF
:10923800ACE80F0038697969ACE8030004F29716C6
:10924800ACF8008084F8B391B04684F8B2E104F237
:10925800B31918F8011F2868F8F766F8C145F8D15E
:10926800C44BC54A1B781278013B12F00100DBB2EF
:1092780014BFC0214021172B03D8C04A134493F8C8
:1092880030A0BF4B1A8893071ABF002341F0100182
:10929800012312F4027F18BF022312F0100F18BF27
:1092A800062312F0200F18BF1023002841F0B281C6
:1092B8004FF0030C94F86E910A9389F0460383EA01
:1092C8000313DAB2130983F0920343EA022383EA11
:1092D800C2031BB283EA0310C0B2C3F3072282EAB7
:1092E800101242EA002282EAC00212B282F0C80ECC
:1092F8008EEA0E1E5FFA8EFEC2F30722002382EA70
:109308001E1203208DF82CA08DF82FC08DF82D305B
:1093180042EA0E2C8DF82E108DF830000AAA07CAE2
:109328008CEACE0E0FFA8EFEDFF868A2E3718EEAA1
:109338000E1CAAE803005FFA8CFCCEF3072E8EEA17
:109348001C1E4EEA0C2181EACC0C94F808E08AF83D
:1093580000200FFA8CFC8EEA0C0E8EEA0E1E5FFAC5
:109368008EFECCF3072282EA1E1242EA0E22607AAF
:10937800A17A94F80BC0637182EACE0212B250400F
:1093880080EA001E5FFA8EFEC2F3072080EA1E10F4
:1093980040EA0E2080EACE0000B2414081EA011185
:1093A800C9B2C0F3072282EA111242EA012282EA14
:1093B800C10212B28CEA020C8CEA0C1C5FFA8CFC1B
:1093C800C2F3072282EA1C1242EA0C2294F80CE04B
:1093D800607BA17B94F8108084F8049082EACC0228
:1093E80012B28EEA020E8EEA0E1E5FFA8EFEC2F3EB
:1093F800072282EA1E1242EA0E2282EACE0212B244
:10940800504080EA0010C0B2C2F3072282EA10126C
:1094180042EA002282EAC00212B2514081EA0111F6
:10942800C9B2C2F3072282EA111242EA012282EA91
:10943800C102E17B13B281EA030282EA0212D2B2CC
:10944800C3F3072383EA121343EA022383EAC2031E
:109458001BB288EA030282EA0212D2B2C3F30723DC
:1094680083EA121343EA022383EAC2031BB283F09E
:10947800320282EA0212D2B2C3F3072383EA12133A
:1094880043EA022383EAC2031BB29AB24FF0FE0CEE
:109498004FF0090EC82009F10101DBB284F802C0BF
:1094A80084F803E04FEA122CA07184F86E11228030
:1094B80084F812C0637438687968BA68B7F80C9091
:1094C8000AF5C47EAEE807000AF5CC7A8EF8028069
:1094D800AEF8009084F8A8C184F8A73116F8011FE7
:1094E8002868F7F721FFB245F8D1029BC4F8583134
:1094F800FFF770B994F8AC32204AC4F8A8B202EB6E
:109508008302926C42B312AD04F2B3231D4E45F8A8
:10951800203D002104F2C52331800B9380211523BF
:10952800A52784F8B232284684F8B11284F8B072BC
:10953800904728463188F9F73FFC0A9D124804F500
:109548002C716D1A152DA8BF15252A4627F000F98C
:109558000E4A94F8AC3215700D4A013382FB03129F
:10956800A2EBE37202EB42029B1A84F8AC32FFF7DB
:1095780042B900BF80750020EC5F00205C3403080E
:10958800B85900201C5B0020283A00203D3A0020F2
:109598005655555500240020D24AD34B92F80BE07B
:1095A8003068D4F81C211B88D049801A4FF47A728D
:1095B800DFB202FB0EF21B0A8F770F7590424FF055
:1095C8000007CB774B758F700F7180F0F083C84B15
:1095D800DFF840E31B68C74AC74817680068926805
:1095E800C4F818B18EFB038CDB17C3EB6C13DFF8E0
:1095F80028C38EFB008E8CFB07988CFB029CD2172D
:10960800C2EBAC0203F5FA734FEAE07C9BB2CCEBF9
:109618006E1CFF1700F5EA4EC7EBA8070EF1300ED7
:109628008B761B0A0CF1780C4FEA2E2E3030CB7655
:109638004FEA272813120F7781F81D8081F8202020
:1096480081F8213081F824C081F823E081F82200D4
:10965800FFF719B8DFF8C492D9F80000F7F754FEFD
:1096680000283FF4A5A8D9F800000121F7F748FE23
:109678000222002387F8742088F80030FFF798B892
:1096880094F8341194F83531D8F800004A1C0133A5
:1096980084F8342184F83531F7F746FEFFF75BB8D4
:1096A800964CDFF87C924FF0000A0AE01B2B00F082
:1096B80005830D2B00F018824FF0010389F8013063
:1096C8003868F7F72DFE002838D03868F7F720FEFD
:1096D80083B27E2B32682AD099F801100029EFD185
:1096E80094F83621002AE1D07D2B00F0128294F8FC
:1096F80044E1BEF1000F04D080F02003DBB284F80F
:109708004411511CC9B22244092984F8361182F83F
:10971800383100F0F2810829D2D8B4F84221134434
:1097280003EB132303F0FF03A4F84231C8E784F8DE
:1097380036A184F837A189F801A0C1E794F845312A
:1097480033B194F8393184F84501302B00F05A8749
:1097580094F837216A4BDFF8CCC1DFF8CCE1DFF8A9
:10976800CCA10127104600283FF405A83268A2EBD7
:109778000802012A00F2B38194F84691B9F1000F6A
:1097880040F0B38294F8471133F8112012B984F8E5
:109798004771E8E70131B2F5826F84F8471100F0AC
:1097A80021811FD9B2F5E26F00F0C28035D9B2F538
:1097B800046F00F0CC80B2F5116F00F0D580B2F5DF
:1097C800E46FD0D110464F4A176C918A642303FB8B
:1097D80007F393FBF1F119F061FD002384F83731A9
:1097E800FEF7C9BFB2F5007F00F0D8802DD8B2F5DA
:1097F800807F00F04A81B2F5887FB4D1DCF8002080
:109808005207B0D53C4B4FF48870196819F046FDE3
:10981800002384F83731FEF7AEBFB2F5C06F00F011
:10982800D180B2F5E06F9ED1364A906B918A64235D
:1098380003FB00F34FF4E06093FBF1F119F02EFD08
:10984800002384F83731FEF796BFB2F5047F00F0A5
:109858002C81B2F5806F86D194F848310133DBB2A0
:10986800032B00F25D8142F2107184F8483101FB4C
:1098780003F1254B1B88002B40F050810131234B0D
:109888001B78DF07224B1B8848BF0431D80748BF25
:109898000A319A0748BF14311F0648BF2831D80536
:1098A80048BF28315A0748BF64311F0748BFC8312D
:1098B800980548BF01F5C8719A0648BF01F57A7145
:1098C800DF0648BF01F5FA61580648BF01F57A611D
:1098D8004FF4806019F0E2FC002384F83731FEF77A
:1098E8004ABF00BF4862002040620020B45D0020EB
:1098F8001C780020205B0020EC590020F823002071
:109908005C340308B448002038780020EC5F00205D
:10991800B85900201F85EB5167666666EC38002051
:109928001C000020347800200078002056620020B7
:1099380010467E4AD76B918A642303FB07F393FB97
:10994800F1F119F0ABFC84F83791FEF714BF784BAE
:10995800B3F9041001EB81011046490019F09EFC8F
:1099680084F83791FEF707BF9EF80520002A3FF4D8
:10997800FAAE9AF8001000293FF4F5AE6D4B1B883B
:1099880003EB83035B004FF4116093FBF1F119F0D3
:1099980085FC002384F83731FEF7EDBE9EF80610EB
:1099A80000293FF4E0AE644B64491B68104681FB14
:1099B8000321DB17C3EBA10119F070FC84F8379180
:1099C800FEF7D9BE9EF80620002A3FF4CCAE5A4BCB
:1099D8004FF4C060996819F061FC002384F83731AE
:1099E800FEF7C9BEDCF8002012F020097FF4BBAEF8
:1099F800534A1168090600F1EF85524A127B002A82
:109A08003FF4B1AE94F84911032900F26886DFE803
:109A180001F0322819024C4B1B6859799A79DB7985
:109A280001F1407101EB022101EB0341002384F8AD
:109A380049314FF4826019F031FC002384F8373142
:109A4800FEF799BE414B1A68137A507992781B0435
:109A580003EB002313444A1C84F8492103EB0161FA
:109A6800E7E73A4B1A68D379107952781B0403EB6D
:109A780000231344EFE7354B1A689379D0781278AE
:109A88001B0403EB00231344E5E7DCF8002051072F
:109A98007FF569AE2E4B4FF48070196819F0FEFB04
:109AA800002384F83731FEF766BE9EF80520002AA9
:109AB8003FF459AE9AF8001000293FF454AE214BF8
:109AC8005B7B002B00F0B0851A4B1B8893FBF1F1F0
:109AD80001EB810149004FF4047019F0DFFB00230A
:109AE80084F83731FEF747BE4FF0010184F836118C
:109AF80084F83831A4F84221E2E5B4F84221C2F1F1
:109B0800FF0293427FF4D8AD4FF0010384F845314A
:109B1800D2E54FF0010384F84431D1E50231AEE6D5
:109B2800012384F8483142F21071A2E6B4480020BB
:109B3800BC59002040620020205B002067666666F2
:109B4800CC4D002048620020B8780020DC59002065
:109B58001C7800203B685E2098473B6802209847A5
:109B6800FF201DF0C1FE0378FF2B00F0328590F92D
:109B780001304FEAE3785FFA88F8D8B219F030FC80
:109B8800404619F02DFC3B685E2098473B6803204F
:109B98009847FF201DF0A8FE0378FF2B00F01485DE
:109BA800B0F90830D8B2C3F30729DFF8B88219F042
:109BB80017FC484619F014FC98F80530002B40F0C3
:109BC800D7820AA99E4819F0D1FB3B685E209847C6
:109BD8003B6813209847BDF928805FFA88F019F090
:109BE800FFFBC8F3072019F0FBFB3B685E20984792
:109BF8003B681B209847BDF92A805FFA88F019F066
:109C0800EFFBC8F3072019F0EBFB3B685E20984791
:109C18003B68232098474E2019F0E2FB002019F0FA
:109C2800DFFB0AA9864819F0A1FB3B685E2098472C
:109C38003B6812209847BDF928805FFA88F019F030
:109C4800CFFBC8F3072019F0CBFB3B685E20984791
:109C58003B681A209847BDF92A805FFA88F019F006
:109C6800BFFBC8F3072019F0BBFB3B685E20984791
:109C78003B6822209847452019F0B2FB002019F0D4
:109C8800AFFB3B685E20984794F81431FEF7EBBCB5
:109C9800FCF78EFC6B4B1B68C01A40F6B833984231
:109CA80000F28681DFF8C0A19AF804303A2B00F060
:109CB800B183002388F80030FEF77ABD3868F7F7DB
:109CC8002FFB00287FF4F8AC4FF0010384F83731FC
:109CD800F6E4C4F8283184F82031DFF8908119F0CF
:109CE8002BFB94F82C31FEF71BBD5749062019F0C1
:109CF800F7F8002384F8460184F83731FEF73BBDB6
:109D08004FF000083B68D6F8009084F814815E2074
:109D180098473B684D4C17209847404619F060FB20
:109D28004B4BA3FB09239B0BA4FB03125209C2EB69
:109D38000212A3EB8203D8B219F052FB3B685E20F3
:109D480098473B6818209847424BA3FB09239B0977
:109D5800A4FB03125209C2EB0212A3EB8203D8B28E
:109D680019F03EFB404619F03BFB3B685E209847E4
:109D7800FEF77CBC0AF1FF3A84F867A1FFF7B5BB90
:109D88000CF1FF3C84F866C1FFF76FB9013B84F81A
:109D98005F31FFF793B8013B84F85E31FEF76DBF82
:109DA8002D493A2019F09CF82870FEF718BD2B4B66
:109DB80032681B78C4F81C21013B012B3FF607AC25
:109DC800102202238A700B7101E43B68DFF8A0902F
:109DD8005E2098473B6810209847214AD9F8003000
:109DE80082FB032ADB17C3EB6A1A5FFA8AF019F0C1
:109DF800F7FACAF3072019F0F3FA3B685E20984790
:109E08003B6821209847D9F80030154AD81782FBBB
:109E18000329C0EB6910642202FB10300028B8BF88
:109E28004042C0B219F0DCFA404619F0D9FAFEF700
:109E3800A6BD19F071FA01233B70FEF742BC00BFC2
:109E480080969800643800209D32020889888888A6
:109E580073B2E745D34D62108D340208287800208C
:109E68001F85EB51007800204C380020E85C00206A
:109E78001C780020AA4B1B88DA0515D4D80600F1F7
:109E88001B84990600F127845A0600F133841807C9
:109E980000F13D84D90700F1FA8413F0020F0CBFDA
:109EA8004FF004084FF00C089E4B9F4A1B78D2785D
:109EB80003F001030AB143F002035320029319F09F
:109EC800B5F99A4A128802EB820202EB82029000EC
:109ED80080B219F091F9002019F08EF9944A954949
:109EE80012883868C2EBC212520081FB0231114459
:109EF8004FEAE27ACAEB612A5FFA8AFA5146F7F723
:109F080013FA8D4B38681A78029B48EA03088A4B83
:109F18008AEA020A002183F800A0F7F705FA414609
:109F28003868F7F701FA844B834A1B78386888EA5F
:109F38000303DBB219461370F7F7F6F994F85031BA
:109F4800002B7EF478AD4F2019F070F91AF076F8EE
:109F58001AF074F81AF072F801213868F7F7E4F982
:109F6800764A754B92F800801B78734A386808F077
:109F7800010883F0010341461370F7F7D5F96E4BDA
:109F88006D4A1B78386888EA030319461370F7F797
:109F9800CBF994F85031FEF74EBD694B9FED697AC5
:109FA800D3ED007AF8EEE77A67EE877AFFF76EB8B6
:109FB800654AB2F8523100210133A2F8523188F8CB
:109FC8000010FEF7F5BB614E614B00930024A6F12B
:109FD8003F01604B604A089106F8404C5F4909967A
:109FE8000AA8F8F7C1FF089E731C08933470089BF1
:109FF8002922591C08911A70089BEA22591C0891B9
:10A008001A70089BC822591C08910AA81A7025F0D2
:10A0180077FC471C0AA93A46089826F099FB089A43
:10A02800D31901330893D455089B5A1C08921C7005
:10A03800089B5A1C08921C70089B5A1C08921C709A
:10A04800089B5A1C08921C70089B5A1C08921C708A
:10A05800089B5A1C08921C70089B5A1C08921C707A
:10A06800089B5A1C08921C70089B5A1C08921C706A
:10A07800089B5A1C08921C70089B5A1C08921C705A
:10A08800089BFF22591C08911A70089B01229918F5
:10A0980012A808911A7050F8283D9B1B337019F0CC
:10A0A800C1F92C70FEF79BBB884689460846049187
:10A0B80005918E4606910391FEF712BE284A234B5E
:10A0C80012680B93A3F1400500202121D70003F863
:10A0D800400CA97040F1CD8222490326104B1B8801
:10A0E800580500F1C382DA0700F1F28203F0020397
:10A0F8001D4A002B1CBF032611461C4F324638460A
:10A1080026F026FBF31912A80133B91E40F8203DAA
:10A1180000225B1AF2556B7019F084F9FEF71CBC2B
:10A12800B8590020EC5F0020184900204062002048
:10A13800167800200308208070600020FC7700203B
:10A148001C7800200AD7233CF8230020345D002027
:10A15800E5590020A45F0308AC5F0308B85F030853
:10A168002C780020905F0308A05F0308F75C0020AC
:10A178009E4B93F800A0BAF1000F3FF422AD9C4A21
:10A18800B4F816E111883B6802924FEA0E1E64206B
:10A198001FFA8EFE00FB01A14FEA4A00B1FBF0F165
:10A1A8004EEA012E1FFA8EFEC1F303215E204EEA0D
:10A1B800010998473B68062098475FFA89F019F02B
:10A1C8000FF94FEA192019F00BF9B4F81631029A71
:10A1D8008849B2F800904A7A01339BB2012A93FB6E
:10A1E800FAF00AFB1033A4F8163100F041836E230D
:10A1F80081484A7B03FB09F380FB03014FEAE379BB
:10A20800C9EBA1092AB1794B1FFA89F91B7899FB87
:10A21800F3F93B68DFF8F8A15E2098471FFA89F93F
:10A228003B683A209847AAFB093A4FEA5A1A1FFA9C
:10A238008AF3D8B2029319F0D3F8029B180A19F0DE
:10A24800CFF83B685E2098473B683B2098476423DB
:10A2580003FB1A939BB26948053380FB0320DB1785
:10A26800C3EBA000C0B219F0BBF8002019F0B8F891
:10A278003B68DFF890A1DFF884915E2098473B683F
:10A2880028209847DAF8003089FB0329DB17C3EB4D
:10A29800A9095FFA89F019F0A3F8C9F3072019F0A2
:10A2A8009FF83B685E2098473B6804209847B8F8B9
:10A2B8000830002B40F02282DAF8083083F31008C7
:10A2C8005FFA88F019F08CF8C8F3072019F088F8BD
:10A2D80077E4C4F824B187F80090FEF7F2B9484A49
:10A2E800434B0B9212AEA2F13D0046F8200D19889F
:10A2F800444FA2F1400300204FF00A0E02F8400C30
:10A30800082283F801E030469A70F8F72FFD3B6881
:10A318003A49DA1781FB0313C2EBA30399B230461B
:10A32800F8F724FD06F042FFBF680A9B3A0C591C57
:10A338000A911A700A9B3A0A591C0A911A700A9BC8
:10A348005A1C0A921F700A9B5A1C0A9218703046AF
:10A3580019F068F8FEF7FDBA2B4F9FED2C8AB7F974
:10A36800022027480B9007EE902AF8EEE77A12AE03
:10A3780067EE887AA0F13D01FDEEE77A46F8201DE8
:10A3880000F8403C0823CDED027A00F83F3C1E233C
:10A39800BDF8081000F83E3C3046F8F7E7FCB7F97E
:10A3A800003007EE903AF8EEE77A304667EE887AA2
:10A3B800FDEEE77ACDED027ABDF80810F8F7D6FC85
:10A3C800B7F9043007EE903AF8EEE77A304667EED0
:10A3D800887AFDEEE77ACDED027ABDF80810F8F735
:10A3E800C5FC304619F01EF8FEF7B0BA56620020D8
:10A3F8004062002048620020310CC3306766666600
:10A40800345D0020205B0020BC59002058A08B41FF
:10A418001F85EB519AF80240C4B1013CE4B2013403
:10A4280054445146002211F8013B534083EA031378
:10A43800DBB2120ADF0042EA03228C4287EA1313D6
:10A4480082EA0302EFD1002A7FF433ACB24AB34F59
:10A45800B34B1288B349B44CFA61DFF8F8921A6822
:10A4680009689B68FA62B4F85221F866FB64D9F867
:10A478000000F963FA65F5F73FFF029000287EF4C3
:10A4880092A90221D9F80000F6F73AFF94F854315E
:10A498009AF803200392642B4FF0040287F8742083
:10A4A80040F05C8194F85531072B04BF9DF80830C3
:10A4B80084F8553194F85531069307EB031ADAF806
:10A4C80004100291084625F01BFADAF808100591E5
:10A4D8005FFA80FA084625F013FAC0B204900AEB36
:10A4E8000002069B9148029902900832C27123F03B
:10A4F8000F0286468272049803F00F0300EBCA002D
:10A508008EF80D3052468EF80E000EF10F0026F030
:10A518001FF9874B049A05990AF10900184426F097
:10A5280017F90298C37903F1010ACBB1013B5FFA2D
:10A5380083FC0CF1080CDFF820E284440023073088
:10A5480010F8011B59408B00CA0883EA410302F046
:10A5580018024B404EFA02F253408445DBB2EFD169
:10A56800734A03980AF8023019F03CFD94F8553103
:10A578000022013384F8553184F85421029BDDF818
:10A5880008A09B785BB11AF80510D9F80000F6F717
:10A59800CBFE01359AF80230EDB2AB42F3D894F80D
:10A5A80054310322013384F8543187F8742088F831
:10A5B8000020FFF751B80221D8F80000F6F7A0FEF6
:10A5C80094F82C31FEF7ACB84FF000094846FFF775
:10A5D800ECBA4046FFF7D2BA1023042218460AA95B
:10A5E8008DF82A908DF82B908DF82C908DF82D9061
:10A5F8008DF828308DF8292018F030FE84F837912E
:10A60800FEF7B9B84B49881F18F00EFD84F84601CB
:10A61800FFF79EB8484AD278002A0CBF4FF0040CC6
:10A628004FF0050CFEF746BE3B4B1988FFF750BAB2
:10A638000123D8F800003B70F6F76AFE0746D8F801
:10A648000000F6F765FE7F067EF43BA88E287EF4B0
:10A6580038A894F82031002B7EF450A8374BC4F862
:10A6680028312D2384F82C31FEF732B803263449DB
:10A6780043E5344B344A1B68344903F4800383426E
:10A6880016BF11460426032628E523499A790B8824
:10A6980003EB830303EB83034FEA83081FFA88F86D
:10A6A800002A00F003811E4B1B680FFA83FA06F09C
:10A6B8007DFD40B2FEF71CBA4FF03408FFF7F4BB3B
:10A6C800984699461846049305930393FEF708BBEA
:10A6D8001F49042611E54FF02408FFF7E5BB4B1C82
:10A6E800DBB2042B84F849314FEA01617FF4A1A958
:10A6F800FFF79CB94FF01008FFF7D6BB06F056FDE0
:10A7080018F06EFE002018F06BFEFFF75ABA4FF0F3
:10A718002008FFF7C9BB00BF406200201C000020D2
:10A72800205B00201C780020F8230020505E0020C9
:10A73800565E00203825002018490020B45D00200E
:10A74800945F0308CC4D0020905F0308885F0308DE
:10A75800985F0308EC3800200007090E97F875A0E9
:10A76800654904951AF00F0F04BF0AF1010A5FFA50
:10A778008AFABAF1070F28BF4FF0010A4FEA0A1CFC
:10A7880007EB0C03187C5D4B02930A18002392F820
:10A7980024105A4A93725FFA8CF31A46584B96461D
:10A7A80007EB0C024EEA000001291870D26803F189
:10A7B80001000CD90239C9B28D1C1D44034603F8A7
:10A7C800012BAB424FEA1222F9D101310844BC44B3
:10A7D80022F060030AF1010A9CF811205FFA8AFA54
:10A7E8001343BAF1080F037000F101035AD04FEA7E
:10A7F8000A1C07EB0C01424A087C3F4901449A1A9B
:10A8080091F8241055180EF1100E132D5FFA8EFED4
:10A81800C6DD049D0298DFF8F4E0D1B28B1DDBB2EF
:10A8280043F04002C27103F1010CCBB14B1DDBB206
:10A838000833C31804930EF10100002310F8011B1C
:10A8480059408B0083EA4103CA084B402D4902F066
:10A85800180241FA02F25340049A8242DBB2EDD167
:10A8680003980CF80E3087F875A019F0BBFB85E645
:10A878003B685E2098473B68392098475FFA89F023
:10A8880018F0AEFD4FEA192018F0AAFDF0E44FF0D9
:10A898000808FFF709BB1C4B9046B3F900A06420D9
:10A8A800FEF726B9164A049D9A1AB3E74FF0FF330C
:10A8B800FBE698469946184604930393FEF710BAA8
:10A8C800984699461846049305939E460393FEF7C7
:10A8D80007BA0393FEF704BA98460393FEF700BA43
:10A8E800984699460393FEF7FBB998469946184649
:10A8F8000393FEF7F5B900BF5C340308505E0020EF
:10A908005D5E00200007090E205B0020565E0020D7
:10A918002DE9F04F724B734A1C7893B000F59C41B7
:10A928002031814607911160002C00F00D856E4A98
:10A938001268904240F22E826C4A6D491768DFF81F
:10A94800E8B10492013C1C706A4C039107F48057EB
:10A95800002F40F02C82039B5B7D002B40F0C084CD
:10A96800049B1B681D0400F11A87634B9945A37863
:10A9780000F29D83002B40F09D83604B0593049B60
:10A988001F6817F4805940F05584039BBBF9066093
:10A998005B8B9E42B4BF00260126594B1B6813F0FF
:10A9A800805300F00E82059A127812F0010200F02E
:10A9B8000F8203985349408C91ED037A07EE900A71
:10A9C800F8EEE77AB4EEE77AF1EE10FA80F2E18772
:10A9D800002E40F004824C4D95F8A010002940F05C
:10A9E800FE814A494A480D6895F82D5000210160BA
:10A9F800416081604749002D40F0F2810D70002AC6
:10AA080040F0F381444B1A78002A50D10399BBF9DE
:10AA180000E04F8B898BBBF90200BE45CCBF802577
:10AA2800002545F040038E45A8BF2B469B0843F000
:10AA38008005B842C8BF2B4643F040058842A8BFEE
:10AA48001D46BBF904E0BBF90600AD0845F08003DC
:10AA5800BE45C8BF1D4645F040038E45A8BF2B46DE
:10AA68009B0843F0800E284DB842C8BF734643F098
:10AA7800400E95F8A2708842B8BF73469F4201F015
:10AA88002181A5F8A42085F8A620244985F8A230BC
:10AA98000F78002F01F06D805F2B01F0F8806F2B8D
:10AAA80000F0CF87059B1B78DB0740F19187049B5B
:10AAB8001B4A1B68069203F00403002B40F0FB843A
:10AAC8000DF14008174D0023C8F8043005F150096E
:10AAD800109340F6330A192740F2833629E000BF65
:10AAE8009C380020E436002098380020CC4D002007
:10AAF8005C4F002018490020404B4C00EC5F0020C0
:10AB08002C78002058620020C4260020DC59002040
:10AB18003C730020202900208C400020992100202F
:10AB28003478002084750020C85F002004354D4526
:10AB380020D0AA78EB789A4217FB0261F6D26A789D
:10AB4800043217FB03633BF912205245A8BF524653
:10AB5800B2F5617FB8BF4FF461728A42E6DD9A426E
:10AB6800E4DC29782429E1D840460435F8F784FB49
:10AB78004D45DED1B34B98E803001F78B24B83E80C
:10AB88000300002F00F022840121AF48F8F784FB6E
:10AB9800002840F0A681E378002B40F0A281AB4C5E
:10ABA80023881DB225F00105AEB2B342268000F01D
:10ABB8008986A74D02270E204FF014094FF0FF0891
:10ABC8002F7085F8019085F802801FF0F5FF39464F
:10ABD8009D482688F8F760FB002841F0258026F07C
:10ABE80002039BB2B34223800AD0994B1421FF225F
:10ABF80002250E201D7059709A701FF0DDFF2688FF
:10AC0800944BDFF89CA21978DAF804000393B5078F
:10AC180008BF81F00201C1F34001F7F795FB242139
:10AC28008948F8F739FB30B9059A1378590744BFB2
:10AC380023F004031370069B1B6813F00A0F24D03B
:10AC480005218148F8F728FB002800F06F86258841
:10AC58006B0740F169877C480621F8F71DFB00283F
:10AC680000F051866F0640F17C8707217648F8F797
:10AC780013FB50B1784B794AB3F90430784982FB19
:10AC88000302DB17C3EBA2030B800C216E48F8F715
:10AC980003FB2288002800F0408142F480739A4226
:10ACA800238009D06A4B02251421FF220E201D7033
:10ACB80059709A701FF080FF6A4B1B78082B00F0C0
:10ACC80038810E2B00F03581049B1B685E0544D546
:10ACD800654B1B79002B00F0E98014215A48F8F7DE
:10ACE800DBFA002840F0E78018F00CFC01201FF088
:10ACF800ABFE90B3DFF8AC8100254FF0CC0902E041
:10AD0800DDB2022D29D809FB05F76B1C58F807603E
:10AD1800002EF5D1C378554A90F9020052F8233035
:10AD2800019603220092012132461FF015FB0346CB
:10AD380005EB450000EB0010049353B1314608EBD6
:10AD48008000CC2228F019F8049B48F80730013518
:10AD5800EDB21EF081FD0028D3D1059B1B78DD07DD
:10AD680040F1FA804249434A01230B701370039B58
:10AD7800DAF80000197801F00101F7F7E5FA069B07
:10AD88001D686A0700F15881EB0600F1728113B063
:10AD9800BDE8F08F384B394A1F68049307F4805791
:10ADA8000392DFF804B1364C002F3FF4D4AD0021F4
:10ADB8002548F8F771FA00287FF4CDAD1BF08EFB1B
:10ADC800C9E578023FF5EFAD059A127802F0010265
:10ADD8002C4D002185F8A010002E3FF402AE2A4920
:10ADE80001200870002A3FF40DAEF9067FF50AAE7F
:10ADF800264A1278D2063FF505AEB9F1000F7FF466
:10AE080001AE002B7FF4FEAD7D023FF5FBAD204B7C
:10AE18001B78002B01F042831E4B9B78002E41F0DB
:10AE28004D833BB11C4A1D4B12681B689B1A002BB3
:10AE3800C1F2E9831020134D1FF0BEFE012385F8EF
:10AE4800A130DFE58A4800202C780020B85900207E
:10AE58008C350020C0600020BC59002067666666FB
:10AE6800683200208075002048620020A45503083D
:10AE7800ED5F002094320020CC4D00205C4F002074
:10AE880018490020C426002020290020FC77002033
:10AE980099210020DC780020F8600020086100205B
:10AEA800C460002010460020C85F0020059B1B7866
:10AEB800D8077FF519AF3C2018F0FCFE00283FF4B6
:10AEC8004CAF07F029FB3C2018F0A7FE00283FF400
:10AED80044AF07F021FB3C2018F09FFE0028F0D17A
:10AEE8003BE7069B1B689A077FF559AEAC4C268852
:10AEF800F3073FF574AE46F001039E4223803FF40A
:10AF08006EAEA84B1421FF2202250E201D70597029
:10AF18009A701FF051FE268861E622F480739BB276
:10AF28009A4223807FF4BEAE9F4B1B78082B7FF498
:10AF3800C8AE228822F040039BB29A4223803FF495
:10AF4800C3AE984B02251421FF220E201D705970A4
:10AF58009A701FF031FEB7E6944B93F80090B9F160
:10AF6800000F5FD1DFF89082914F18F8030C3E78FC
:10AF78004146A8F1030523F0ABFC002800F0B88394
:10AF8800002E40F00A8405F10801687923F0A0FC3E
:10AF9800002841F095818749A87A23F099FC002878
:10AFA80000F0B983022E41F08F818349E87B23F0BA
:10AFB8008FFC002841F08C818049287D23F088FC93
:10AFC800002800F0B983042E41F086817C49687E10
:10AFD80023F07EFC002841F083817A49A87F23F082
:10AFE80077FC002800F0B983062E41F04C817649A1
:10AFF80095F8230023F06CFC002840F0158773496E
:10B0080095F8280023F064FC002800F0B983082E86
:10B0180040F0F4866E4995F82D0023F059FC00287D
:10B0280040F0B9836B4B01221A7023F0D4FE069BC3
:10B038001D686A077FF5A8AE032023F073FC00287B
:10B0480000F05886238813F008067FF49DAE082088
:10B058001FF0C2FE6048614B006818606049614A91
:10B06800069D614BBBF806002D68088016601E60BF
:10B078008AE6162023F056FC002800F01D86238857
:10B0880013F400747FF483AE4FF400701FF0A4FE35
:10B098005148534D5149534A534BBBF80660006819
:10B0A8002E80086014601C6013B0BDE8F08F0BB9E7
:10B0B8000123A3704D4B05931B201F7894F8216042
:10B0C80023F030FC012E07F00109824600F0DB85F1
:10B0D80007F00203069394F82030DFF82081444DEE
:10B0E800052B00F29A80DFE813F08B004F00060072
:10B0F800D800F900BD00012E04BF052384F82030D4
:10B10800B9F1000F00F00D81039B3A4FB3F9181005
:10B11800B8F80030002261F30F0263F31F420023E6
:10B1280061F30F0361F31F43CBF8042039686269A8
:10B13800CBF80030914200F21384012E41F0DC81FB
:10B14800032294F820300692CAE723F017FC01285E
:10B1580007D1284FB8F802303A68642101FB03236D
:10B168002361BAF1000F04D098F80630002B40F0A4
:10B178008C80012E51D01F4F22693B689A42C0F043
:10B18800F485012384F82030012E6BD098F807301D
:10B19800012B00F0CF800CF0A1FA94F820309FE743
:10B1A800B85900208C35002080750020ED5F002004
:10B1B8009200002090340020953400209A3400201A
:10B1C8009F340020A4340020A9340020AE3400208D
:10B1D800B3340020943200201C78002080320020F4
:10B1E800743200207832002070320020EC5F00209A
:10B1F80038780020F860002086340020843500204C
:10B20800B9F1000FA1D14FF48060BAF1000F00F03E
:10B2180077831FF0E1FD00232361069B002B3FF499
:10B22800AEAB06981FF0C8FC049B1F6817F4805942
:10B238003FF4ABAB1D21B248F8F72EF800287FF495
:10B24800A4ABB04A039BD2881B8BBBF90660991A42
:10B258008E4240F3948513449E42B4BF00260126D3
:10B26800FFF79BBBA84F3A68B8F80230642101FB8E
:10B2780003234FF480600022236184F82020E270C9
:10B288001FF092FD94F820302AE70CF027FA0322E9
:10B298004FF47A7384F82020E3619B4F2B8843F0A6
:10B2A80002032B801BF01AF93A68E369134404225D
:10B2B800A36184F82020012E40F051853B68A269E3
:10B2C8009A42AAD2914B187818B923F02BFB002880
:10B2D800A3D12B8823F002032B80C4E78A4FEAE727
:10B2E800039A013BD27D3BF91330002A40F03383A7
:10B2F800A3F57A73B3F57A7FA8BF4FF47A7323EA7C
:10B30800E37307EE903A9FED827AF8EEE77A67EEFC
:10B31800877A804AFCEEE77A17EE903A1380FFF7B7
:10B3280024BB794F3B6847F230520323E26184F82B
:10B338002030B3E70CF0D2F9032240F6B83384F892
:10B348002020E361704FA9E7734F3B78002B00F092
:10B358004F87724BDFF8D881DFF8D8B1DFF8D8A172
:10B36800039345465E46049099460EE019F804108A
:10B378009847032C28DC88B93B782AF8020F013457
:10B388009C4205F1040580F2DD80072CE1B23046CD
:10B39800DBF80430EADD984700B2EDE738F82420FE
:10B3A8006B88801A4FF47A719B1A01FB00F040F603
:10B3B800CA0290FBF3F00844904240F2EE23A8BF83
:10B3C80010469842B8BF184600B2D5E7DFF86CA11E
:10B3D800DFF86C81524D0AF15A064FF001095146C7
:10B3E8001AF8010C23F074FAF8B19AF804009AF8E4
:10B3F80002309AF803E000EB400105EB8101013BC4
:10B40800D1F8B42003EB4303434493420DD095F89D
:10B41800E02081F8B0E009FA00F022EA0000C1F863
:10B42800B430C1F8B87085F8E0000AF1060AB245F0
:10B43800D5D13C49344A3C4B3C4D09681B78D2F87D
:10B44800009008910793A5F1B00A00266B685BB3DA
:10B458001F784FB3AA68A9EB0202002A0ADB9AF800
:10B46800E0200121B14022EA010209F5FA718AF8C7
:10B47800E020A960079ABAB12A7859780432D2B282
:10B48800002940F08C8203993BF91220098B01F1C5
:10B49800C800824240F335849AF8E0109A7841FA5D
:10B4A80006F3D80740F1A5840136042E05F10C05F2
:10B4B800CCD1FFF769BB1A4D95F8AA3053B1059B5B
:10B4C8001B78DE0706D5039BBBF906205B8B9A42E7
:10B4D80000F3658411210A48F7F7DEFE002800F022
:10B4E800468295F8AE302BB995F8A83013B93223B7
:10B4F800A5F8AC30012385F8AE30FFF7E1BA00BFFC
:10B508002C78002068350020F86000209921002060
:10B51800AAF1823F16780020F03800205C4F002006
:10B52800C4260020B87800208D59002074270020F8
:10B538000839002068490020C22600209D330020D9
:10B54800B0340308DDF81090C44A04921146C44A86
:10B558000968A2FB092A42F201020A404FEA9A1A34
:10B56800059200F00082BF4DBF48C04CC04A95F814
:10B5780000E0007884F800E01070BEF1000F04D0FD
:10B58800BB4A92F800E08EF0010EBA4D0F2085F804
:10B598002400002B00F0FA82B74B039E0C931B7813
:10B5A800B6F826C00B931C463B78B78C039EB34A6B
:10B5B800368B0E962646A2FB0442520802EB420244
:10B5C800B21AD2B2CDF824C001F48051089295F88D
:10B5D8002580DFF8C0B2DFF8E8C20A900AF5967253
:10B5E80076460F9105F1280400200692CDF8349094
:10B5F800AE46002E00F03A823EF910201FFA82F97A
:10B60800B9454FEA400103D3099DA94540F272822A
:10B618005CF82020924580F032823BF90120059D9C
:10B62800002D40F04682013098422BF8012004F1A9
:10B638000604DEDB0A98924ADDF834908EF82580FD
:10B648000F280CBF012100218EF82400117000F092
:10B65800A4828C4C8C4E8D4F35883868A1686268FE
:10B66800E06045F00405401A90427F4F3580804DD8
:10B678004FF0010188BF00223970297088BF84F813
:10B688002120002B00F09B82049A03991768804EB2
:10B69800B1F824C0B1F818E07E4817F48057354651
:10B6A80040F0D38239460EE06A7802EB820202EB60
:10B6B800820202F2EE2292B20131994220F8022B64
:10B6C80005F102050ED016F81120002A00F01682A6
:10B6D800022AE9D00131028820F8022B994205F1AB
:10B6E8000205F0D10C9A137801331370FFF730B9C3
:10B6F80008F10501687923F0EBF800283FF44BAC1A
:10B70800012E40F0DD8505F10D01A87A23F0E0F85F
:10B71800002840F0D9856049E87B23F0D9F8002853
:10B728003FF44AAC032E40F0D3855C49287D23F0D2
:10B73800CFF8002840F0D0855949687E23F0C8F832
:10B7480000283FF44AAC052E40F0CA855549A87F29
:10B7580023F0BEF8002840F09685534995F8230059
:10B7680023F0B6F800283FF44AAC072E40F05C837B
:10B778004E4995F8280023F0ABF8002840F03E83A6
:10B788004B4995F82D0023F0A3F800283FF44AAC64
:10B79800092E3FF447AC4FF009094B4631E3354DCC
:10B7A800D5F88830A9EB0303002BFFF6DEA8414A41
:10B7B80095F88C30517C079AC5F8882001333E4AA9
:10B7C800039E32F81120B17D03F00F0385F88C3009
:10B7D8002B4492B292FBF1F283F8902095F89010E6
:10B7E80095F8912095F8923095F89C000A4495F8C0
:10B7F8009310134495F89420194495F895300A4409
:10B8080095F89610134495F89720194495F89830B0
:10B818000A4495F89910134495F89A20194495F814
:10B828009B300A44134495F89D1095F89F201844BE
:10B8380095F89E3001440B441A4442F30B12642AD3
:10B84800F17DA8BF642213B209B1C2F1640307EE07
:10B85800903A9FED1A7AF8EEE77A58E5CC4D002039
:10B86800D34D6210C0360020EC0000208D59002016
:10B87800ED000020C42600209D380020ABAAAAAA0B
:10B88800664900201849002038780020F860002018
:10B898003C390020C85F0020953400209A340020ED
:10B8A8009F340020A4340020A9340020AE340020A6
:10B8B800B3340020746000209060002014AE23414F
:10B8C800A03800200221C648F7F7E6FC00283FF41C
:10B8D80086A92580B7073FF593A946F00203B3422E
:10B8E80023803FF48DA9BF4B02201421FF2218703A
:10B8F8000E2059709A701FF05FF92688FFF780B9FB
:10B908001FF052FA87E425F040039BB2AB42238034
:10B918003FF4ABA9B34B02251421FF220E201D7062
:10B9280059709A701FF048F9FFF79FB9238823F0E0
:10B938000405ADB2AB4225803FF48DA9A94B022581
:10B948001421FF220E201D7059709A701FF034F9CF
:10B958002588FFF780B9C3F53B6308331BB2C7E4FA
:10B9680003230693DFE4A04A92F800E005E695F881
:10B97800A830002B3FF4A4A8059B1B7813F0010303
:10B988007FF49EA8012285F8A83085F8A920FFF742
:10B9980097B8964D012185F8A010FFF720BA012924
:10B9A80000F0E0839AF8E0200123B3400136134306
:10B9B800042E8AF8E03005F10C057FF447ADFFF757
:10B9C800E3B8059B8A4A1B781060D80700F1F58117
:10B9D80095F8A61000297FF46AA8B5F9A430322B8F
:10B9E8007FF765A895F8A2200120572A85F8A600B8
:10B9F80000F02E84049B1B6813F0040302D05A2A1B
:10BA080000F039855D2A00F0B1845B2A00F0D38408
:10BA18005E2A00F0DD84562A00F01285972A00F08D
:10BA28001E85A72A40F06A847249049B0A781B681D
:10BA380042F004020A70704A069203F00403FFF70A
:10BA48003CB8B2F5FA7FFFF632A895F8A620002A8E
:10BA58007FF42DA8059B1B78012185F8A610D9072E
:10BA680000F142841AF07CF8FFF721B8002F3FD08C
:10BA78005CF8202092454FEA4001FFF4CEAD5F4AC2
:10BA88005E4D525C05EB0109002A00F09D80022AF8
:10BA980047D199F8012002EB820202EB820202F2FE
:10BAA800EE2292B2032833DD059D12B2002D3FF439
:10BAB800BAAD089D24F81520B8F1000F03D10B9DED
:10BAC800022D7FF6B0AD2288B4F80290B4F8048055
:10BAD8004A4490444A4A0FFA88F882FB0852494D72
:10BAE800A2EBE87225F8018012B24FF001089AE53E
:10BAF8003A464100069D4CF8205090E5CAB2022A09
:10BB080004D9032A7FF4E6AD6246D5E57246D3E54B
:10BB1800012505FA00F90A9D25EA090512B20A95D8
:10BB28007DE53BF80120BDE745F004039D422380F5
:10BB38000AD02C4B02251421FF220E201D705970AB
:10BB48009A701FF039F825882F4B304AB3F9043022
:10BB58002F4982FB0302DB17C3EBA2030B80FFF71D
:10BB68007AB845F04003AB4223807FF4D3AEFFF7A9
:10BB78007CB839461A48F7F78FFB00283FF421AF05
:10BB880085F8A77019F0ECFFFEF78CBF2149224A0F
:10BB98000C91DFF890B0012111701B21104805931A
:10BBA800F7F77AFB059B00287FF453AD1B4C1C4F1D
:10BBB800E2683B68A3609B1AC82B00F23B83049B96
:10BBC8001F6807F480578DE5C2B2022A40F2C88286
:10BBD800032AA6D10E9A0F9D002D08BF3A4661E7A9
:10BBE8002C7800208C3500208D590020C426002098
:10BBF8000C610020FC770020347800203C390020BC
:10BC08005655555534270020BC590020676666668E
:10BC1800543200209D380020664900201849002031
:10BC2800F8600020C85F002026F001039BB2B342F1
:10BC380023803FF44FAE0E202F7085F8019085F8D1
:10BC480002801EF0B9FF268844E600210FE06A78DA
:10BC580002EB820202EB820202F2EE2292B2013180
:10BC6800994220F8022B05F102053FF43BAD16F886
:10BC780011201AB1022AEAD00288F0E7CAB2032AD0
:10BC8800FAD87246EBE700230693FFF724BAB2F519
:10BC9800FA7FFEF60CAF95F8A630002B7EF407AFBE
:10BCA800059B1B7801210B4085F8A61000F0A482A3
:10BCB8001AF014FCFEF7FBBE4FF400701FF074F886
:10BCC800FFF765B8BE4ABF491068B5F9A420C7692F
:10BCD80081FB07018911FF17781A00F5FF407F30B3
:10BCE80082423EF7D2AEC91B0A4412B2A5F8A4207C
:10BCF800FEF7CBBE08201FF057F8069B1D68FFF71C
:10BD080043B8C8398A423DDA9AF8E0109A7841FA7D
:10BD180006F3D9073FF5C8AB5242012009921FF03C
:10BD28002BF87B1E099A162B00F2C280DFE813F06D
:10BD3800B001C6019701EF01DC01030282016D0128
:10BD4800560131011A01C000EF0105010302820109
:10BD58006D01EF00D900C300AE00960080003A687C
:10BD6800E3691344A361FFF758BA0BF0B7FC032249
:10BD780040F6B83384F82020E361FFF78FBA012634
:10BD8800FEF70BBE9AF8E0300122B24023EA020324
:10BD980009F5FA728AF8E030AA60FFF785BB00213E
:10BDA8008948F7F779FA00287FF494AB322385F8AD
:10BDB800AA00A5F8AC30FFF78DBB844B1B78002B8D
:10BDC8003EF475AEE378002B7EF471AE95F8A7309B
:10BDD8000133DBB2032B85F8A7307EF668AE7C4BC7
:10BDE8005B7813B9002E7EF462AE1AF077FBFEF78B
:10BDF80059BE002A0CBF012002208FE74FF0080926
:10BE08004B4603EB83031D4487F80090A9786878B4
:10BE180012F030FA059B6F4A1B7801211170D9077F
:10BE28007FF503A9FEF7A3BF4FF007094B46E8E7E4
:10BE3800DAF8E400DFF8A08190F8361098F80230BC
:10BE480011446429A8BF642121EAE17180F8361001
:10BE5800002B40F08B831CF00FFFA3E5DAF8E40019
:10BE6800DFF8748190F8371098F802301144FE29F1
:10BE7800A8BFFE2121EAE17180F83710002BEAD033
:10BE8800162022F0ADFDDAF8E400E4E70898DFF8C0
:10BE9800488141781144B1F5967FA8BF4FF4967157
:10BEA80021EAE171417098F80230002B40F0588384
:10BEB800DAF8E400CFE7DAF8E400DFF81C818178EB
:10BEC8001144C829A8BFC82121EAE171817098F8F6
:10BED8000230002BBFD0142022F082FDDAF8E400F3
:10BEE800B9E7DAF8E400DFF8F08041781144C829AE
:10BEF800A8BFC82121EAE171417098F80230002BEF
:10BF0800A9D0132022F06CFDDAF8E400A3E7DAF8F0
:10BF1800E400DFF8C48001781144C829A8BFC8210B
:10BF280021EAE171017098F80230002B93D01220B9
:10BF380022F056FDDAF8E4008DE7DFF89C800898D7
:10BF480098F80230417911446429A8BF642121EA94
:10BF5800E1714171002BABD00E2022F041FDDAF8DF
:10BF6800E40078E7DAF8E400DFF86C80017A98F802
:10BF780002301144C829A8BFC82121EAE171017221
:10BF8800002B3FF468AF0B2022F02AFDDAF8E4001A
:10BF980061E7DAF8E400DFF84080C17998F8023008
:10BFA8001144C829A8BFC82121EAE171C171002B39
:10BFB8003FF451AF0A2022F013FDDAF8E4004AE713
:10BFC800385E0020D34D62102C7800208D59002057
:10BFD800DC7800209432002010780020DAF8E400A1
:10BFE800DFF87885817998F802301144C829A8BF0C
:10BFF800C82121EAE1718171002B3FF42CAF09209F
:10C0080022F0EEFCDAF8E40025E7DAF8E400DFF8DD
:10C018004C85417998F802301144C829A8BFC82135
:10C0280021EAE1714171002B40F05382112F7FF416
:10C0380046AF10E7DAF8E400DFF82085017998F8D0
:10C0480002301144C829A8BFC82121EAE171017151
:10C05800002B40F0D082102F7FF447AFFBE6089901
:10C06800DFF8F8840F791744642FA8BF642727EAFC
:10C07800E7770F7122F0CEFC98F80230002B3FF4DE
:10C0880017AF0320394622F0ABFCDAF8E400E2E609
:10C098000898DFF8C88401781144FA29A8BFFA2162
:10C0A80021EAE171017098F80230002B3FF400AFEB
:10C0B800012022F095FCDAF8E400CCE60898DFF8D5
:10C0C8009C84817811446429A8BF642121EAE17124
:10C0D800817098F80230002B3FF4EAAE022022F07B
:10C0E8007FFCDAF8E400B6E60898DFF87084C179D6
:10C0F80098F80230114481F30801C171002B3FF414
:10C10800D7AE052022F06CFCDAF8E400A3E6089B21
:10C11800DFF84884997998F8020011446429A8BF87
:10C12800642121EAE1719971002840F0DA810D2F2C
:10C138007FF405AFBCE6DAF8E400DFF82084C178C4
:10C1480098F802301144C829A8BFC82121EAE17132
:10C15800C170002B40F05F820F2F7FF4DCAE7AE6CF
:10C168000E9A9FE43BF912209978B2F5617F4FF45B
:10C17800966393FBF1F332DB40F633019142A8BF9B
:10C1880011460C2FA1F5617191FBF3F100F0F980D4
:10C19800182F7FF407ACC9B2C8290B46A8BFC8231B
:10C1A800DAF8E400C27DDFB297423FF4FBAB9A1A9B
:10C1B800DFF8A883C77548BF0732D71098F8023050
:10C1C8000137FFB23BB9002F3FF4ECAB38461EF005
:10C1D800D3FDFFF7E7BB182022F002FCF3E70C2F92
:10C1E80000F0E680182F7FF4DDAB00210B46D7E77F
:10C1F800C34A0392FFF7A8B9C249096811F400318C
:10C2080040F0EA800B46C048C65C0F2E03F10C03D1
:10C218003DD001311529F7D1049BBC491B68069113
:10C22800FA3AA5F8A420002203F0040385F8A62012
:10C23800FEF743BCB64A049B1F68138823F0040327
:10C248001380012307F4805784F82130FFF74ABA96
:10C25800AE4AB04B069210461A68AF494FF47A734B
:10C26800B3FBF2F3C3EB431203EB82030268DB0078
:10C278005707A1F8B43000F1A280049B1B6803F0B3
:10C288000403FEF71ABC4FF006094B46B9E5A34E66
:10C29800D6F800E04B00BEF1000F07D05F1800EBA6
:10C2A80087079EF801E07F787745B5D20B449C4F0D
:10C2B8009C4900EB8300002330603B800B60ABE7B8
:10C2C8004FF001094B469CE54FF002094B4698E5B3
:10C2D8004FF003094B4694E54FF004094B4690E5AF
:10C2E8004FF005094B468CE5049B8F491B680A6093
:10C2F800864A069203F00403FEF7DFBB0021BB2A3F
:10C30800109100F09880B72A00F09180BE2A00F0C2
:10C318009580BD2A67D0792A00F05A817A2A00F0E0
:10C3280050819E2A00F047819D2A00F03D81AE2A67
:10C3380000F03381AD2A00F02981EF2A00F0208136
:10C34800FD2A00F01781FB2A00F04F81FE2A00F039
:10C358004681F72A00F067817B2A7EF4A8AB4FF468
:10C36800FA61022021F064FBFEF7A1BB6F4B0022AB
:10C3780001206F4D6F492A700B601EF0FDFCFEF71F
:10C3880096BBCFB26A4B09915B78BB423FF40AABCC
:10C39800DFF8C881384621F025FC98F80230099961
:10C3A8001BB1C9B20C2022F01BFB0137FFB20AE710
:10C3B80000273946E6E7604B01220220D9E7049BB3
:10C3C8005E4A1B680A21118003F00403FEF775BB5F
:10C3D8005B4B02220320CCE75A490978032900F075
:10C3E800868019460FE74FF6FE73574A47489689E5
:10C3F8000690D089334401449381D1810CF06CFAC2
:10C40800F6F790FA0CF050FAF9F7F4FD01201EF057
:10C41800B3FC049BB5F8A4201B68FA3A0021A5F8E0
:10C42800A42003F0040385F8A610FEF746BB0B46CC
:10C438004FF6FE71D9E70B460221D6E70223D4E76F
:10C448000CF04AFAF6F76EFA0CF02EFAF9F7D2FD6C
:10C4580001201EF091FC95F8A220FFF7DFBA049B9B
:10C468003A4A1B684FF4C8711180284A069203F0B3
:10C478000403FEF722BB95F8A820002A40F0DE80CE
:10C4880095F8AA3083F0010385F8AA30002B40F014
:10C49800D0800C201EF090FBFEF709BB002E3EF466
:10C4A800C9AC2B4D95F8A130002B3EF4ABAA1EF079
:10C4B80067FB002385F8A130FEF7A4BA002BF0D063
:10C4C8002449254A09684FF47A7000FB0313136066
:10C4D800E7E71120099222F083FADAF8E400099AD2
:10C4E800A4E50D20099222F07BFA099A1FE61EF0B6
:10C4F80047FBB5F9A4208FE603230693FEF791BE08
:10C508005C4F002090330020B03C030834780020B2
:10C5180038780020BC4D0020384B0020D02800205F
:10C528006A2900206C2900200C610020EC3E0020C4
:10C53800E0590020DC5900203A3F0020D67800203E
:10C54800883F002028780020403A0020D878002032
:10C55800C4260020F8600020086100201078002020
:10C56800152022F03DFADAF8E40074E4172022F0EE
:10C5780037FA9DE40021012021F05AFAFEF797BA14
:10C588000021084621F054FAFEF791BAFF21002055
:10C5980024F090F895F8A220CFE60121002024F09D
:10C5A80089F895F8A220C5E60021FF2024F082F83A
:10C5B80095F8A220BBE6012024F07CF895F8A2208B
:10C5C800B2E6224A137A43F001031372FEF76FBAF8
:10C5D8001E4A137A23F001031372FEF768BA00218A
:10C5E800032021F025FAFEF762BA0021022021F08B
:10C5F8001FFAFEF75CBA1020099222F0F1F9DAF876
:10C60800E400099A27E5124D19F068FF002385F820
:10C61800A130FEF7F7B90F20099222F0E1F9DAF814
:10C62800E400099A98E50021042021F001FAFEF7B8
:10C638003EBA0B201EF0C0FAFEF739BA054A85F853
:10C64800A81085F8A9000692FEF737BA4C490020D1
:10C65800C4260020347800202DE9F0478C4B1B7845
:10C66800DB07074644D58B4B8B4D1C788B4E012C32
:10C6780059D01CD3022C07D189498A4A09881288C3
:10C68800914201D901241C70EB7AE3B12B89D3B113
:10C69800854B1B78BBB104F089FD002800F09B8016
:10C6A8002B7B83422CBF0121002131700CE07C4997
:10C6B8007E4A098810886A7B801A8842E2DAEB7A17
:10C6C8000024002BE2D131782A79632A06D8022C7B
:10C6D800774E00F0BA803378002B5DD1754AAB7A7B
:10C6E8008C4238BF0C461470002B4CD1BDE8F08743
:10C6F8006B4B694D19885B88E878CB1A83EAE3723B
:10C708008142A2EBE3721DD32B788B421AD3614B83
:10C718001C78E01E012861D96749097802294FD0A1
:10C72800012C5E4EA5D15F4A5D491288687B098855
:10C73800121A914239DD5D4A12888A42A4D2002435
:10C748001C70A1E7B1EB400FE1DC524B1C78E11EF5
:10C75800012940F29480022ADEDC57494F4E0878BE
:10C76800DFF84481DFF844C1DFF838E10021032411
:10C77800022834701C7088F80010ACF80010AEF86D
:10C78800001081D11FE0012C71D0022C0BD10720A1
:10C79800BDE8F0471EF010BA7068381A474B984247
:10C7A80058DD72709AE7BDE8F08702241C706BE7C9
:10C7B800022AD2DD4049097802294FF0040464D1E5
:10C7C8003949364E09783E48022ACCBF0022012258
:10C7D800C28081804BE70221317075E7022A9BDC19
:10C7E80095F800C091FBFCFC0CF1010CBCF1080FA2
:10C7F800DFF8B4A0304EA87895F801E096F80080EC
:10C808002A4CDFF8A090254EA8BF4FF0080C8AF8F4
:10C8180000C01FFA8CFA10FB0AF01EFB0AFE80B259
:10C82800DFF88CA02080A9F800E000244FF0640E07
:10C83800B8F1020F34701C70CAF804408AF801E09D
:10C848007FF439AF0FFA8CF1BDE73078A0B9012336
:10C8580077603370C2F164021A4B00FB02F083FB6D
:10C868000023C017A0EBA3506430707036E708208F
:10C87800BDE8F0471EF0A0B97368F81A8EE7032CDC
:10C8880096D10D49097802299AD0044EFCE600BFDA
:10C89800EC5F0020CC29002000780020D22900205D
:10C8A80040620020D029002056620020CE290020B6
:10C8B8006032002028780020546100207F9698007C
:10C8C800586100206BCA5F6B2DE9F04F2DED0C8B82
:10C8D800404B1B7893B0012B039001F0BC803E4C79
:10C8E80094F80021002A41F0C780072B01F0CE8080
:10C8F8004FF0000ADFF8ECB0DBF8043058469847F0
:10C90800002800F06F81BBF8B46000228BF8552036
:10C91800002E40F06687BBF93C50DBF82410BBF9C9
:10C928003E00DBF82820BBF94030691ACBF83010FC
:10C938002A490191821ADBF82C00CBF834200D46E5
:10C948001B1A9BF85610CBF838300BF130000EF05C
:10C9580077F82B68990040F1E980DBED0D5ADBEDA3
:10C968000C7A1F4A94ED416AD4ED426A94ED437AF9
:10C97800D4F810311268B8EEE58ADBED0E5AF8EEFD
:10C98800E77AF8EEE58A013377EE867A38EE268A7A
:10C9980078EE878A9342C4ED417A84ED428AC4EDE9
:10C9A800438AC4F8103101F0F1820A4B1E78142E24
:10C9B80002F0A1840023D4F818510293062D00F246
:10C9C800A880DFE815F0F712E6120B127B121100AF
:10C9D8002114BA1354610020AC270020CC4D00204C
:10C9E800C43A0020384B0020D44B1A78D4F81C7174
:10C9F800DFF8B8E39FEDD27AF8000EEB000383ED81
:10CA0800007A002A7AD0CF49B0EE476AF0EE476A3A
:10CA18000023F1EC017A013367EEA77A05EE903A2C
:10CA2800B4EEE77AF1EE10FAF8EEE55AB8BFB0EED8
:10CA3800677A9A4276EEA76AA7EEA56AE9D1F5EE7B
:10CA4800C06A0EEB0003F1EE10FA83ED007A55DDB3
:10CA5800C6EE265ABC4BBD4A1288F7EE007A75EE30
:10CA6800E75AD3ED007A65EEA77AFDEEE77A17EE7E
:10CA7800903A812B43F317839342A8BF134607EEDE
:10CA8800903AF8EEE77AB24BC11903EB810393EDC4
:10CA9800057AD3ED003A93ED066A93ED014AD3ED9A
:10CAA800046AD3ED034A93ED025AA3EEA77AA4EEE3
:10CAB800276A66EEC76AA7EE646ABDEEC77AE5EE36
:10CAC800276A17EE101A812983ED056AC3ED066AF5
:10CAD80043F3E6828A42A8BF0A4607EE902AF8EE98
:10CAE800E77AFCEEE77ACDED047ABDF810300EEB6C
:10CAF8000002938017B9132E03F0A687152E42F073
:10CB0800BF817044DFF8A882838828F81730D4F8EA
:10CB18001851904B013583FB05235A19EB17C3EBCA
:10CB2800A203C3EBC303ED1AC4F818518A4B1B7850
:10CB3800002B01F0E380894DCDF808A0DFF874825E
:10CB4800DFF86C92DDF804A005F5BC770026844B6D
:10CB5800DBED087A1B78172B01F0258495ED007A18
:10CB6800B8EEC78A082B28EE278A07D1B0EE480A04
:10CB7800019323F0F5FF019B29F81600DAF800204D
:10CB880092000BD5002E04F00981B0EE480ADBF8BC
:10CB9800143207F170009847B0EE408AB0EE480AA8
:10CBA800DBF83431A7F170009847DBF8A431384638
:10CBB80098476B4B1B78032BB0EE408A01F0ED834E
:10CBC800D5F8F800DBF8B830B0EE480A98470136D7
:10CBD800032E07F12407A8EC010A05F10405B6D1D4
:10CBE800DDF808A05E4B1F78072F00F0BA8694F88E
:10CBF80028310493002B40F0C2865A4B5B79002BF6
:10CC080040F0E9850123564A84F828311278072A2A
:10CC180001F0748600230593534B94ED4C9A93EDE1
:10CC2800007A524BD4ED4BCAD3F800A0504B029374
:10CC3800F7EE007A37EEC9CA00252CEE07CA4D4B2D
:10CC4800DFF87491DFF874B1DFED4B8A9FED4BAAE2
:10CC5800DFED3BBADFED4A9A9FED4ABADFED4AAA0B
:10CC6800DFF85C81494F0193B4EEE7CAF1EE10FAA0
:10CC780088BFB0EE67CA2E46454B99ED008A2B4413
:10CC8800D3ED007AF5EE407AF1EE10FA17D0414B69
:10CC98002B44D3ED006A38EE667AB0EEC76AF4EE3C
:10CCA800C67AF1EE10FA08D5B5EEC07AF1EE10FAB0
:10CCB800CCBF37EEA68A36EEE78A83ED008A364B7C
:10CCC8001A8893077ED0022E7CD09AF82E10334B08
:10CCD80007EE901A2B4493ED007A4B42F8EEE76A80
:10CCE80007EE903A26EE877AF8EEE77AB4EEE77A1E
:10CCF800F1EE10FA0AD407EE901AF8EE677AF4EE1D
:10CD0800C77AF1EE10FA88BFF0EE477A244B25492E
:10CD180003EB460331F91600B3F90C30C01A07EEDD
:10CD2800100AB8EEC77AD007E7EE687A40F12F8686
:10CD38001D4B93ED008A27EE888A43E0CA3A00200B
:10CD480000000000AC270020CC3A0020C83A0020A0
:10CD5800003D002093244992C03A0020684B0020EF
:10CD680054610020244B0020BC650020DC590020C1
:10CD7800BC4D002030730020CDCCCC3DAE47813F68
:10CD88000000C84200003443610BB63B3C730020EE
:10CD9800B0650020EC280020B8590020F8280020B1
:10CDA800403A0020BC59002098650020E83C00204B
:10CDB80058610020C04D0020E0280020A464002015
:10CDC80048730020029B94F864212B44D3ED01DAC8
:10CDD80038EE6DDA002A3DD0D34BD4F86821039998
:10CDE8001B688A1A9A4235DD9AF84830022B01F0FE
:10CDF800BC85022E03F05987CC4B1B68990740F17C
:10CE08006487CB4BCB49DFF8A0E331F916C09EED20
:10CE1800008ADFF898E3C7ED00BA03EB460028EE76
:10CE2800288AB0F90C00A0EB0C0007EE900AF8EE87
:10CE3800E77ADEF8000027EE888A904238EE6DDA4D
:10CE4800C1F27980F7EE007AB4EEE79AF1EE10FAC3
:10CE580001F14880B84B2B4493ED000A019B2CEE5E
:10CE6800800A022E20EE0D0AA3EC010A019303F0BA
:10CE78004487B24B9BED007AD3ED007AB04BD7EDE7
:10CE8800006A93ED006AAF4B67EE277A2B4427EED2
:10CE98008C7AD3ED007A67EE277AF0EE665AEDEEDB
:10CEA800275AB1EE467AF4EEC75AF1EE10FA08D4D2
:10CEB800F4EEC65AF1EE10FA8CBFB0EE467AB0EE38
:10CEC800657A94ED4C6AF7EE007AB4EEE76AF1EE13
:10CED80010FAACBF0123002343B1F0EEE66AF0EE8E
:10CEE800C77AF4EEE67AF1EE10FA01D587ED007A0A
:10CEF800022E03F0D386944A944B52F826001B68FE
:10CF0800B0EE6D0A9847924A924B52F826001B6879
:10CF180098479AF8373023B18F4B1B88002B00F0C5
:10CF2800BA85B0EE6B8A8D4B9BED007A38EE400ADD
:10CF38002B4493ED008A83ED000A9AF8483030EECE
:10CF4800480AC0EE077A2BB3854B1B78DB0721D53F
:10CF5800B7EE007AB4EEC79AF1EE10FA04DB94F853
:10CF68006431002B00F06587D4F86831039AD31A2E
:10CF78006D4A12689A420DDD7A4B93ED007AB0EE55
:10CF8800CDDAB4EEC7DAF1EE10FA40F1F0870023FB
:10CF980084F86431744B94F874212B4493ED007A2F
:10CFA8002CEE877A67EE277AC8ED007A32B9019BB2
:10CFB800C7ED00BA43ED01BAC8ED00BA0136032E39
:10CFC80009F1040908F1040807F1040705F104054B
:10CFD8007FF452AE654B1B78072B01F01482012BAE
:10CFE80001F091840023029394F87C31002B40F0E7
:10CFF80097855F4B5F4A1B68126813F4805C92F850
:10D008002C2040F0A4865C495C4891ED006A408B76
:10D018005B4984ED636A91ED007A5A4984ED647A3C
:10D0280007EE900AF8EEE76AD1ED037A564984EDE7
:10D03800616A37EE467A77EEE67AD1ED006A84EDDA
:10D04800607A012184F89411C7EEA65A4F485049D6
:10D0580090ED005A4F489FED506A90ED004A4F48B6
:10D06800DFED4F6AD0ED004A91ED007A35EE045AB3
:10D07800F7EE007AF4EEE75A35EE245AF1EE10FA9C
:10D0880088BFF0EE675A25EE065AF4EEE65AB1EE7E
:10D09800476AF1EE10FAB4EEC65AB8BFF0EE665A17
:10D0A800F1EE10FAC4ED665A00F1FD87B4EEC75AE6
:10D0B800F1EE10FA88BFB0EE475A3449DFED366A10
:10D0C800D1ED017A334991ED014A344977EE847AFA
:10D0D800D1ED014A77EEA47A67EEA67AB4EEE76A54
:10D0E800F1EE10FA08DCB4EEE77AF1EE10FA8CBF34
:10D0F800B0EE676AB0EE476A2449DFED276AD1EDE2
:10D10800027A2449D1ED024A264977EEA47A91EDB4
:10D11800007A67EEA67AB1EE473AF4EEC37AF1EEFA
:10D1280010FA4ED444E000BFC465002034780020D3
:10D13800403A0020BC5900206C6500209400002073
:10D14800E065002078650020AC640020A864002019
:10D1580000650020FC640020B85900201829002030
:10D16800EC5F0020D0650020846500205461002019
:10D17800CC4D0020DC590020D07300205C4F0020EB
:10D188005C35002058620020703500203073002084
:10D19800E46500203C7300206F12833A4873002036
:10D1A80000000000E865002098650020C0650020A8
:10D1B800F4EEC77AF1EE10FA8CBFB0EE473AB0EE53
:10D1C800673AED49497809B9B1EE433A002A41F086
:10D1D8003E82F7EE003ADFF8C8B39BF80020002A39
:10D1E80002F03782E549DFEDE67AD1ED024AD1ED6A
:10D1F800016A91ED037A66EE244AE5EE264AE3EEEB
:10D20800074A63EEA44AF4EEE74AF1EE10FAB4BF17
:10D21800B0EE674AB0EE644A98BFF0EE647A012A2D
:10D22800CDED0A4A02F0368291ED067AD1ED052A53
:10D23800D1ED076A26EE077AA5EE227AA3EE267AC2
:10D2480023EE877AB4EEE77AF1EE10FAB4EEC47AF8
:10D258008CBFF0EE676AF0EE476AF1EE10FA88BF0D
:10D26800F0EE676AB4BFF0EE447AF0EE477A022A2D
:10D278008DED0B7A00F0DE8091ED0A7AD1ED092A66
:10D2880091ED0B4A26EE077AA5EE227AA3EE047AF0
:10D2980023EE877AB4EEE67AF1EE10FAB4EEE77A86
:10D2A8008CBFB0EE664AB0EE474AF1EE10FA98BF6E
:10D2B800F0EE446AA8BFF0EE477A032A8DED0C7AA7
:10D2C80000F0B88091ED0E7AD1ED0D2A91ED0F4A5C
:10D2D80026EE077AA5EE227AA3EE047A23EE877A61
:10D2E800B4EEE67AF1EE10FAB4EEE77A8CBFB0EE5F
:10D2F800664AB0EE474AF1EE10FA98BFF0EE446A7B
:10D30800A8BFF0EE477A042A8DED0D7A00F09280DE
:10D3180091ED124AD1ED112A91ED137A26EE044AC5
:10D32800A5EE224AA3EE074A23EE844AB4EEE64A63
:10D33800F1EE10FAB4EEE74A8CBFB0EE667AB0EEC2
:10D34800447AF1EE10FA98BFF0EE476AA8BFF0EE03
:10D35800447A052A8DED0E4A6CD091ED164AD1ED2E
:10D36800152A91ED177A26EE044AA5EE224AA3EE75
:10D37800074A23EE844AB4EEE64AF1EE10FAB4EE18
:10D38800E74A8CBFB0EE667AB0EE447AF1EE10FA56
:10D3980098BFF0EE476AA8BFF0EE447A062A8DEDF2
:10D3A8000F4A47D091ED1A4AD1ED192A91ED1B7A0F
:10D3B80026EE044AA5EE224AA3EE074A23EE844A43
:10D3C800B4EEE64AF1EE10FAB4EEE74A8CBFB0EEDE
:10D3D800667AB0EE447AF1EE10FA98BFF0EE476A3A
:10D3E800A8BFF0EE447A072A8DED104A22D091EDBD
:10D3F8001E7AD1ED1D2A91ED1F4A26EE077AA5EE79
:10D40800227AA4EE037A27EE237AB4EEE67AF1EED6
:10D4180010FAB4EEE77A8CBFB0EE666AB0EE476AEF
:10D42800F1EE10FA8DED117A98BFF0EE466AA8BFBA
:10D43800F0EE477A77EEE67AF7EE006AF4EEE67AEF
:10D44800F1EE10FAC4ED4C7A43F39A8286EEA77A8D
:10D45800022ADDED0B7A67EE244A67EE877ACDED76
:10D468000A4ACDED0B7A2DD0DDED0C7A67EE877A7E
:10D47800032ACDED0C7A25D0DDED0D7A67EE877A9B
:10D48800042ACDED0D7A1DD0DDED0E7A67EE877A90
:10D49800052ACDED0E7A15D0DDED0F7A67EE877A85
:10D4A800062ACDED0F7A0DD0DDED107A67EE877A7A
:10D4B800072ACDED107A05D0DDED117A27EE877AAF
:10D4C8008DED117A2F49096811F0805800F0968780
:10D4D800F6EE005AC4ED665A002A02F0B18094F9BB
:10D4E8009401D4ED644A284D284994ED636A284E86
:10D4F800284FDFF8B0E0B5F81AA0C978B6F9069059
:10D5080097ED005A9EF800E0D4ED606AD4ED617A98
:10D5180007EE100AFDEEE44A1F4814EE905A007810
:10D52800FDEEC64A03F0100603F4800300F001077D
:10D53800B8EEC77A14EE900A0193002941F0C6802C
:10D548000E49002E40F07C8791ED006A9DED0A5A45
:10D55800124B25EE866AA5EE076AB0EE675AA6EE6C
:10D56800265ABDEEC56A16EE10EA16EE106AAE45EA
:10D57800A8BF2E4618E000BF80750020DC340020CC
:10D58800000000002C7800205C4F00201849002083
:10D59800C85F0020B8340020EC5F002090730020A2
:10D5A80035610020806A00207045C8BF064606EE37
:10D5B800106AB8EEC66A012A83ED006A00F0DC80C2
:10D5C80091ED046A9DED0B5A25EE866AA5EE076A71
:10D5D800B0EE675AA6EE265ABDEEC56A16EE10EAF8
:10D5E80016EE106AAE45A8BF2E467045C8BF06465F
:10D5F80006EE106AB8EEC66A022A83ED016A00F0E8
:10D60800BB8091ED086A9DED0C5A25EE866AA5EE61
:10D61800076AB0EE675AA6EE265ABDEEC56A16EE40
:10D6280010EA16EE106AAE45A8BF2E467045C8BF70
:10D63800064606EE106AB8EEC66A032A83ED026A49
:10D6480000F09A8091ED0C6A9DED0D5A25EE866AE0
:10D65800A5EE076AB0EE675AA6EE265ABDEEC56A71
:10D6680016EE10EA16EE106AAE45A8BF2E467045B3
:10D67800C8BF064606EE106AB8EEC66A042A83EDED
:10D68800036A79D091ED106A9DED0E5A25EE866AEF
:10D69800A5EE076AB0EE675AA6EE265ABDEEC56A31
:10D6A80016EE10EA16EE106AAE45A8BF2E46704573
:10D6B800C8BF064606EE106AB8EEC66A052A83EDAC
:10D6C800046A59D091ED146A9DED0F5A25EE866AC9
:10D6D800A5EE076AB0EE675AA6EE265ABDEEC56AF1
:10D6E80016EE10EA16EE106AAE45A8BF2E46704533
:10D6F800C8BF064606EE106AB8EEC66A062A83ED6B
:10D70800056A39D091ED186A9DED105A25EE866AA2
:10D71800A5EE076AB0EE675AA6EE265ABDEEC56AB0
:10D7280016EE10EA16EE106AAE45A8BF2E467045F2
:10D73800C8BF064606EE106AB8EEC66A072A83ED29
:10D74800066A19D091ED1C6A9DED115A65EE865A4C
:10D75800E7EE055AE6EEA57AFDEEE77A17EE901A9F
:10D768008D42A8BF0D468842C8BF054607EE905AAD
:10D77800F8EEE77AC3ED077A2FB922B19200D349C0
:10D78800D34822F0E5FFD34B1B68002B40F0A4845C
:10D79800D14B1B7893B19BF8000060B1CC4ECF4FB2
:10D7A8000025E8B23B68B6EC010A98479BF80000F0
:10D7B80001358542F5DBCA4B1B689847C94B1B7876
:10D7C800072B00F03586012384F8003113B0BDEC37
:10D7D8000C8BBDE8F08FC44B1B78013BDBB2FFF725
:10D7E80012BAC24B02934FF47A751B68B5FBF3F378
:10D7F800C3EB4315BE49DFF8248391F80190B9497A
:10D80800B8F906000F7803EB8503DD00ADB2AE4230
:10D8180001F08586DBF88810BBF93CE0DBF86C305A
:10D828004A1C07EE90EA7344012ACBF88820CBF80B
:10D838006C30F8EEE77A01F07F86DBED1E5ADBEDFF
:10D84800206A07EE102A37EEE56AB8EEC75A012EAD
:10D8580086EE057A37EE257A77EEC77A8BED1F7A52
:10D86800E7EE866A8BED1E7AF0EE667ACBED216ADA
:10D87800CBED206A02F05080DBF89C10BBF93EE04B
:10D88800DBF870304A1C07EE90EA7344012ACBF8A3
:10D898009C20CBF87030F8EEE77A01F06886DBED73
:10D8A800235ADBED256A07EE102A37EEE56AB8EE53
:10D8B800C75A012E86EE057A37EE257A77EEC77AB3
:10D8C8008BED247AE7EE866A8BED237AF0EE667AA2
:10D8D800CBED266ACBED256A02F04780DBF8B01065
:10D8E800BBF940E0DBF874304A1C07EE90EA734459
:10D8F800012ACBF8B020CBF87430F8EEE77A01F0C3
:10D908005186DBED285ADBED2A6A07EE102A37EE3E
:10D91800E56AB8EEC75A012E86EE057A37EE257A03
:10D9280077EEC77A8BED297AE6EE276A8BED287AAF
:10D93800F0EE667ACBED2B6ACBED2A6A02F03E80D8
:10D94800A8F80600BBF8B430664A013B1778ABF874
:10D95800B43002990023072F4B608B60CB607FF4B3
:10D9680046A9F8F725FEDFF8B48194F82831049326
:10D97800A0EB0A00A8F80000002B3FF43EA9013BE9
:10D9880084F8283113B0BDEC0C8BBDE8F08F94ED12
:10D99800567AB1F90000D4ED576AB1F902E0554A58
:10D9A800F4EEC76A80EAE0738EEAEE71A3EBE073E7
:10D9B800F1EE10FAA1EBEE71B8BFF0EE476A8B42B8
:10D9C800B8BF0B4607EE103A1378B8EEC77A27EEC1
:10D9D800287A002B40F0FE81474B93ED006AB4EEA5
:10D9E800CA6AF1EE10FA40F18487F7EE005A75EE34
:10D9F800C65A3BEE477A65EEAA5A404BA7EE256A0F
:10DA080093ED007A26EE076AB5EEC06AF1EE10FAD9
:10DA180040F2F084C9EE865AB7EE007AB0EE476A53
:10DA2800A6EEE56AF0EE466AF4EEC76AF1EE10FA81
:10DA380088BFF0EE476AF5EEC06AF1EE10FAB8BF9B
:10DA4800F0EE6B6A2E4B93ED007A67EE877AA7EEBD
:10DA5800A68AFFF7B7B92B4B2B4C19682B4ADFF86E
:10DA6800BC8094F80031C9691288A8F80010A8F899
:10DA78000220002B3EF43CAF04F066FD002384F83E
:10DA88000031184B1B78072B7EF432AFF8F790FD66
:10DA98008246FEF72FBF1E4B1E4A2B4493ED007A99
:10DAA800D2ED007A1C4B67EE277AF7EE006AF4EEA7
:10DAB800E67AF1EE10FA93ED007A88BFF0EE667A16
:10DAC80067EE877A27EE888AFFF72DBABC340020E4
:10DAD800907300209C640020886D0020746A0020E8
:10DAE8007C6A00205461002068650020BC4D00203D
:10DAF800244B0020A4650020AC650020A065002010
:10DB08009C650020385E0020AC270020144A0020C5
:10DB180004290020946500209065002058610020A9
:10DB2800D94BDFF8B8B31B789BF80020DD077FF5E9
:10DB380024AE002A3FF427AED4ED573A94ED564A66
:10DB4800D24BD4ED617A93ED005A94ED607AD4ED1E
:10DB5800545A94ED536ACE49CE4BF4EEC43AF3EEE0
:10DB6800046AF1EE10FA77EEA64A00F1578791EDB4
:10DB7800026A26EE656AB0EE674AA6EE074AB4EE78
:10DB8800E44A34EE666AF1EE10FA48BFB0EE456A30
:10DB9800012A83ED006A3FF4F6AD91ED066A26EEA0
:10DBA800656AB0EE674AA6EE074AB4EEE44A34EE78
:10DBB800666AF1EE10FA48BFB0EE456A022A83EDB4
:10DBC800016A3FF4E0AD91ED0A6A26EE656AB0EEAF
:10DBD800674AA6EE074AB4EEE44A34EE666AF1EE06
:10DBE80010FA48BFB0EE456A032A83ED026A3FF493
:10DBF800CAAD91ED0E6A26EE656AB0EE674AA6EEEA
:10DC0800074AB4EEE44A34EE666AF1EE10FA48BF09
:10DC1800B0EE456A042A83ED036A3FF4B4AD91ED92
:10DC2800126A26EE656AB0EE674AA6EE074AB4EEB7
:10DC3800E44A34EE666AF1EE10FA48BFB0EE456A7F
:10DC4800052A83ED046A3FF49EAD91ED166A26EE2F
:10DC5800656AB0EE674AA6EE074AB4EEE44A74EE87
:10DC6800666AF1EE10FA48BFF0EE456A062AC3ED7F
:10DC7800056A3FF488ADD1ED1A6A66EEE56AB0EE42
:10DC8800674AA6EE874AB3EE046AB4EEE44A74EE35
:10DC9800466AF1EE10FA48BFF0EE456A072AC3ED6E
:10DCA800066A3FF470ADD1ED1E6A66EEE55AE5EE00
:10DCB800877AF4EEE74A77EEC67AF1EE10FAC8BF33
:10DCC800F0EE457AC3ED077A5DE5734BC7ED00BA10
:10DCD8001B689342BFF6B6A8704B1A88002384F8D5
:10DCE8006431002A41F011846D4A6E4B117818682E
:10DCF80081F00101F4F728FBFFF7ACB86A4EDFF8B2
:10DD0800E08106F5F47506F51577F6EC017A9BEDDA
:10DD1800080ADBF81432F8EEE77A284627EE800A7C
:10DD28009847A5F1E000DBF834319847A5F1700079
:10DD3800DBF8A4319847D6F8F400DBF8B8309847F8
:10DD48002435AF42A8EC010ADFD1FEF74BBF4E499C
:10DD58000978C80703D45549098BA4F88811544990
:10DD68005448098890ED037A07EE901AF8EEE77A9E
:10DD7800B4EEE77AF1EE10FA40F208864E480088D1
:10DD880007EE900AF8EEE77AB4EEE77AF1EE10FAC9
:10DD9800C0F2CC8549484A49D0ED006A91ED006A45
:10DDA8004848C4ED636ABCEEC75A76EE665A15EE6B
:10DDB800101AC4ED616AC4ED605A84ED646AA4F86F
:10DDC80088110121D0ED006A84F8941177EE677A02
:10DDD800FFF73AB93C4B93ED005AB5EEC05AF1EE55
:10DDE80010FA40F30783394BD3ED004AF5EEC04AE9
:10DDF800F1EE10FA40F3FE8234EEC77A66EEE95A85
:10DE080087EE246AC5EE856AB7EE007AB4EEC76A73
:10DE1800F1EE10FA88BFB0EE476AB5EEC06AF1EECF
:10DE280010FA76EE876AB8BFB0EE6B6A66EE266ABD
:10DE3800FAE5274A92ED007AF0EEE76AF4EEC76A4F
:10DE4800F1EE10FA7FF790A8224A92ED007AF0EEF0
:10DE5800CD6AF4EEC76AF1EE10FA7FF785A81E4A7C
:10DE680099ED007AD2ED006AB0EEC77AB4EEE67AA0
:10DE7800F1EE10FA7FF578A801220399C4F8681129
:10DE880084F86421FFF774B8EC5F0020B8340020F0
:10DE9800DC34002090730020C0650020D060002092
:10DEA800D2600020D4600020684B00205C4F002026
:10DEB8007435002058620020763500206035002037
:10DEC8005C3500207C350020A0650020A865002076
:10DED800D4650020D0650020D86500203561002079
:10DEE800C04D00200299724BD1ED017A93ED007A72
:10DEF800F0EEE77AF4EEC77AF1EE10FA7EF5AAAF03
:10DF0800D1ED027AF0EEE77AB4EEE77AF1EE10FAA4
:10DF18007EF7A0AFD1ED037AF0EEE77AB4EEE77AB8
:10DF2800F1EE10FA7EF796AF624B1B689A077FF501
:10DF3800D3AE6149614BB3F90C20B1F900E06048F8
:10DF4800AEEB020E00688EEAEE72A2EBEE7282422F
:10DF5800BEF680AFB3F90E30B1F90220D21A82EAC8
:10DF6800E273A3EBE27398427EF774AFB4E6554BC5
:10DF780099ED007AD3ED006AB0EEC77AB4EEE67A8E
:10DF8800F1EE10FA7FF706A8FFF701B807EE103A8E
:10DF98004D4BDFF840811B78C4F81061B8EEC77AA2
:10DFA800F7EE006A132B86EE879AB8F90400B4F8E6
:10DFB80014519BED080A01F03482444B444A93ED16
:10DFC800001A93ED053A93ED122A93ED176AD3EDF3
:10DFD800091A93ED0E4AD3ED015AD3ED063A93EDA3
:10DFE8000A7A93ED0F5AD3ED132AD3ED186AD3EDBD
:10DFF800044AD3ED030A67EE897A69EE288A29EE86
:10E00800088AA1EE273A02EB85060021A2EE286ACB
:10E01800C4F80411C4F80811A1EE884AE5EEA73A3D
:10E02800A7EE085A93ED167AD3ED0D5A93ED021A1E
:10E03800D3ED0C1A86ED003AE2EEA86A64EEC34A04
:10E0480027EE467A93ED0B2AD3ED152A86ED204A62
:10E05800E0EEC33A65EEC45A93ED143AC3ED053ABF
:10E06800E1EE274AF0EE477AA1EEC45AE2EE085AEA
:10E07800E2EEC66AE3EE287AC3ED064A83ED0E5A4D
:10E08800C3ED0F5A86ED406AC3ED176AC3ED187ADF
:10E09800C4F80C11013505F01F05A4F81451A8F8AF
:10E0A8000400FEF782BCB0EE465AFFF706B800BF80
:10E0B800CC65002034780020BC590020403A00206C
:10E0C800C8650020D8650020546100206C3D002000
:10E0D800E83A002058610020B94B1B78192B07D863
:10E0E8000121B84A01FA03F31A40002A41F0748466
:10E0F800B54BB64EB64F01931B689D061CD5FB7AEF
:10E10800FF2B04D0B34A12789A4201F2EF80B7F994
:10E118000880FB7DA6F80080FF2B04D0AD4A12785A
:10E128009A4201F2DE80B7F914507580082020F079
:10E13800F9FB002840F03186B7F90600B6F900C0AF
:10E14800B6F902E0B7F91210B7F91E20B6F9045073
:10E15800B7F90430B6F906806045A8BF6046714536
:10E16800A8BF7146AA42A8BF2A469C45A8BF034635
:10E178003380B7F91030B6F908009E45B8BF194684
:10E18800B7F92A307180B7F91C10B7F934E0434564
:10E19800A8BF43468D42B4BF0D461546B7F9362091
:10E1A800B580B7F92850B6F90A108242A8BF0246CE
:10E1B800A845ACBF9846A846B7F94230B6F90C5006
:10E1C800A6F806808B42A8BF0B467045ACBF104628
:10E1D8007046B7F94E203081B7F94000B6F90EE025
:10E1E800AA42A8BF2A468842C8BF0346B7F95A00C0
:10E1F800B7F94C1073817045B7F95830764FA8BFFE
:10E2080070469E45A8BF0346A942D8BF1146B181B2
:10E21800F381BB892BB3DFF8D081DFF8D0A1DFF819
:10E22800B09108F11005B8F9023000EE103A5046E6
:10E23800B8EEC00AF2F7FEF922F092FCB9F9043000
:10E24800B9F9062000B298420AF1240A09F10C092A
:10E2580003DB82421346A8BF034628F8023FA845BD
:10E26800E1D1574B1B78013B182B72D8DFE813F02C
:10E278005F00710071001900710071007100780869
:10E2880071007100710071007100980871007100CF
:10E2980071007100710019008608710071009808FA
:10E2A8005F004E4BB6F908101A6802B111609B69FD
:10E2B800B6F90A2003B11A60019B1B689A0601F19E
:10E2C800E98602220492D9027FF562AAFE7B112E0A
:10E2D8003FF65EAA424B079333F91630DDF81080FB
:10E2E80000EE103A4046B8EEC00A751C1FF0B2F9AD
:10E2F80006F10E074346EDB29E1BFFB2DDF81C90F7
:10E3080000E0454605F10108A819122D5FFA88F8C2
:10E31800C0B23FF43DAA39F9153000EE103AB8EE14
:10E32800C00A1FF097F9B845EBD1FFF731BABB7BAC
:10E33800002B42F079802B4B1B7813F0010342F03D
:10E348007380264A1268002A02F04D841360012364
:10E358000493019B1B68980603D4194A1278052A6E
:10E36800B1D1049A13460233551CDBB21046EDB204
:10E378000493B6F9003000EE103AB8EEC00A1FF068
:10E3880069F9B6F9023000EE103A2846B8EEC00A2C
:10E398001FF060F9019B1B6895E722F0E1FB29F863
:10E3A8001600FEF70DBC95ED007A0BEB4602B8EEB1
:10E3B800C78A928F29F8162028EE278AFEF7DEBB37
:10E3C800A064002032413003CC4D0020807300202F
:10E3D800506600206849002094670020A467002048
:10E3E800C85F0020EC5F00207E7300209862002048
:10E3F800000000005FED026AFFF724BB59023FF5F9
:10E4080067A8FFF769B8F8F7D3F8A94B059A1B78FE
:10E41800DFF8A082801A012BA8F8020000F07582AC
:10E42800072B7EF4DFADF8F7C3F80290FEF7DCBDEA
:10E43800F8F7BEF8029A9F4B801AD880FFF7C3B945
:10E44800002F41F0618191ED006A9DED0A5A9A4BC7
:10E4580025EE866AA5EE076AB0EE675AA6EE265A3A
:10E46800BDEEC56A16EE107A16EE106AAF42A8BF66
:10E478002E46B842C8BF064606EE106AB8EEC66A0F
:10E48800012A83ED006A3FF479A991ED046A9DEDB4
:10E498000B5A25EE866AA5EE076AB0EE675AA6EE15
:10E4A800265ABDEEC56A16EE107A16EE106AAF420D
:10E4B800A8BF2E46B842C8BF064606EE106AB8EE98
:10E4C800C66A022A83ED016A3FF458A991ED086AE9
:10E4D8009DED0C5A25EE866AA5EE076AB0EE675ADE
:10E4E800A6EE265ABDEEC56A16EE107A16EE106A2A
:10E4F800AF42A8BF2E46B842C8BF064606EE106A0D
:10E50800B8EEC66A032A83ED026A3FF437A991ED93
:10E518000C6A9DED0D5A25EE866AA5EE076AB0EEE7
:10E52800675AA6EE265ABDEEC56A16EE107A16EEA2
:10E53800106AAF42A8BF2E46B842C8BF064606EECC
:10E54800106AB8EEC66A042A83ED036A3FF416A976
:10E5580091ED106A9DED0E5A25EE866AA5EE076AC2
:10E56800B0EE675AA6EE265ABDEEC56A16EE107AC8
:10E5780016EE106AAF42A8BF2E46B842C8BF06467C
:10E5880006EE106AB8EEC66A052A83ED046A3FF4FF
:10E59800F5A891ED146A9DED0F5A25EE866AA5EE51
:10E5A800076AB0EE675AA6EE265ABDEEC56A16EEA1
:10E5B800107A16EE106AAF42A8BF2E46B842C8BFFE
:10E5C800064606EE106AB8EEC66A062A83ED056AA4
:10E5D8003FF4D4A891ED186A9DED105A25EE866A8D
:10E5E800A5EE076AB0EE675AA6EE265ABDEEC56AD2
:10E5F80016EE107A16EE106AAF42A8BF2E46B84241
:10E60800C8BF064606EE106AB8EEC66A072A83ED4A
:10E61800066A3FF4B3A891ED1C6A9DED115A65EEA8
:10E62800865AE7EE055AE6EEA57AFDEEE77A17EE8A
:10E63800901A8D42A8BF0D468842C8BF054607EE0E
:10E64800905AF8EEE77AC3ED077AFFF796B81B4AB7
:10E65800517900293EF4BDAD1949097800293EF4E5
:10E66800B8AD1278DFED174A07EE902A164AB8EED1
:10E67800677A128807EE901A06EE902AF8EEE77A83
:10E68800F8EE666A67EE277AB7EE007AC7EEA63A22
:10E69800F4EEE43AF1EE10FA88BFF0EE643AF4EEE4
:10E6A800C73AF1EE10FAB8BFF0EE473AFEF793BD5D
:10E6B80054610020586100209073002000780020E9
:10E6C80056620020713DAA3F40620020002E00F0F3
:10E6D8005482002F41F0D286C049BEF1000F41F0AC
:10E6E8000F8591ED006ADDED0A4ABD4B25EE866A7D
:10E6F800BDEEC55AA4EE876A15EE100AB0EE675A49
:10E70800A6EE265ABDEEC56A16EE107A16EE106A07
:10E71800AF42A8BF2E46B842C8BF064606EE106AEA
:10E72800B8EEC66A012A83ED006A3FF427A891ED86
:10E73800046A9DED0B5A25EE866AA5EE076AB0EECF
:10E74800675AA6EE265ABDEEC56A16EE107A16EE80
:10E75800106AAF42A8BF2E468742B8BF064606EEEB
:10E76800106AB8EEC66A022A83ED016A3FF406A869
:10E7780091ED086A9DED0C5A25EE866AA5EE076AAA
:10E78800B0EE675AA6EE265ABDEEC56A16EE107AA6
:10E7980016EE106AAF42A8BF2E468742B8BF06469B
:10E7A80006EE106AB8EEC66A032A83ED026A3EF4E2
:10E7B800E5AF91ED0C6A9DED0D5A25EE866AA5EE42
:10E7C800076AB0EE675AA6EE265ABDEEC56A16EE7F
:10E7D800107A16EE106AAF42A8BF2E468742B8BF1D
:10E7E800064606EE106AB8EEC66A042A83ED036A86
:10E7F8003EF4C4AF91ED106A9DED0E5A25EE866A7F
:10E80800A5EE076AB0EE675AA6EE265ABDEEC56AAF
:10E8180016EE107A16EE106AAF42A8BF2E4687424F
:10E82800B8BF064606EE106AB8EEC66A052A83ED3A
:10E83800046A3EF4A3AF91ED146A9DED0F5A25EEDC
:10E84800866AA5EE076AB0EE675AA6EE265ABDEEAE
:10E85800C56A16EE107A16EE106AAF42A8BF2E46A9
:10E868008742B8BF064606EE106AB8EEC66A062AA0
:10E8780083ED056A3EF482AF91ED186A9DED105A5A
:10E8880025EE866AA5EE076AB0EE675AA6EE265A06
:10E89800BDEEC56A16EE107A16EE106AAF42A8BF32
:10E8A8002E468742B8BF064606EE106AB8EEC66A1C
:10E8B800072A83ED066A3EF461AF91ED1C6A9DED6F
:10E8C800115A65EE865AE7EE055AE6EEA57AFDEE90
:10E8D800E77A17EE901A8D42A8BF0D468842D8BF36
:10E8E800284607EE900AF8EEE77AC3ED077AFEF7B6
:10E8F80044BF3C4B93ED006AFFF786B8F7F758FE24
:10E908000590FEF789B9DFF81081F7F751FE364A0E
:10E91800D4F8783112680290C31A9A1AC4F87801A8
:10E92800A8F80430A8F80620FEF75EBBB4F8880102
:10E93800884240F245852D482D49D0ED007A91ED69
:10E94800007A2C48C4ED637A77EE676AC4ED617A81
:10E958000121C4ED606A84ED647AD0ED006ADFEDD0
:10E96800267A84F89411FEF76FBB244B1B88002B82
:10E9780040F04585224A234B11781868F3F7E4FCE8
:10E98800D4F86821039B9A1AFEF733BA1E491F4828
:10E99800D1ED006A1E4990ED006A0978C4ED636AFA
:10E9A80084ED646A002940F0B78476EEC65AF0EE2A
:10E9B800466ABCEEC76A1748C4ED605A16EE101ACC
:10E9C800C4ED616AA4F88811FF21D0ED006A84F8CB
:10E9D800941177EEC77AFEF737BB00BFDC3400200E
:10E9E80090730020A0650020647500206035002029
:10E9F8005C3500207C35002000000000D06000203D
:10EA0800D2600020D4600020D0730020643500203C
:10EA1800806A00207835002058610020D1ED015A25
:10EA280065EEC65AB0EE674AA5EE874AB4EEE44AE8
:10EA380074EE665AF1EE10FA48BFF0EE455A012A14
:10EA4800C3ED005A3EF49FAED1ED055A65EEC65AA5
:10EA5800B0EE674AA5EE874AB4EEE44A74EE665A09
:10EA6800F1EE10FA48BFF0EE455A022AC3ED015AFA
:10EA78003EF489AED1ED095A65EEC65AB0EE674A42
:10EA8800A5EE874AB4EEE44A74EE665AF1EE10FA3F
:10EA980048BFF0EE455A032AC3ED025A3EF473AE5E
:10EAA800D1ED0D5A65EEC65AB0EE674AA5EE874A13
:10EAB800B4EEE44A74EE665AF1EE10FA48BFF0EE8E
:10EAC800455A042AC3ED035A3EF45DAED1ED115AFE
:10EAD80065EEC65AB0EE674AA5EE874AB4EEE44A38
:10EAE80074EE665AF1EE10FA48BFF0EE455A052A60
:10EAF800C3ED045A3EF447AED1ED155A65EEC65A39
:10EB0800B0EE674AA5EE874AB4EEE44A74EE666A48
:10EB1800F1EE10FA48BFF0EE456A062AC3ED056A21
:10EB28003EF431AED1ED196A66EEC66AB0EE674AB8
:10EB3800A6EE874AF3EE045AB4EEE44A74EE656A28
:10EB4800F1EE10FA48BFF0EE456A072AC3ED066AEF
:10EB58003EF419AED1ED1D6A26EEC66AE6EE077AD6
:10EB6800F4EEE47A77EEE57AF1EE10FAB8BFF0EE5B
:10EB7800457AC3ED077AFEF706BEC949BEF1000F14
:10EB880041F04A8191ED006ADDED0A4AC54B25EE58
:10EB9800866ABDEEC55AA4EE876A15EE100AB0EE75
:10EBA800675AA6EE265ABDEEC56A16EE10EA16EEAC
:10EBB800106AAE45A8BF2E467045C8BF064606EE89
:10EBC800106AB8EEC66A012A83ED006A3EF4D4AD35
:10EBD80091ED046A9DED0B5A25EE866AA5EE076A4B
:10EBE800B0EE675AA6EE265ABDEEC56A16EE10EAD2
:10EBF80016EE106AAE45A8BF2E468645B8BF064633
:10EC080006EE106AB8EEC66A022A83ED016A3EF47F
:10EC1800B3AD91ED086A9DED0C5A25EE866AA5EE16
:10EC2800076AB0EE675AA6EE265ABDEEC56A16EE1A
:10EC380010EA16EE106AAE45A8BF2E468645B8BF44
:10EC4800064606EE106AB8EEC66A032A83ED026A23
:10EC58003EF492AD91ED0C6A9DED0D5A25EE866A53
:10EC6800A5EE076AB0EE675AA6EE265ABDEEC56A4B
:10EC780016EE10EA16EE106AAE45A8BF2E46864577
:10EC8800B8BF064606EE106AB8EEC66A042A83EDD7
:10EC9800036A3EF471AD91ED106A9DED0E5A25EEB2
:10ECA800866AA5EE076AB0EE675AA6EE265ABDEE4A
:10ECB800C56A16EE10EA16EE106AAE45A8BF2E46D3
:10ECC8008645B8BF064606EE106AB8EEC66A052A3B
:10ECD80083ED046A3EF450AD91ED146A9DED0F5A30
:10ECE80025EE866AA5EE076AB0EE675AA6EE265AA2
:10ECF800BDEEC56A16EE10EA16EE106AAE45A8BF5C
:10ED08002E468645B8BF064606EE106AB8EEC66AB5
:10ED1800062A83ED056A3EF42FAD91ED186A9DED44
:10ED2800105A25EE866AA5EE076AB0EE675AA6EE77
:10ED3800265ABDEEC56A16EE10EA16EE106AAE4502
:10ED4800A8BF2E468645B8BF064606EE106AB8EE3E
:10ED5800C66A072A83ED066A3EF40EAD91ED1C6A79
:10ED68009DED115A65EE865AE7EE055AE6EEA57A4C
:10ED7800FDEEE77A17EE901A8D42A8BF0D4688423D
:10ED8800D8BF284607EE900AF8EEE77AC3ED077A6F
:10ED9800002F7EF4F8ACFEF7F0BC94F8BC31012BE0
:10EDA80001F0A184404B97F916005A8897F90AE0B8
:10EDB8001B883E4910FB03F31EFB02F281FB020C89
:10EDC80081FB0301D217DB17C2EB2C12C3EB211313
:10EDD80042441D4432807580FFF7AEB9344FD4EDFC
:10EDE800017A94ED006A38887B6977EEA77AF0EEAD
:10EDF800006AB0EE677AA6EE267A013804EBC00204
:10EE0800D6EE267A083A1033F6EE003A27EE237A41
:10EE180067EEA37A84ED207AC4ED217A254C274643
:10EE280004F1800192ED027A92ED036AD7ED036A4C
:10EE3800D7ED027A53ED014A13ED025A37EE674ACD
:10EE480076EEC65A77EE277AE4EE845A0138A2F1B4
:10EE58000802E5EE047A07F1080703F1080336EE25
:10EE6800267A01F10801E4EE877AE5EE475A67EE63
:10EE7800A37A25EEA37AC1ED007A81ED017AD1D18A
:10EE8800142E7DF446AEF7F793FB029BDFF828803B
:10EE9800C01AA8F80200D4F81851FDF73ABE00BF0E
:10EEA800DC34002090730020BC5900201F85EB51F2
:10EEB800D03A0020AC27002058610020DFF8949455
:10EEC80099F80020900801F08986DFF88CE400F1B9
:10EED800010C4FEA4C1C0EEB0C070EF12003AEF1AF
:10EEE800700113ED076A53ED056A13ED037A53EDCC
:10EEF800017A53ED025A13ED084A53ED064A13ED11
:10EF0800045A26EE066A66EEA66A27EE077A67EEC8
:10EF1800A77AA4EE046A20339F42E4EEA46A01F1C2
:10EF28001001A5EE057AE5EEA57AF1EEC65AB1EE26
:10EF3800E66AF1EEC76AB1EEE77A41ED085A01EDEB
:10EF4800076A41ED066A01ED057ACAD1ACF1200CD9
:10EF5800E64404EB001012F0030318BF0EF1080E8C
:10EF68000FD05EED017A1EED027A67EEA77A013BBB
:10EF7800E7EE077A0EF1080EB1EEE77AA0EC017A17
:10EF8800EFD1142E01F00C860135C4F81851FDF7A5
:10EF98002DBDE34FE348BA68B98920F051FCE24B34
:10EFA8001E78142E01F07885D4F818510135C4F86C
:10EFB800185114E7DA4FB7F800E0D7F804C04FEA61
:10EFC8005E084FEA880204EB8E055FEADE0E04EB6A
:10EFD800020300F0A08010320EF1010ED34803EBBB
:10EFE8000E1E2A4410330CF1100605F1100151EDE4
:10EFF800032A51ED043A10ED043A10ED032A51EDBD
:10F00800026A11ED016A50ED020A10ED010A12EDD3
:10F01800044A12ED035A53ED044A53ED035A13ED13
:10F02800027A53ED017A12ED021A52ED011A73EECB
:10F03800238A32EE228A40ED048A00ED038A70EEBC
:10F04800A68A30EE068A40ED028A00ED018A74EE47
:10F05800848A35EE858A43ED048A03ED038A77EEC8
:10F06800018A37EEA18A43ED028A03ED018A73EE25
:10F07800633A75EE655A16ED035A32EE623A74EE4B
:10F08800644A25EE638A16ED044A23EE052A64EEE7
:10F09800652AA3EE048A10339E4524EE843AA3EE33
:10F0A800842A00F1100006F11006A5EE853A01F158
:10F0B800100102F11002E4EE852A01ED078A01ED44
:10F0C800082A02ED073A42ED082A56ED055A16EDD0
:10F0D800065A70EEE66A30EE466A31EE477A71EE0D
:10F0E800E77A26EE253A65EEE63A25EE674A67EEB8
:10F0F800054AE6EE053AA6EE853AA7EE254AE7EE7A
:10F10800A54A01ED063A41ED053A02ED064A42EDFF
:10F11800054A7FF46CAF1FFA88F862464146814879
:10F1280019F0DAFE41467A68284619F0D5FE7E4B7A
:10F138001B78142B7FF4AFAEA5E6D4F81CC1B4F845
:10F1480014917B4BC9F120085FFA88F809EB4C173A
:10F1580003EB87075FEA980301F084840133180101
:10F168007449724A07EB000E07F1100313ED024AC7
:10F1780013ED035A13ED016A13ED047A51ED024AB7
:10F1880051ED035A51ED016A51ED047A64EE244AB7
:10F1980065EE255A66EE266A67EE277A10339E4595
:10F1A80042ED024A42ED035A42ED016A42ED047A09
:10F1B80001F1100102F11002D8D15F49A0F110024B
:10F1C800174401EB020E224418F0030309D0B7ECF0
:10F1D800017AFEEC017A67EE277A013BE2EC017ACC
:10F1E800F5D1B9F1000F41F0C980142E7DF491AC2E
:10F1F800F7F7DEF9029BDFF86481D4F81851C01ADA
:10F20800A8F80200FDF785BCD4F81C714B4B4C4A9A
:10F21800DFED4C7AD2ED008A4B4AF9000B44F8EE48
:10F22800688A9B8809EE103A643BC82BA8BFC8239C
:10F2380068EEA78AF8EE497A782BB8BF782368EE8B
:10F24800A78A07EE903A3944B0EE680A02EB8108C3
:10F25800B8EEE78A21F0D0FCB8EEC99AF0EE409AF1
:10F26800B0EE680A21F02AFC38EE097A79EE487A7D
:10F2780028EE098A67EE877AB7EE006A88EE277A61
:10F28800142EF8EE007A77EE076A60EE277A89EE98
:10F29800A67A77EE065A36EE477AC6EE256A67EE04
:10F2A800A67A27EE267AC8ED006A88ED047AC8EDBA
:10F2B800026AC8ED017AC8ED037A01F06384234B32
:10F2C800194A013783FB073CACEBE77C0CEB4C0C91
:10F2D8000135A7EB0C0C1678C4F81851C4F81CC1FA
:10F2E8002DE71B4A32F91350FEF71FBF184A32F9AF
:10F2F8001380FEF70EBFF7F75BF90B4B02901E78F1
:10F30800142E05BFDFF85480D4F81851D4F81851DA
:10F31800A8F80050FDF752BB76EE665AFFF749BBD6
:10F32800D03A0020AC27002054610020BC270020E0
:10F33800E83A0020783C0020683C0020E83C0020A7
:10F34800BC4D002027D4D236504D00205655555577
:10F35800C85F0020CA3A00202C28002058610020ED
:10F36800D54BB6F906101A6802B111609B69B6F957
:10F378000820002B7EF49FAFFEF79EBFDFF8808346
:10F38800002538F9023B00EE103AE8B2B8EEC00AA0
:10F3980001351EF05FF9042DF3D10495FEF7D9BFAE
:10F3A800DFF86083002538F9023F00EE103AE8B232
:10F3B800B8EEC00A01351EF04DF9062DF3D1ECE781
:10F3C800BE49BF48D1ED007ABE4990ED007A097870
:10F3D800C4ED637A84ED647A002901F0CB8277EE7C
:10F3E800676AB948C4ED617AC4ED606AFF21D0ED5F
:10F3F800006ADFEDB67A84F89411FDF725BEB449AA
:10F408004B69002B3DF4F5ACB248B34B008893FB35
:10F41800F0F00B684FF0010E186081F811E0FDF76D
:10F42800E8BCAE4EAE4F96ED004A96ED057AD6EDA5
:10F43800014A96ED066AD6ED046A96ED035AD6EDB2
:10F44800025A67EE897A07EB8503A4EE277AA4EEC1
:10F45800A76A66EEC76AA5EE476AE5EEA76A20EED8
:10F46800070A86ED056AC6ED066A83ED007A29EE7D
:10F47800088A21F075FB69EE288AD6ED0E5AD6ED7A
:10F48800176A96ED091AD6ED121A96ED0F5A96EDEF
:10F49800187A96ED0A2AD6ED132A96ED0D6AD6ED5E
:10F4A800167A96ED0C3AD6ED0B3A96ED154AD6ED4E
:10F4B800144AE1EE085A002207EB8503E8EEA16A38
:10F4C80000B2C4F80421A2EE085AC4F80821C4F80E
:10F4D8000C21A8EEA27A26EE656A67EEE67AA3EE1C
:10F4E800655AA3EE886AA6EEC47AE8EEA47A86ED99
:10F4F8000E5AC3ED205A86ED0F6AC3ED406A86EDB9
:10F50800177AC6ED187AFEF7C5BD71494A69002A0F
:10F518003DF4A0AC0A6813604B74FDF79BBCBBF9C3
:10F528003C30CBF8242007EE903A0122F8EEE77A37
:10F53800CBF86C30CBF888200023012ECBED1F7A56
:10F54800CBED1E7ACBF8803001F07682AE427EF4A5
:10F5580093A9BBF93E30CBF8703007EE903A002201
:10F568000123F8EEE77ACBF82820CBF89C3000236B
:10F57800012ECBED247ACBED237ACBF8943001F031
:10F588005F82AE427EF4AAA9BBF94030CBF8743052
:10F5980007EE903A00220123F8EEE77ACBF82C2008
:10F5A800CBF8B0300023012ECBED297ACBED287AA9
:10F5B800CBF8A8307EF4C4A99FED448A032F39D034
:10F5C800B9F1000F09D007EE909AF8EEE77AF4EE59
:10F5D800C87AF1EE10FA01F10A83424ADBF8743076
:10F5E800126894F82011A8F8060003EB550393FB62
:10F5F800F5F50023CBF82C5093621363D36231B135
:10F60800394B1B8823F40063002B7EF49BA9374BEE
:10F618001B6813F4003341F0078235491A46C85C69
:10F62800012803F10C0300F042850132152AF6D1B6
:10F63800FEF788B9B0EE480A21F092FA00B2BFE7A7
:10F648002C4B187800F00107002F7EF49CA8FEF7D9
:10F6580094B82949DFED297A0968C4ED4C7A11F08C
:10F66800805840F03C8513F4800800F0DA824FF0AF
:10F678000008B6EE007A67EE877AF4EEE75AF1EE04
:10F6880010FA48BFF0EE675A40F12985C4ED665A72
:10F69800FDF722BF74EE677AB7EE007AF4EEC77A08
:10F6A800F1EE10FAC4ED4C7A41F36A8184EEA77A40
:10F6B8008DED0A7AFDF706BFA4670020D0730020FD
:10F6C80064350020806A00207835002000000000A2
:10F6D800D8600020F060002020A107006C3D0020C9
:10F6E800E83A0020385E0020387800209033002067
:10F6F800B03C0308EC5F00202C780020000000805C
:10F708008673002082730020BCF1000F01F0168080
:10F7180091ED006A9DED0A5AAE4B25EE866AA5EE7C
:10F72800076AB0EE675AA6EE265ABDEEC56A16EE0F
:10F73800107A16EE106AAF42A8BF2E46B842C8BF6C
:10F74800064606EE106AB8EEC66A012A83ED006A1C
:10F758003EF419A891ED046A9DED0B5A25EE866AD0
:10F76800A5EE076AB0EE675AA6EE265ABDEEC56A40
:10F7780016EE107A16EE106AAF42A8BF2E46B842AF
:10F78800C8BF064606EE106AB8EEC66A022A83EDBE
:10F79800016A3DF4F8AF91ED086A9DED0C5A25EE2B
:10F7A800866AA5EE076AB0EE675AA6EE265ABDEE3F
:10F7B800C56A16EE107A16EE106AAF42A8BF2E463A
:10F7C800B842C8BF064606EE106AB8EEC66A032AF3
:10F7D80083ED026A3DF4D7AF91ED0C6A9DED0D5AA9
:10F7E80025EE866AA5EE076AB0EE675AA6EE265A97
:10F7F800BDEEC56A16EE107A16EE106AAF42A8BFC3
:10F808002E46B842C8BF064606EE106AB8EEC66A6B
:10F81800042A83ED036A3DF4B6AF91ED106A9DEDBD
:10F828000E5A25EE866AA5EE076AB0EE675AA6EE6E
:10F83800265ABDEEC56A16EE107A16EE106AAF4269
:10F84800A8BF2E46B842C8BF064606EE106AB8EEF4
:10F85800C66A052A83ED046A3DF495AF91ED146AF2
:10F868009DED0F5A25EE866AA5EE076AB0EE675A37
:10F87800A6EE265ABDEEC56A16EE107A16EE106A86
:10F88800AF42A8BF2E46B842C8BF064606EE106A69
:10F89800B8EEC66A062A83ED056A3DF474AF91EDA9
:10F8A800186A9DED105A25EE866AA5EE076AB0EE35
:10F8B800675AA6EE265ABDEEC56A16EE107A16EEFF
:10F8C800106AAF42A8BF2E46B842C8BF064606EE29
:10F8D800106AB8EEC66A072A83ED066A3DF453AF8C
:10F8E80091ED1C6A9DED115A65EE865AE7EE055AB0
:10F8F800E5EEA67AFDEEE77A17EE902A9542A8BFC4
:10F9080015469042D8BF284607EE900AF8EEE77AE7
:10F91800C3ED077AFDF737BF012A41F38D8007EE63
:10F92800101AB8EEC77AC7EE876AB1EEE68A032FD7
:10F9380015D0B9F1000F09D007EE909AF8EEE77AE2
:10F94800F4EEC87AF1EE10FA01F15181DBF86C306F
:10F9580003EB550393FBF5F3CBF82430F6E5B0EE53
:10F96800480A21F0FDF800B2E3E7012A41F3688074
:10F9780007EE101AB8EEC77AC7EE876AB1EEE68AC4
:10F98800032F15D0B9F1000F09D007EE909AF8EEC1
:10F99800E77AF4EEC87AF1EE10FA01F12881DBF883
:10F9A800703003EB550393FBF5F3CBF82830E8E50B
:10F9B800B0EE480A21F0D4F800B2E3E7012A7FF755
:10F9C800FBAD07EE101AB8EEC77AC7EE876AB1EE3C
:10F9D800E68AF3E590730020974B1B88DF0540F11A
:10F9E800D787964B964A93ED017AD3ED006AD3ED0B
:10F9F800027A944B0793BDEEC77AB3F906E0924BAF
:10FA08000193FDEEE66A17EE103AFDEEE77A118BE8
:10FA1800ADF82A3016EE902A17EE903AADF8282065
:10FA2800ADF82C30894A8A48B2F90230B2F9002080
:10FA3800884DD0ED007A9FED887A88484FF47A7621
:10FA480003F5E16306FB03F302F5E16206FB02F24C
:10FA580085FB03761E44DB1785FB0275C3EBE623A3
:10FA680077EEC77A079E0078378806901544D21734
:10FA78003046C2EBE522FDEEE77A35467688AD885A
:10FA88008446A3F5FA73761A0089ADF8403017EE6C
:10FA9800903AA2F5FA72ADF83260BCF80E60ADF893
:10FAA80042206D1A401ABCF80A20ADF82E30BCF876
:10FAB8000C30ADF83450ADF83800751A0698684E19
:10FAC800ADF83E50AEEB010E7F1A521A5B1A0021B8
:10FAD800ADF836E0ADF83070ADF83A20ADF83C300E
:10FAE80031607160B160F160002801F0CD805D4B3C
:10FAF800DFF87C815C4FCDF820B08A46994609949E
:10FB08003CE012AB03EB440030F9200CA9F80000EC
:10FB180098F902E001230D4403FA04F4534B57F813
:10FB280025501EFB00F083FB003EC017039B2C42B0
:10FB3800C0EB6E100CBF01244FF0FF3498420EDB6F
:10FB4800059B02FB03F2494B83FB0253D217C2EB1E
:10FB58006313A3EB0C031BB28342A8BF034636F81A
:10FB6800112003FB042326F81130069B0AF1010A31
:10FB78009A4508F1070809F102097BDA98F80600A6
:10FB8800002837D198F8001098F9052005924D0003
:10FB9800681807EB800098F90430C288808898F8C4
:10FBA80003E098F80140121A92B2304802FB03F3BE
:10FBB80080FB03C0DB17C3EB60134FEA520CA3EBC7
:10FBC8000C031BB20393BEF1000F9AD012AB03EBE8
:10FBD800440BB9F900003BF920BC584513DA8644B8
:10FBE800704503DCF3455846A8BF704600B2A9F833
:10FBF80000008DE71630C0B21EF094FE0028C1D177
:10FC0800A9F80000B1E783DDA0EB0E0EDE4503DBAB
:10FC18007045A8BF704683460FFA8BF0A9F800001C
:10FC280076E7B6EE007AF4EEC75AF1EE10FA3FF72F
:10FC380020ADFDF751BC00BFB85900205862002024
:10FC48005C4F0020C85F0020CC4D0020BC5900202C
:10FC580090730020C5B3A2910080BB4428640020A3
:10FC68008073002048290020506600201F85EB5132
:10FC78002C640020DDF820B0099C97F90A0033882D
:10FC8800634A644910FB03F3F87A097882FB03524C
:10FC9800FF284FEAE373C3EB621200F0E683814268
:10FCA80040F2E383079B33F9100097F916507388E5
:10FCB80010443080564AF87D15FB03F382FB03524B
:10FCC800FF284FEAE373C3EB621200F0CB83814253
:10FCD80040F2C883079B33F9100097F92250B38884
:10FCE800104470804A4A97F8230015FB03F382FBFF
:10FCF8000352FF284FEAE373C3EB621200F0AF83AD
:10FD0800814240F2AC83079B33F9100097F92E50DB
:10FD1800F3881044B0803E4A97F82F0015FB03F390
:10FD280082FB0352FF284FEAE373C3EB621200F031
:10FD38009383814240F29083079B33F9100097F92F
:10FD48003A5033891044F080314A97F83B0015FB4C
:10FD580003F382FB0352FF284FEAE373C3EB6212FB
:10FD680000F07783814240F27483079B33F91000D7
:10FD780097F94650738910443081254A97F847000F
:10FD880015FB03F382FB0352FF284FEAE373C3EB2F
:10FD9800621200F05B83814240F25883079B33F97B
:10FDA800100097F95250B38910447081184A97F897
:10FDB800530015FB03F382FB0352FF284FEAE3735A
:10FDC800C3EB621200F03F83814240F23C83079B01
:10FDD80033F9100097F95E50F3891044B0810C4A4A
:10FDE80097F85F0015FB03F382FB0352FF284FEAE5
:10FDF800E373C3EB621300F02383884280F020830F
:10FE0800079A32F910201344F381019BFEF774B965
:10FE18001F85EB5168490020D1ED004A9DED0A4A43
:10FE2800B54B65EEA44AFDEEC53AE4EE074AB0EEDE
:10FE3800674AA4EEA64A13EE900AB4EEC46AF1EE3D
:10FE480010FAF0EE444A88BFF0EE454AFDEEE44A67
:10FE580014EE90EA14EE906AAE45A8BF2E4670459F
:10FE6800C8BF064604EE906AF8EEE44A012AC3EDDC
:10FE7800004A3DF481ACD1ED044A9DED0B4A65EE94
:10FE8800A44AE4EE074AB0EE674AA4EEA64AB4EEE6
:10FE9800C46AF1EE10FAF0EE444A88BFF0EE454A23
:10FEA800FDEEE44A14EE90EA14EE906AAE45A8BF5F
:10FEB8002E468645B8BF064604EE906AF8EEE44A38
:10FEC800022AC3ED014A3DF457ACD1ED084A9DED35
:10FED8000C4A65EEA44AE4EE074AB0EE674AA4EE7F
:10FEE800A64AB4EEC46AF1EE10FAF0EE444A88BFAE
:10FEF800F0EE454AFDEEE44A14EE90EA14EE906AFC
:10FF0800AE45A8BF2E468645B8BF064604EE906AA1
:10FF1800F8EEE44A032AC3ED024A3DF42DACD1EDD4
:10FF28000C4A9DED0D4A65EEA44AE4EE074AB0EE90
:10FF3800674AA4EEA64AB4EEC46AF1EE10FAF0EEEF
:10FF4800444A88BFF0EE454AFDEEE44A14EE90EAD2
:10FF580014EE906AAE45A8BF2E468645B8BF064641
:10FF680004EE906AF8EEE44A042AC3ED034A3DF42D
:10FF780003ACD1ED104A9DED0E4A65EEA44AE4EEBD
:10FF8800074AB0EE674AA4EEA64AB4EEC46AF1EE98
:10FF980010FAF0EE444A88BFF0EE454AFDEEE44A16
:10FFA80014EE90EA14EE906AAE45A8BF2E46864538
:10FFB800B8BF064604EE906AF8EEE44A052AC3ED97
:10FFC800044A3DF4D9ABD1ED144A9DED0F4A65EED4
:10FFD800A44AE4EE074AB0EE674AA4EEA64AB4EE95
:10FFE800C46AF1EE10FAF0EE444A88BFF0EE454AD2
:08FFF800FDEEE44A14EE90EA6C
:020000040801F1
:1000000014EE906AAE45A8BF2E468645B8BF064698
:1000100004EE906AF8EEE44A062AC3ED054A3DF480
:10002000AFABD1ED184A9DED104A65EEA44AE4EE5F
:10003000074AB0EE674AA4EEA64AB4EEC46AF1EEEF
:1000400010FAF0EE444A88BFF0EE454AFDEEE44A6D
:1000500014EE90EA14EE906AAE45A8BF2E4686458F
:10006000B8BF064604EE906AF8EEE44A072AC3EDEC
:10007000064A3DF485ABD1ED1C4A9DED114A65EE73
:10008000A45AE7EE045AE6EEA57AB4EEE76AF1EE7A
:1000900010FAC8BFF0EE457AFEF76EBE04230325C2
:1000A00004930220FEF769B98223FCF724BDDFED3B
:1000B000157AFCF7ECBCD4F8245153003DB19818E4
:1000C00001EB80006D784078A842BDF43FAC13444A
:1000D00001EB83010023C4F82411A4F8BE31C4F855
:1000E000C031FDF733BCB7EE007A77EE677AF4EEF5
:1000F000E75AF1EE10FA88BFF0EE675AFFF7CABA76
:100100009073002000000243D1ED004A9DED0A4AA1
:10011000D94B65EEA44AFDEEC53AE4EE074AB0EECF
:10012000674AA4EEA64A13EE900AB4EEC46AF1EE52
:1001300010FAF0EE444A88BFF0EE454AFDEEE44A7C
:1001400014EE907A14EE906AAF42A8BF2E46B842E1
:10015000C8BF064604EE906AF8EEE44A012AC3EDF1
:10016000004A3DF40FABD1ED044A9DED0B4A65EE1C
:10017000A44AE4EE074AB0EE674AA4EEA64AB4EEFB
:10018000C46AF1EE10FAF0EE444A88BFF0EE454A38
:10019000FDEEE44A14EE907A14EE906AAF42A8BFE6
:1001A0002E468742B8BF064604EE906AF8EEE44A4F
:1001B000022AC3ED014A3DF4E5AAD1ED084A9DEDBE
:1001C0000C4A65EEA44AE4EE074AB0EE674AA4EE94
:1001D000A64AB4EEC46AF1EE10FAF0EE444A88BFC3
:1001E000F0EE454AFDEEE44A14EE907A14EE906A81
:1001F000AF42A8BF2E468742B8BF064604EE906ABB
:10020000F8EEE44A032AC3ED024A3DF4BBAAD1ED5D
:100210000C4A9DED0D4A65EEA44AE4EE074AB0EEA5
:10022000674AA4EEA64AB4EEC46AF1EE10FAF0EE04
:10023000444A88BFF0EE454AFDEEE44A14EE907A57
:1002400014EE906AAF42A8BF2E468742B8BF06465A
:1002500004EE906AF8EEE44A042AC3ED034A3DF442
:1002600091AAD1ED104A9DED0E4A65EEA44AE4EE46
:10027000074AB0EE674AA4EEA64AB4EEC46AF1EEAD
:1002800010FAF0EE444A88BFF0EE454AFDEEE44A2B
:1002900014EE907A14EE906AAF42A8BF2E468742C1
:1002A000B8BF064604EE906AF8EEE44A052AC3EDAC
:1002B000044A3DF467AAD1ED144A9DED0F4A65EE5C
:1002C000A44AE4EE074AB0EE674AA4EEA64AB4EEAA
:1002D000C46AF1EE10FAF0EE444A88BFF0EE454AE7
:1002E000FDEEE44A14EE907A14EE906AAF42A8BF95
:1002F0002E468742B8BF064604EE906AF8EEE44AFE
:10030000062AC3ED054A3DF43DAAD1ED184A9DEDFC
:10031000104A65EEA44AE4EE074AB0EE674AA4EE3E
:10032000A64AB4EEC46AF1EE10FAF0EE444A88BF71
:10033000F0EE454AFDEEE44A14EE907A14EE906A2F
:10034000AF42A8BF2E468742B8BF064604EE906A69
:10035000F8EEE44A072AC3ED064A3DF413AAD1EDAC
:100360001C4A9DED114A65EEA45AE7EE045AE6EEEA
:10037000A57AB4EEE76AF1EE10FAC8BFF0EE457A5E
:10038000FEF7A9BA3D4B4FEA88075FEA990801EBEF
:10039000070E03EBCC1C274400F07D8408F1010814
:1003A0004FEA08180CEB08000CF110030EF11001D5
:1003B00007F1100213ED024A13ED035A13ED016A1F
:1003C00013ED047A51ED024A51ED035A51ED016AE1
:1003D00051ED047A64EE244A65EE255A66EE266AEB
:1003E00067EE277A1033984242ED024A42ED035AF3
:1003F00042ED016A42ED047A01F1100102F11002AE
:10040000D8D1A8F11008C4440EEB0801474419F0F4
:1004100003093EF4EEAEBCEC017AF1EC017A67EE32
:10042000277AB9F10109E7EC017AF4D1FEF7E1BED0
:10043000134BB6F90A201B68002B00F0D8831A6012
:1004400001230493FDF789BFB7F95C20DFE4B7F916
:100450005000C3E4B7F94400A7E4B7F938008BE4CF
:10046000B7F92C006FE4B7F9200053E4B7F9140092
:1004700037E4B7F908001CE490730020E83A002044
:10048000A4670020BCF1000F00F01683A9499DED80
:100490000A4AD1ED004A65EEA44AE4EE074AB0EEFE
:1004A000674AA4EEA64AF0EE444ABEF1000F06D019
:1004B000B4EE446AF1EE10FAC8BFF0EE454ABDEE64
:1004C000C55A15EE106ABDEEE45A04EE906A15EEB8
:1004D000103A9E4200F3D983AB42A8BF2B4605EEEB
:1004E000103AB8EEC55A944B012A83ED005A3DF4F8
:1004F0004EA991ED045A9DED0B4A25EE855AA4EEC6
:10050000075AB0EE674AA5EE264AB0EE445ABEF14D
:10051000000F00F0B083B4EEC46AF1EE10FA40F3BD
:10052000AA833046A842A8BF284605EE100AB8EEB6
:10053000C55A022A83ED015A3DF429A991ED085AC2
:100540009DED0C4A25EE855AA4EE075AB0EE674A97
:10055000A5EE264AB0EE445ABEF1000F00F08183AA
:10056000B4EEC46AF1EE10FA40F37B833046A84241
:10057000A8BF284605EE100AB8EEC55A032A83ED37
:10058000025A3DF404A991ED0C5A9DED0D4A25EE59
:10059000855AA4EE075AB0EE674AA5EE264AB0EE99
:1005A000445ABEF1000F00F05283B4EEC46AF1EE7B
:1005B00010FA40F34C833046A842A8BF284605EE07
:1005C000100AB8EEC55A042A83ED035A3DF4DFA899
:1005D00091ED105A9DED0E4A25EE855AA4EE075A6C
:1005E000B0EE674AA5EE264AB0EE445ABEF1000FBF
:1005F00000F02383B4EEC46AF1EE10FA40F31D83D9
:100600003046A842A8BF284605EE100AB8EEC55AE3
:10061000052A83ED045A3DF4BAA891ED145A9DEDD4
:100620000F4A25EE855AA4EE075AB0EE674AA5EEAA
:10063000264AB0EE445ABEF1000F00F0F482B4EE48
:10064000C46AF1EE10FA40F3EE823046A842A8BF29
:10065000284605EE100AB8EEC55A062A83ED055A5B
:100660003DF495A891ED185A9DED104A25EE855A56
:10067000A4EE075AB0EE674AA5EE264AB0EE445AF9
:10068000BEF1000F00F0C582B4EEC46AF1EE10FABC
:1006900040F3BF823046A842A8BF284605EE100AA4
:1006A000B8EEC55A072A83ED065A3DF470A891EDBD
:1006B0001C5A9DED114A65EE855AE4EE075AE5EEA7
:1006C000A67ABEF1000F00F09C82F4EEC67AF1EE3D
:1006D00010FA40F196823246AA42A8BF2A4604EE9A
:1006E000902AF8EEE44AC3ED074AFDF750B81349E3
:1006F00097F916E00B8897F90A20B1F90200104922
:100700001EFB03F3524200FB02F081FB03E21211D5
:1007100081FB00E1DB17C017C0EB2110991AD31A37
:1007200001440344A8EB01011D4431807580FDF7AD
:1007300007BD00BFDC34002090730020BC590020AE
:100740001F85EB5191ED006ADDED0A4A25EE866AC0
:10075000A4EE876AF0EE674AE6EE264ABDEEE46A4A
:1007600016EE103A984200F39881AB42A8BF2B4690
:1007700006EE103AB8EEC66AB8F1000F00F03F83FB
:10078000D54B012A83ED006A3DF401A891ED046A7E
:10079000DDED0B4A25EE866AA4EE876AF0EE674A25
:1007A000E6EE264ABDEEE46A16EE106AB04200F3A9
:1007B0007181AE42A8BF2E4606EE106AB8EEC66A38
:1007C000B8F1000F00F00983022A83ED016A3CF4BE
:1007D000DEAF91ED086ADDED0C4A25EE866AA4EEE7
:1007E000876AF0EE674AE6EE264ABDEEE46A16EE48
:1007F000106AB04200F34881AE42A8BF2E4606EE12
:10080000106AB8EEC66AB8F1000F00F01383032A2D
:1008100083ED026A3CF4BBAF91ED0C6ADDED0D4A4D
:1008200025EE866AA4EE876AF0EE674AE6EE264A6F
:10083000BDEEE46A16EE106AB04200F32281AE42C9
:10084000A8BF2E4606EE106AB8EEC66AB8F1000FD1
:1008500000F0E782042A83ED036A3CF498AF91ED3F
:10086000106ADDED0E4A25EE866AA4EE876AF0EE88
:10087000674AE6EE264ABDEEE46A16EE106AB0421A
:1008800000F3FC80AE42A8BF2E4606EE106AB8EE1A
:10089000C66AB8F1000F00F07C82052A83ED046A75
:1008A0003CF475AF91ED146ADDED0F4A25EE866AD2
:1008B000A4EE876AF0EE674AE6EE264ABDEEE46AE9
:1008C00016EE106AB04200F3D680AE42A8BF2E46A4
:1008D00006EE106AB8EEC66AB8F1000F00F0868224
:1008E000062A83ED056A3CF452AF91ED186ADDEDFE
:1008F000104A25EE866AA4EE876AF0EE674AE6EEB5
:10090000264ABDEEE46A16EE106AB04200F3BF80DC
:10091000AE42A8BF2E4606EE106AB8EEC66AB8F11F
:10092000000F00F07582072A83ED066A3CF42FAFB2
:1009300091ED1C6ADDED114A65EE865AE7EE245A08
:10094000E5EEA67AFDEEE77A17EE902A904203DCF8
:10095000AA42A8BF2A46104607EE900AF8EEE77AA8
:10096000B8F1000F7EF4D8AF019A002A7EF4D4AF1C
:10097000D145B8BFF0EE457AFEF7CEBF77EEC76A35
:10098000F0EE477AFEF731BD5449096811F08058FE
:100990007EF473AEFEF76BBE514B9FED526A93ED42
:1009A000007A514BD3ED003A4D4BD3ED017A4E4BCB
:1009B00093ED014A4A4BD3ED026A4B4BD3ED024A09
:1009C0004A4B37EE237A93ED005AD3ED015A484B48
:1009D000019377EE847A37EE057A76EEA46A77EEA5
:1009E000A57A27EE067A66EE866A67EE867A19465B
:1009F000BDEEC77AFDEEE66AFDEEE77A17EE102A45
:100A00000968CDED036A17EE903AADF82820CE04C0
:100A1000BDF90C20ADF82A30ADF82C2000F1D480BF
:100A2000344A354B0792198BB2F906E0FEF7FEBF48
:100A3000324B1B78032B00F031810023FEF7F1BD10
:100A40009FED2F8AFEF777BF9FED2D8AFEF79CBFA3
:100A50009FED2C0ADFF8C08025EE800A20F084F894
:100A6000D4F81851A8F80600FCF757B82649274AC9
:100A70008E46FEF7ADBB06EE100A2BE706EE100A17
:100A800005E706EE100ADFE606EE100AB9E606EE06
:100A9000100A42E706EE100A90E606EE100A69E632
:100AA000F5F78AFD1A4BDFF870801E78029BC01A9A
:100AB000A8F80200FEF77CBA0AAB03EB8202FDEE57
:100AC000C54A9446474672461249034814EE906A56
:100AD000A046E64628E000BF907300202C78002056
:100AE000307300203333333F3C73002048730020C1
:100AF000CC4D0020C85F00205C4F002028780020EB
:100B0000000000000000C842683C0020AC27002024
:100B100054610020DC340020586100209E45E0EC48
:100B2000014A01F110012ED0D1ED004AB3EC014A87
:100B300065EEA44AE7EE044AB0EE674AA6EEA44A80
:100B4000F0EE444A32B1B4EE446AF1EE10FAC8BF96
:100B5000F0EE454AFDEEE44A14EE90CA664504EE16
:100B6000906A04DCAC45A8BFAC4604EE90CAF8EE2F
:100B7000E44A002FD2D1019C002CCFD1D145B8BF7F
:100B8000F0EE454ACAE74446FCF701BEF5F714FD0E
:100B9000029BDFF80083D4F81C71D4F81851C01AF6
:100BA000A8F80200FEF78FBBF5F706FDA64BDFF8AD
:100BB000E4821E78029B99F80020D4F81851C01ADC
:100BC000A8F80400FEF7E4B9A04B07931946A04B20
:100BD000B1F906E0198B8E45BCBF5242ADF82C200E
:100BE000FEF724BF9B4800F1800EFEF7B8B9012341
:100BF0000493FDF7B2BBA8F80600ABF8B450FCF7BD
:100C0000ACBEFDEEE77A17EE902AB242FFF669AD70
:100C100062E5BDEEC55A15EE100AB042BFF63BAD17
:100C200005EE106A3CE5BDEEC55A15EE100AB0425D
:100C3000BFF60CAD05EE106A0DE5BDEEC55A15EE1A
:100C4000100AB042BFF6DDAC05EE106ADEE4BDEE80
:100C5000C55A15EE100AB042BFF6AEAC05EE106AEA
:100C6000AFE4BDEEC55A15EE100AB042BFF67FAC38
:100C700005EE106A80E4BDEEC55A15EE100AB042CA
:100C8000BFF650AC05EE106A51E405EE106A28E498
:100C9000714FFEF7F6BF7146FFF7B9BB19F074FF4D
:100CA000FCF754BE94F87431002B7CF497A9FCF740
:100CB00082B9DFED6A7AF4EEE7DAF1EE10FA62DC7F
:100CC000DFED677AF4EEE7DAF1EE10FA5BD4654B0C
:100CD000D3ED007AB1EE677AB4EEC7DAF1EE10FA2E
:100CE00054D4B4EEE7DAF1EE10FA88BFB0EE67DA6A
:100CF0005D4BC7ED00BA1B689342BCF6A7A8FDF791
:100D000017B95A4A5A4B10681B689847594B9BEDC4
:100D1000007AD3ED007A584BD7ED006A83ED020AD2
:100D2000564B67EE277A2B4427EE8C7AD3ED007A68
:100D3000534B67EE277AF0EE665AEDEE275A93EDA5
:100D4000006AB1EE467AF4EEC75AF1EE10FA08D412
:100D5000F4EEC65AF1EE10FA8CBFB0EE467AB0EE61
:100D6000657A484B1B78012B02D0192B7CF4ADA877
:100D7000DFED457AB4EEE7DAF1EE10FACCBF0123ED
:100D80000023FCF7ADB89FED41DAB1E7B0EE47DAEA
:100D9000AEE7019E002E7FF480ADD145B8BFB0EE26
:100DA000456A7AE5132B05D1B0EE480A1FF0DCFE48
:100DB000A9F80000B0EE480ADBF81432344898472E
:100DC000214B1B78132BB0EE408A7BF4EBAE1FF067
:100DD000CBFEA9F80200FBF7E5BE019E002E7FF4D2
:100DE000F3ACD145B8BFB0EE456AEDE4019E002EEC
:100DF0007FF476ADD145B8BFB0EE456A70E5019B92
:100E0000002B7FF4BDACD145B8BFB0EE456AB7E466
:100E1000019E002E7FF487ADD145B8BFB0EE456A84
:100E200081E5019E002E7FF415ADD145B8BFB0EE2F
:100E3000456A0FE5019E002E7FF4E9ACD145B8BFAD
:100E4000B0EE456AE3E400BF54610020C85F0020B3
:100E50005C4F0020AC2700205066002000C0F84402
:100E600000C0F8C4DC650020C0650020506500208B
:100E70006465002094000020307300207865002015
:100E8000E0650020A0640020000096420000000001
:100E9000504D002058610020024B1A889B78028038
:100EA00083707047F8340308084B196861B130B497
:100EB0005D68074C642202FB05F2B2FBF1F222806E
:100EC00030BC002018605860704700BF74290020B3
:100ED000144A0020704700BFF0B53B4B5B79012BF3
:100EE00083B03AD0022B0FD0384B00221A805A80A0
:100EF000374B1B78022B05D1344A364B5188128868
:100F000019805A8003B0F0BD334B1B681B01EFD52D
:100F1000FF2016F0EDFC03780A2B51D8B0F902201F
:100F20002E49D31781FB0212C3EBA2039BB207EE3B
:100F3000903AB8EE670A2A4C04F10C006381EFF78F
:100F40007DFBFCEEC07A214A6389CDED017A5380A6
:100F5000BDF8043023811380CAE7224A224B9278DD
:100F60001F4D33F81240A4B207EE904A05F1340049
:100F7000B8EE670AEFF762FB1C4A144910789678BE
:100F80005378FCEEC07A00EB4010CDED017ABDF84D
:100F9000042044F6FB77C3EB033300FB027200FB33
:100FA0000474B2FBF3F2B4FBF3F3B2FBF6F2B3FB5F
:100FB000F6F392B29BB22A866B860A804B8097E743
:100FC0009FED0B0A0023B6E7007800204062002066
:100FD0005461002058610020CC4D00206766666691
:100FE000742900207460002090600020D73E00200B
:100FF00000000000F8B5304D304C31496E79314B6E
:10100000314A324F0420087084F8580000216420CF
:10101000012EA4F85A10A4F85C10397019705960A8
:101020005870118051802DD0022E0ED0A979284AF7
:1010300000230229136084F85E305360936034D03B
:1010400004292DD001290ED0F8BD282204F1080072
:1010500021F097FE4CF250319FED1E0A04F10C0076
:10106000F2F7C0F8E2E71C4A236653609360D3604E
:101070009FED1A0A02F110004CF25031BDE8F84021
:10108000F2F7B0B8282204F1300021F07AFE4CF2D9
:1010900050319FED100A04F13400F2F7A3F8C5E7D0
:1010A0000F4AC4F8A0305360F8BD0E4AC4F894301B
:1010B00053609360F8BD00BF0078002074290020C1
:1010C0002878002060320020406200205662002014
:1010D000205B0020CDCCCC3DD4290020CDCCCC3E13
:1010E000142A0020082A00202DE9F0432F4DD5F8BE
:1010F000A83083B01BB195F8AC30022B02D003B0FE
:10110000BDE8F0834FF020084046294C05F1B009B6
:10111000012655271DF00AFCA0B199F800300BB943
:10112000217891B908F101085FFA88F8B8F1230F26
:1011300004F1010409F10109E1D040461DF0F6FB7C
:101140000028EAD189F80000ECE7D5F8A80050B3F0
:101150000DF1080EAA220EF8052D8DF802108DF85B
:1011600000708DF801608DF80430694655225340B7
:10117000082213F0800F02F1FF324FEA430318BF39
:1011800083F0310312F0FF02DBB2F2D1714502D0DD
:1011900011F8012FEBE7AA2269468DF803308DF88C
:1011A00004200FF039FF89F80060BBE774290020A4
:1011B000FC3403081F4B1878002839D01E4A1389C5
:1011C000FBB11E4A9FED1E6AD2ED026A07EE903A0D
:1011D000F8EEE66AF8EE677A07EE103A77EEE66A1E
:1011E000B8EEC77A66EE866AC6EE877AFDEEE77AD3
:1011F00017EE900A6428A8BF642020EAE070C0B20D
:10120000704710B40F4B54781B88117804FB1032D0
:10121000091B642300FB01F003FB02F3B3FBF0F0B6
:101220006428A8BF64205DF8044B20EAE070C0B2D7
:10123000704700BF5662002000780020205B00202D
:101240000000C842406200202DE9F04F794D81B086
:10125000F5F7B2F9D5F8B8400022C5F8B420002C53
:1012600000F0A580237D052B074617D9216A236945
:101270000B44C31A9342B8BF05F1B8010ADBD5E0AD
:10128000137D052B0AD9136A12691344FB1A002B2C
:1012900080F2CC8051F8042F002AF1D14FF0010BDD
:1012A0000023B9461E46C5F8B43098469A462746EC
:1012B00023E07A6A39693B7DA9EB0204B4FBF1F4BF
:1012C0000134A4B213FB04F3013301369BB2B6B26E
:1012D0003C83FB82984506D2BBF1000F01D1012C63
:1012E0005FD99846BA46D5F8B430013305EB83028E
:1012F000C5F8B430D2F8B87047B3BB68C3B1FC8A44
:10130000002CD6D1396A4846A9EB01019847D0B1E3
:1013100095F81C31002B52D13B7DC7F82490013643
:1013200001334FF00102B6B23A83FB820124D1E7C8
:101330003B6A3A69A9EB0304B4FBF2F4A4B23C8320
:1013400034BBFB8AC6E73C83FB8AC3E72B686A6829
:101350003949013316443C4685E848004F46C1F8F8
:1013600000A0BAF1000F27D0DAF8203095F81C2140
:10137000AAF81640FB1ACAF81C30CAF82090002AB6
:1013800035D1DAF80C30484601B0BDE8F04F1847C7
:101390003B7D13FB04F3013301369BB2B6B2FB82F3
:1013A00098E73A7D062A04BF9846BA469BE72B6821
:1013B000214A01332B60146001B0BDE8F08FF5F7CE
:1013C000FBF81E4B1E4A1F4C11681A68A0EB09005F
:1013D00002EB000E2268C3F800E09042A1EB51112D
:1013E000014438BF1046164A2060116094E7F5F7B3
:1013F000E3F8DAF80C3004469847F5F7DDF8DAF848
:101400002C20DAF82830DAF83010001B9042A3EBD9
:1014100053130344014438BF1046CAF82830CAF8B1
:101420003010CAF82C0001B0BDE8F08F4FF0000B6F
:1014300036E700BF74290020385E0020044A0020EF
:10144000084A00200C4A0020F0B43423184F194AEF
:1014500003FB00F3D2F82061FC58FD18002E6B68E6
:101460004B600C600DDDD2F8B8309D421DD0B83213
:10147000002303E052F8044FA54216D00133B342D3
:10148000F8D10022342303FB00700A720369CB6099
:10149000037D4B72836AC56A046BC2690A615B098A
:1014A0004D618C61CB61F0BC70470122EAE700BF5F
:1014B000F41A0020742900202DE9F041244ED6F8BA
:1014C0002051172D27DC002D3DDDD6F8B83098428D
:1014D00021D005F1804106F1B807013907EB810100
:1014E0003B4603E053F8042F904214D08B42F9D1CD
:1014F000D6F8B8409CB1237D017D8B420ED3154AAE
:10150000002405E052F8043F4BB11B7D8B4206D30B
:101510000134A542F6DA0020BDE8F08100248046BF
:10152000601C80002A1B011F06EB840439443844E8
:101530009200013521F00BFCC4F8B880C6F82051A8
:101540000120BDE8F081E6D106F1B807D0E700BF81
:10155000742900202C2A0020192830D0172807D8F9
:10156000184B342202FB003019B1C3680BB1A3E75A
:10157000704770B5144DD5F82041002C0FDDD5F81B
:10158000B83098420CD005F1B8063346002203E08B
:1015900053F8041F884206D00132A242F8D170BD30
:1015A000002205F1B8069000011DA21A92003144F4
:1015B0003044013C21F0CBFBC5F8204170BD034B0A
:1015C0001868D1E7F41A002074290020385E002042
:1015D00010B54FF4804082B019F03AFA00B30022FF
:1015E000032390F90200009301924FF4E1334FF48A
:1015F000804118F0B5FE0C4BC3F8A80070B101246F
:1016000002221720214683F8B04083F8B14083F8C6
:10161000B24083F8AC20FFF79FFF204602B010BD18
:10162000014BD3F8A800E9E774290020F0B50D4676
:1016300085B006460068EFF741FE95E81800E41A09
:101640000023039324238DF808304D238DF80930AF
:10165000B5F90A30FF2C2246A8BFFF2201333DD046
:101660002B7B002B0CBF3E233C238DF80A30FE2C35
:101670002B898DF80B208DF80C3031DD23128DF87D
:101680000D408DF80E3007273A4602A93068EFF773
:101690001BFE02ABDA190DF10B0100238A4221D1A6
:1016A000002C8DF807300CDD224629683068EFF7F2
:1016B0000BFE2B689DF807201919994216D18DF859
:1016C000072001220DF107013068EFF7FDFD3068BA
:1016D000EFF7EEFD04F1090005B0F0BD2123C4E7EA
:1016E0000527D1E711F8010B4340D7E713F8010BA9
:1016F0004240E2E72DE9FF470024104E07460D4621
:101700009846204601EB0209A246A159A31971B1DE
:101710000A79142A0BD0694618468DE82002ADF8E4
:101720000870ADF80AA08DF80C80FFF77FFFCC346D
:10173000B4F5197FE9D104B0BDE8F0871046002068
:101740007C4B1B7893B12DE9F0417B4B7B4C9B7913
:10175000D4F82451C4F82401013B82B0451B032B6B
:1017600000F2B680DFE803F022709907744A136034
:10177000536093607047D4F83431C31A002B0ADDEC
:1017800000F5C3350022A035114601236E20C4F8B0
:101790003451FFF7AFFF6A4BD4F8A420D4F8A0105F
:1017A00099605A601A6002B0BDE8F081654A664BE4
:1017B000D279DFF8B48133F81220B8F902306348E7
:1017C000B8F9001092B207EE902A40F6E44707FB02
:1017D00002F6C3EB1633B8EE670A4FF47A7606FBCF
:1017E00003F393FBF1F3E366EEF728FFE06ED4ED2D
:1017F000197ADFED576AB8F90210514BB8F900E0D9
:10180000586000FB05F207EE102AB8EEC77ABCEE6E
:10181000C06AE7EE267A8DED016ABDF80420C4EDBA
:10182000197ABDEEE77A07FB02F7C1EB173706FB23
:1018300007F683ED027A96FBFEF684ED187AA6662B
:101840001E6002B0BDE8F0811DF09CF8002847D072
:10185000404B414A1B78B4F82A11D2ED037AC4F800
:101860009C10DB0756D401FB05F207EE902ADFED52
:10187000386A334BB8EEE77AD4ED267A5960E7EE52
:10188000267A1960BDEEE77AC4ED267A84ED257AD2
:1018900083ED027A02B0BDE8F081304B1B6819017C
:1018A00081D5FF2016F024F803780A2B88BF002189
:1018B000234B9CBFB0F90420B0F90610C4F82C11DA
:1018C00088BF0A46C4F830215A601A6099606AE7F6
:1018D0001B4B00221A605A609A6002B0BDE8F0818A
:1018E0001E4B1B68DE06B3D51A4BB4F82A111B78C1
:1018F000C4F89C10DA07B6D5B4F92821184B00FBC0
:1019000002F083FB0023C017C0EBA3100144C4F80E
:101910009C10A8E7FDEEE77A124E17EE900AA0F5AC
:101920007A7202FB02F386FB0306D817C0EB26107F
:101930001044E1E75662002000780020742900205E
:10194000205B00207460002090600020E4290020CB
:101950002FE33E31EC5F002058620020CC4D002088
:10196000D34D62101F85EB51F03200202DE9F34773
:10197000012019F06DF8174EDFF85CA00024CC2789
:1019800008B1022C02D902B0BDE8F08707FB04F8C9
:1019900056F8085015B10134E4B2F1E7C37890F974
:1019A00002005AF8233001950322009201212A46B1
:1019B00018F0D6FC814648B104FB0760CC222946CA
:1019C00021F0DFF9013446F80890E4B217F048FF3F
:1019D000D6E700BF10460020A45503082DE9F04FBC
:1019E0002DED088BBE4CBF4BC4F84C3887B000239C
:1019F000C4F85038F1F7B4FEF0F75EF8F0F760FF86
:101A000008B9F3F7ADFDF4F7F9FA0522B649B7487E
:101A100021F002FA08B1F3F7A3FD94F85438B44D5D
:101A200043F0010384F85438B24B9A78B24B1A70E1
:101A3000B24B1B682B600FF013F901210220F0F765
:101A400091FCF0F771FE2B681F070BD5AC4B1A7A8F
:101A50000A2A07D80123934040F20342134201D0DF
:101A60000EF088FF6420A74EF4F74CFEF3F768FEF3
:101A7000A54ADFF8C4E20023B146985D03F10F01E7
:101A800003F11307314437440EEB000A11F8018FBC
:101A9000B8F1000F05D09AF80CC0C44508BF82F811
:101AA00058C091F80480B8F1000F05D01EF800C0AE
:101AB000C44508BF82F859C08F42E7D1B2F8581028
:101AC00041B104EB800009EB03015165C0F85828CF
:101AD00002F517722033602BCFD12868C0F3801035
:101AE0000EF046FC2B68DE0740F1B8830EF0D0FB09
:101AF000B4F87068854B94F86C081E80002E40F096
:101B0000B383EFF7B3FF824A8249106094F86D28DF
:101B1000003218BF01220A7058B194F86E38C671AD
:101B2000002B4FF02402827114BF11210121F0F724
:101B300033FA0020F4F79EFE774B784803F1300C1F
:101B40004FF0000853F8057C77B313F9092CA1185E
:101B500000EB021691F872E891F8759891F878A860
:101B6000991E11F801BFF34591F802B008BF86F83D
:101B700004E0CB4591F804B008BF86F80590D34542
:101B800008BF86F806A09942EBD1110142181679D8
:101B900056B1567946B1967936B147505979D171D7
:101BA0009979117282F80C8010336345CAD12C20C8
:101BB000EFF75CFF30B12C2282710022C27120212C
:101BC000F0F7EAF90EF05AFADFF87091DFF8708159
:101BD00059F8063C0293002B3AD019F90A6C1423E9
:101BE00003FB06871A460021384621F0CAF8A219DD
:101BF000A9F1030A92F87B3892F87DB803931AF89A
